:020000040800F2
:10000000F8650020CD9C02089D8902089F8902089E
:10001000A1890208A3890208A5890208000000003E
:10002000000000000000000000000000A789020896
:10003000A989020800000000AB890208AD89020806
:10004000D19E0208D59E0208D99E0208DD9E0208B4
:10005000E19E0208B5890208E59E0208E99E0208B1
:10006000ED9E0208F19E0208F59E0208F99E020824
:10007000B7890208C1890208CB890208D58902081C
:10008000FD9E0208019F0208DF890208059F020801
:10009000099F02080D9F0208119F0208159F020880
:1000A000199F02081D9F0208219F0208259F020830
:1000B000299F02080000000000000000E9890208F2
:1000C0002D9F0208319F0208359F0208399F0208C0
:1000D0003D9F0208419F0208459F0208499F020870
:1000E0004D9F0208519F0208000000000000000020
:1000F0000000000000000000000000000000000000
:1001000000000000559F020800000000599F0208EF
:100110000000000000000000F3890208F5890208D1
:100120005D9F0208619F0208659F0208699F02089F
:100130006D9F0208000000000000000000000000A9
:10014000719F0208759F0208799F02080000000055
:100150007D9F0208819F0208859F0208899F0208EF
:100160008D9F0208919F0208959F020800000000E1
:10017000999F02089D9F02080000000000000000F7
:10018000A19F0208A59F0208A99F020890F2000003
:100190001C00000054464C33140020001C001800C2
:1001A000140010000C0000000800040014000000FF
:1001B0001C00000090000000E800000044DA00008D
:1001C00054DA000010F200000300000001000000FB
:1001D0001000000000000A0010000C0008000400DD
:1001E0000A0000000C0000001C0000003C000000A1
:1001F0000F00000073657276696E675F6465666103
:10020000756C7400010000000400000098FFFFFFFF
:100210002B00000004000000080000006F757470DF
:1002200075745F3100000000010000000400000050
:100230007E25FFFF04000000060000006172677366
:100240005F300000020000003400000004000000E5
:10025000DCFFFFFF2E000000040000001300000080
:10026000434F4E56455253494F4E5F4D45544144BE
:100270004154410008000C00080004000800000080
:100280002D00000004000000130000006D696E5F87
:1002900072756E74696D655F76657273696F6E00F5
:1002A0002F00000058D9000050D90000C0D800002D
:1002B00030D80000A0D7000010D7000080D6000082
:1002C000F0D50000E0B50000D0950000C08D000022
:1002D000B07D0000A06D000090650000606500002A
:1002E0005063000030630000A062000088620000DC
:1002F0005862000008620000B861000068610000F8
:100300005061000040190000301100002009000079
:10031000100100000801000000010000F8000000CA
:10032000F0000000E8000000E0000000D80000003D
:10033000D0000000C8000000C0000000B8000000AD
:10034000B0000000A8000000A0000000980000001D
:100350009000000088000000680000000400000019
:10036000AE26FFFF04000000540000000C00000057
:1003700008000E0008000400080000001000000043
:100380002400000000000600080004000600000031
:10039000040000000000000000000A0010000C0033
:1003A000080004000A000000020000000200000033
:1003B0000400000006000000322E31332E30000011
:1003C0000E27FFFF0400000010000000312E352E24
:1003D000300000000000000000000000E80FFFFFF8
:1003E000EC0FFFFFF00FFFFFF40FFFFFF80FFFFF11
:1003F000FC0FFFFF0010FFFF0410FFFF0810FFFFBE
:100400000C10FFFF1010FFFF1410FFFF1810FFFF6C
:100410001C10FFFF2010FFFF2410FFFF2810FFFF1C
:100420006E27FFFF0400000000080000D9C885BE49
:10043000FBE65A3E3C51363ECEC3D63D6C571F3D7F
:10044000B84DBCBD5535CB3DBFDDD2BD33F4243EE8
:10045000F6C804BE712CB83E0536E1BD7948883D2A
:100460004B37F43D43C975BD0FEFFA3D5FA7323EF0
:1004700027025F3E7BC87B3E0274643E12C74C3E3F
:100480004D20B0BEE2F38EBE7E658CBE536A733ED5
:10049000BB3F2FBDA9F886BDB43B8A3E13E3C63DE2
:1004A000ECA3C43D91E8813ED672933E55589B3DE6
:1004B000B9E8DABE999110BED9C7303EC5D227BE81
:1004C0004D39713E5B175CBEE9F1333E94A693BE95
:1004D00032CF433D38A995BECB5781BE60CEC03EDA
:1004E00009F06E3D80BA213E396BA6BE2BAD42BDF0
:1004F00026E68CBE3723E1BDE80F66BEF857A3BCE5
:10050000573E173EFBAB273E0745823EBCF070BE10
:100510006897573EA85860BE35B1B93DA5D815BDFE
:1005200061F72BBEE57A4CBD5EC2973D500EB9BC5B
:1005300030E351BD0DE5363D33A4AD3ECF6A0B3DF2
:10054000AEE475BE6453A53E46A494BEF008033DD8
:10055000B93AA53DC5FD953D3522DD3D509AE2BC39
:100560004CC71D3EABFB9A3E5649983E8CF11D3E52
:1005700008D6ABBE2DB2273E69981BBEEF289B3E26
:1005800068D468BE7CEE1BBE3B5160BEEDEF2E3CD6
:10059000F63065BDA3AF5D3EA98DCC3ECB8017BEC6
:1005A0002219A23D9CB4923E7066853DD29A0DBD43
:1005B0006056713DFE8C78BC1BAC23BEBEAADABD72
:1005C0007E17E73E7C44263EA36EA63DA2EEADBE5E
:1005D000D2F5143D5C62193E292F793E9AAD2F3E2B
:1005E000B74ED83DD8082CBEE2865A3E6BD54B3E5E
:1005F00085CA133E6B1368BDC0597FBEC1C96A3D31
:10060000B982623E4DDE5D3EA8BBEF3DD718393D55
:100610007D9EDB3DC44CC6BD5553C7BD2E51443EE7
:10062000F9E2123EDFBD543D4B8CC43DB02874BB93
:10063000D82A413E57082DBED21E32BE68CC7DBEA0
:1006400036A9D83E1D02023E276AB5BC03568EBEAF
:10065000430C7F3EC518D93DC3CE80BC799AB63EC7
:10066000B64B8F3E96178E3E448F0D3D11141CBC29
:1006700027D56B3E7D3E293DC1AE2E3E9887763D07
:10068000D914B5BC81862ABE8180223EFEA29A3E44
:100690009B4FDE3D500891BD1D5006BE26BBDE3D82
:1006A000C01B953E65A705BE80BEF33DAD6C5CBD2D
:1006B000D01C2EBE122EAABDCAB1833EDD42A73C7D
:1006C000C098DFBDAD09433D5BB0053E6A413D3D8D
:1006D000533042BDC00C8C3E4453743EADAC0CBD97
:1006E000C2E4863E1EB5643D1C081B3E2082423E8D
:1006F000E105C13CFDF2523E44C26E3E8C2F963E57
:10070000877467BEA680D0BD4A3646BEC26AC93E5F
:10071000E4616F3E4474903D722ED93D3E1E1D3EF5
:1007200035FBAFBAD7E1053F5D73B13E251C083EEE
:100730009F868C3E3B7F703D62D2573EB686CA3D57
:10074000FFDA593E44F93D3E5D5255BCFC381C3E33
:100750005613A93DF6592B3D288430BD9857A23D2C
:10076000C366873D661DB7BD8C79073EE891213E83
:100770004B1A143EF2068E3EFD8099BE2F3474BE95
:10078000E237933E6A6F7B3D4D0884BCA6F9813EFB
:10079000FD9A95BD5E998D3EA6B04CBEA20D493E18
:1007A0007674513E6B3204BC474F01BE2B65BF3E91
:1007B000098D61BE7BCAA6BDCB3363BEFD68D9BDC2
:1007C00058BF96BB79111CBE9B1ADCBD73164BBE7D
:1007D0001619813E54AE863D40D38ABEB6C1E73E6F
:1007E000494EF9BD08DDA0BC15F9623E6C10023E11
:1007F000E2A8BB3D390648BECA8E5ABEB0BBC7BED2
:1008000076160B3E753B0EBEB84E74BEF9A0F5BD14
:10081000288F8DBEA2BDD23DA1F77ABE7AB0C43E6C
:100820003589C23EB8B08DBDF2DF1E3E35F33FBC08
:10083000CE245B3E233DBA3EF78FCA3E4321EE3CB9
:10084000DAE9D5BD3E9701BE50A5993DD3D6B43D5A
:10085000B1B408BE1369263E4C2183BDCC212F3E86
:10086000D11F57BEAC26E83C7CCC983ED957533DAF
:100870000F7DAABE2C7F2ABE45B23E3E78568C3EE6
:100880000F1E00BD3E1C2B3E1B0F5DBEDA1D053E3C
:100890004F72D9BC70A9973E1A49F33EC59279BCF4
:1008A00070A084BD9517983EAF63A83ED9C4793D2A
:1008B0003E3F373EC7EB8ABE5AFB8DBD42D5073E51
:1008C00063D09F3E45A2943E9817113E634611BEE9
:1008D000A3C52F3EF357343E63812F3E697A5ABB3E
:1008E00034197B3DB780F0BC4C665ABE3BC5063E12
:1008F000848F113E99B2B5BD4B7E1EBED59E0DBCF8
:10090000E0B97D3EB76B5C3E1E9EAE3E11B35F3ECE
:1009100058FC6DBEE5D6383E6553A03C58C8B33E82
:10092000881EC93DB80641BB5E23093E13F1803ED7
:10093000B6F0143E9108E7BD843364BE17FDE63D72
:10094000345A8B3EF8EF1ABC62385E3EA164C0BDDB
:10095000681EAF3ECFF307BE703EACBD5809703D78
:100960003A153C3EB8CE83BD86A4A1BD30DB523ED5
:100970007D679E3D8FDF5B3E46A05B3E615CA6BD12
:10098000236A663EC22B843E2E05A33D2D60993E10
:10099000432A00BE198B643D9322CEBD42F9A73E87
:1009A0001BDA2F3E75A3A93D36FF3ABE873DE13DD8
:1009B000B5F7593DA11E943EAF66143E74EB03BEDD
:1009C000BE9F28BDC5CD8FBEDD60693D37DAAB3E29
:1009D0007C08B5BDD369CD3E7E0779BDE542813D3A
:1009E000B827513EFD4E663EA234753CC91DD73D29
:1009F000B969373E7163113E5132A43E9DB7C33D84
:100A0000055709BE2162BCBECDE194BE4CB7983EED
:100A1000903C623E4541623E8795AA3E2C9CBD3C7F
:100A20006E7092BE88DDD93D4C75953ED9F5A43CDB
:100A3000AE036D3ECE94B23DDE86BABB2EF5513E7E
:100A40009519D0BD798E823D781DABBC33012B3E0C
:100A50001DED33BED9ED8B3E8B0E7F3EBF679B3CB9
:100A60009353593CE7AF2E3E8A23913E03D27F3EFB
:100A700032C56A3DF1B14F3E9D569F3D922EB63E26
:100A80002D094FBE82C8E83D9AE45ABEF2949E3DBD
:100A900018E06D3D0D3C0F3EE6DC903E04724FBE0B
:100AA000591D273E92439A3E1B7F563EC7433DBD8C
:100AB000A096C33D25EB243D8FEE4B3EF61CA63E93
:100AC000B5DE9A3D9195BA3D279CB5BD2F45A73E11
:100AD000A07F073E5A029D3ED72A9C3E765F01BE0C
:100AE000C2A0B1BD01F7113D71AAAD3D1616FDBD05
:100AF0007E1A97BE476584BD488B943ECBEAA33EE1
:100B00004EF4B2BED36FB1BDA3E9BF3D5420393E10
:100B10001D4A12BE048E803E25A10E3E376900BEDE
:100B20000C79373EED3B7E3E6B12A13CFFB5C03DDC
:100B30002DAEF13D5D953B3EB2BA5B3EDD7EAF3EF4
:100B4000EA1F1ABE2F0689BD94AB623EC216B63E9E
:100B5000364F73BE346A7EBB5380173EF5DB8ABDC9
:100B60007F45843DF59D27BD042C943EB3FF5EBDBB
:100B7000A467D0BD6943933E2DB6EF3E6758D03C85
:100B8000338399BD0FC6823E3AD889BE3A40953E1E
:100B90007F8422BD5EBA3B3D059CD73EBA56103ECF
:100BA00089BE6DBDA783003F19F3053D0F5CDE3C98
:100BB00016C5833D8A5A433E01D9BEBC4EA72DBD02
:100BC0009C201CBE3BA6893E115353BEBAD7A73EFC
:100BD000FA37873DE1A595BCBC49A73ECAE2C6BD30
:100BE00079BA31BDC9A3A53D14AA343EC8230E3C31
:100BF00004F98CBE3014CC3D3C58833EE086BE3EAA
:100C0000682BA0BD48965EBDE5C744BE98E79D3EF3
:100C10005C43AC3EA3FB933ED74D713E39962DBE4F
:100C200095F2C73D1235E13D28C5B43E7A2FFFFF4E
:100C30000400000000080000882F11BE93C820BDEA
:100C4000B78BF83BC68162BEC48C733DA8FF1B3EC8
:100C5000E334203CCFDC16BE4962EA3D972EFC3BD4
:100C6000A52B8C3E76544ABDBBF8183D422EFD3D67
:100C7000A028B3BEF0469DBE4467A7BE8B1DABBC8B
:100C800093C19B3E1C7874BE8561323E1B3754BEB7
:100C900060BA07BEDA264A3C8C1A61BDE1E9293EFA
:100CA0007A4819BE5A4F61BEE3407D3E11605EBE78
:100CB000368770BB40FB2D3EBBB0073E6281A9BEAC
:100CC0009E6C1E3EE135A33E63D3C7BEC957D7BC59
:100CD000B450283DA053843EA5A1023F69AF22BE77
:100CE000310EFFBD57C83E3E15EEC83E87EB393E7C
:100CF000990B583D6423FE3B0A8ED03D0A38CD3E09
:100D00003185B2BD5D178F3E831BFC3DCC2349BEB0
:100D1000A69751BD3CC088BE04D4AC3DE319A0BD2C
:100D20004290A0BECDF4A13D17C23A3EAB1650BED4
:100D3000FB200F3E4BD9D4BEF66B833E7D17373E6A
:100D400017D938BDFC167BBE0445433D3A44063EE8
:100D50001C74653E696386BEC0D48BBCF70BBB3E7A
:100D60001BAB9E3EB46B3D3E36FEC83D927E0D3EB3
:100D70009ACF6C3E5B9EC83D091168BEB3BEAA3CCB
:100D80001F4DC93E298723BEAB50483E2EB2E2BE5E
:100D900017102BBE204B0D3E8AE0133EF80DC5BD4B
:100DA00020792EBEBA98103D6B70B53E753C0FBED3
:100DB0000855983EF74A81BE19FB333E89A781BE8C
:100DC000E0A9D83E0308C8BD8671FD3B222A7FBE3C
:100DD0003056A93EBD00723E633F213D692B663E01
:100DE0006CBBAE3E817CFABC696F81BE7889B0BEB7
:100DF0008C06D2BD362E333E287384BE8C1E863EB2
:100E00008D38CE3E6BA493BD301B013D6A0B9EBE58
:100E100064AE2C3E4148953E1DB3313DDD26E1BE1A
:100E20001E211CBE4EAD55BD559C843D52D579BD8D
:100E3000E1F83E3EF1EB88BD6219443EF8013DBC4D
:100E40009C30263E83C38BBE799B2EBE204F84BE32
:100E500069B4DFBC23780F3E83B9B43D410795BE2A
:100E600009192CBEF4EFBFBE432C7CBE6323393C72
:100E700072A0B9BDDA725FBE469822BED14153BEA0
:100E800009CAC73E319AB2BECB3EE0BD8784AF3EB1
:100E9000C69FAB3D1D4C34BC12416DBE96942EBE18
:100EA000EBF3BE3A141F19BCE6D701BE627A113EBD
:100EB00033862A3EAF1F9EBE6056463E96BB353BEC
:100EC000FC73ECBC6F338EBD6041363EB876CBBE52
:100ED000D8AE003E20052E3DC9437E3E900169BD3F
:100EE000C98306BE190E4CBE9B13FCBD82478A3EC9
:100EF000E38DEBBD082DF43D0977353DC253A0BD10
:100F00001F6DBDBC60EB593EA2789A3EC2F8F0BDA1
:100F1000D98168BD5C33103E2CB22D3EE721A83D3F
:100F2000A2808ABE245D7DBEDC798F3EA85947BE73
:100F30009497A4BE6555A7BE305649BEFD959D3D0C
:100F4000FF4D953E8E1B9E3E229AAEBEEB6E5F3EDF
:100F50005FA380BD0378323E18779A3B93C1C1BD31
:100F60008E60C4BAB3B9D23E7E35DE3E7C38A93D30
:100F70003B25C33D0A6F0DBE4765B63E9A279B3A97
:100F8000A89303BEDE6C783EC0EA0ABEE2DEE83D0E
:100F90006D3BB63E5D7501BEC606F63D2B2A1A3B7B
:100FA0008F38303EAAA80F3E56D7853D429E7DBD64
:100FB0006200C03CF429F7BD3C07883DF82398BE89
:100FC00015EB71BB4A8EDE3E2093DFBC14DFA93DDA
:100FD0006C01DC3DDC7989BE3897193E74A5DDBE15
:100FE0001FF415BD0268A43E74E24C3E8ABF3B3E2E
:100FF000728F8DBDB2D79E3EF212893DC3BB1F3D9D
:101000007DF52EBEA36A913E035E0B3EC277DDBD29
:1010100088EF9A3E11B5513D636CA73E9746D63B8B
:10102000366B013E69D4023E72B048BEFD9AC83D9F
:10103000F954523E5416993E841404BD68910B3DF8
:101040004F470D3DE3A9873E6F031ABD034892BE8B
:101050009437EB3EEBB9603EB73B113EAF2CC63E3A
:10106000E573D13E630B8BBE1B2256BE74EDB2BE40
:1010700018D9BC3E738D743D3522C0BE3C857DBE03
:1010800030FECE3EEF99C9BEDF22FD3AAAF3D1BCB5
:10109000D35B9BBE957C443E806F6B3DA22623BEF6
:1010A000F0A05C3EBF57C9BE477E8CBCE95D00BE68
:1010B000F4A0AA3EB1720D3E3F026FBBB3DE28BE64
:1010C000A89414BE2EFD203BB1F1D63D8B88B0BD57
:1010D00086262ABE11048B3EC03148BEE7596C3EBD
:1010E0005FD457BE4285C7BC8E463FBD2130CABEC5
:1010F00070E6183E52A8DA3C39D05D3D681AC2B994
:101100007854A9BEA75B9BBE8F3933BD2CF6BA3D80
:10111000077D813EB1290CBE4047213D76C1193E75
:10112000512124BEA2E357BE4C521E3E2B9A0C3EC8
:10113000987B473E65F8BB3ED77F773E3811E6BDCA
:10114000142E3C3E184D363E4044F83D8782AA3E60
:101150006ED1373EDA93103E71E3873E73D971BE8C
:10116000AC6E3FBCF1BC0D3F70FE48BE28A78A3D67
:1011700078D3BCBE2F68D4BDC77F2C3ED9B59A3D6D
:1011800038E979BE99ED1C3E4DA7A53D0BD435BE7F
:1011900008CCBABBD5A187BCFB6FEC3EA84A353E54
:1011A000A82983BE5EE3D73EBDE3913E7E2F903CEF
:1011B000E671EF3DEE9C2BBE7994193E8784443E48
:1011C000EF139D3E2E09E6BE608EACBE3AD46CBED7
:1011D0002DF9473E1277103E4DDA78BEAE535D3B97
:1011E000CF462F3E06ED80BE713ED03D03A3ADBE7F
:1011F000B0B3303BB50CCABE3A3839BDB61F6EBE6F
:101200004558C13D1FA2063E7BB5B9BE176EEEBE66
:1012100012F0B93E272F803D31E5ACBD335D053E70
:10122000F7BC273EB134FDBD197D37BEFBA857BEC4
:1012300090D58B3EEA50963E70B5C63D138C36BEB7
:1012400094EF5CBE41F4E0BDD6C4A4BD2B8E0E3E2F
:10125000117D69BEDFC0623E2E036B3D5FC3BCBD26
:101260004F8A523E1953DDBD228C68BE94E4D03EB5
:1012700058E1D7BE5339A73E3ECE6DBE312CB4BE29
:101280003119F73C643F353EDD9F723E3D41973E4C
:10129000B21442BEAFD76BBECBED1E3E6298D6BD38
:1012A000D7F04DBC69A2D8BD9985273E5DFFEABD48
:1012B00071B599BCAB4F953D58178A3E3C74BF3D04
:1012C000BD1B4B3EEA8D08BEC00A70BE61A43BB98F
:1012D0009AE0E3BCF180333EAB62E1BDDA86CB3C01
:1012E00032DE05BE04CED83EC3D3D53E380D333BE7
:1012F0003DC6C43E4D48353D61D96B3EFD7A9EBE2C
:10130000BE8D0CBD39A8BDBCC4A98ABEA08C8FBE41
:1013100025C3893E316396BE3C85C7BDA5B9D7BEFE
:10132000AA48A93E575492BA8F4A013D77F2B23D7E
:10133000CD4F463EAFED73BE802B833CC0F2D8BD8F
:10134000B2D4A73ECB7194BD98928E3D97CC803D90
:101350009FC164BED056653E5326C73D29638F3D6D
:10136000B3BEB73E86F4C53EE40A3D3E3E5FBA3D9D
:10137000CD6F113E70AA6C3E992DFBBD7267EFBB1D
:10138000DE8AB3BD27A2823D298EA93EB5BE2DBE01
:1013900016F8C83D8AC285BD8609A93D9B7946BD20
:1013A00031A8B03EF35F3E3E79D14FBE24582CBEEB
:1013B0002136F13D0990ADBEFFCD3DBE2D8936BE33
:1013C0009C858B3EB55924BE302114BEA4A27FBE9D
:1013D00033641D3C546165BE8C93D4BE0B4C8B3E74
:1013E00003AC99BC6FBD513E85847C3D63B55CBE4A
:1013F000CC018D3ECA782F3EB8BC81BDA9E9C3BDE2
:101400001375D43D0249193E6A3EA4BE0890D0BE71
:10141000B414803EA1EBB93E8FE771BDD285BABE50
:10142000057FC9BC1CC0863D6B74833E8E89333DED
:10143000B7ABCB3DCE7C893E8637FFFF0400000072
:1014400000080000F897793E60A3EDBDEEFF8BBD6C
:1014500001BFD43E36AAA8BD8E0A953D36DA183DA6
:10146000E4CE80BE570AE23ED753BA3E40C7D0BD55
:101470007743413E7A6D10BE1A2063BE0A7BD23E8E
:10148000794F873E7F15E93EF575973C53F4D13E81
:10149000709C9E3E49E94B3E399E463EEE9B153E72
:1014A000A2C5753ECD5839BE5F98103ED74EBCBD23
:1014B0005F3242BE3E5A02BE10917ABD1B9760BE9B
:1014C00048EDB43E1673C53CFF9CB0BD595273BE87
:1014D000B54273BDF3EA243C27C8F1BDFD17E73CD4
:1014E000AB6722BE7C313C3E6BF8ADBD35CE33BE22
:1014F0005B54BD3EC5BEDDBE17F92C3EF09D503E8F
:10150000BB74AD3E8EE9A4BE613C42BEF2166CBD1A
:101510004AF677BE5201213E2CDE34BE3A5D823E51
:10152000A008513EB77CA0BE1E89F13C2B6CF73C55
:101530006EF06EBE9FDAE43D7CCF713E544952BEE0
:101540009D5489BE721262BDC67AC83EBADB7D3E2A
:10155000A8CFE1BD85AD20BEE7B041BE30E491BE6D
:101560009A5A88BE1A04B43E3D0017BE8620B8BE03
:101570001A062BBE4D3A9EBE272BC2BE0735A23C93
:101580006B4A94BE69DDECBDE70B9EBE18AE6E3EA5
:10159000FE4EE2BDAB9E913E871F81BE447A5ABE8D
:1015A000E75406BE4AA366BE202C3E3E7A0705BD20
:1015B000E0282A3E7D0E743E85E6A23E78E9C6BE4E
:1015C000BCBC54BE8B39863CF1FC78BEDC64853EE5
:1015D000E62399BE4F3C7F3EAE14953E3D836C3E64
:1015E0007CE8813D770D7BBE56DA9EBEC18B80BC08
:1015F00053299BBE5ADD323E5D6A3ABCE3DC9D3D19
:1016000075B955BEE07A233EB5EC37BEA27C9DBECF
:101610002C6F9FBE740EA2BE76CAA8BD2E0DA93E29
:1016200029A8EBBE5BE291BEE680A6BDA42F713E69
:1016300012F6A3BE3C2504BEE8380A3E7AAEF3BDDE
:10164000CE643F3E7395883E9DFEA8BD43CE9DBEB1
:1016500012B79F3EB2B18CBD3DB2BDBE93FA29BE5A
:1016600095118ABEB33C34BEA34B18BE4402403D24
:101670000572243ECD45C2BC431EB6BE740186BE73
:1016800095AD1C3EBFA6B33DBBAA5F3EF0C1D63DA3
:10169000D0DC83BEF8F193BE42F135BE9B036CBE35
:1016A000C871753E3E4B223E008202BEC1128DBE05
:1016B0003B7DA23EBDB15FBDBD67BEBEBDCFC7BE57
:1016C000467510BD50C0C43D22A4DABC5B7FEDBBA3
:1016D000D1957F3DB1079EBBDEB4843E88927BBD31
:1016E0008D49A43E0C160CBD46EBF03A2FBD4D3E85
:1016F0007DA9A5BECDA32C3EEA2A15BD87B480BE28
:101700002B9D463E9C7D8B3C22B900BE1CAC263EE8
:10171000D9AE573EB68C84BE7AE292BE21AC733D00
:1017200061972B3EA8A0C1BE1D0FD73D2A9F113E39
:10173000317F813E75AD0ABDD00A0A3E909FF93CCB
:10174000A655543E46B27B3EE34B7F3EFA6EBE3E0C
:1017500049D289BDFF579CBE2FCB34BEF76BAD3D40
:101760005BE9953E1082B7BEE311E43D3A124B3D72
:101770003273E4BD716EC33D9396633D2CDE903EA3
:1017800047A8623E2278A6BDF2B5A2BEF0B6873E5B
:1017900033781FBE507698BEF2413C3E00F30CBE3B
:1017A0006F3197BCD0DB93BE42A48EBD14D34FBD26
:1017B00095BBFEBDFBCBCBBE42B5F03D3377E73CDE
:1017C000A59204BE1183853EAAA5A53E5479553E37
:1017D0005B38063EC6C6953DFB86B5BDFBF99ABE95
:1017E000F9A7683E4D6D393E337CCC3D97C714BE9A
:1017F0009CB39A3E381568BD32E6AABE14D7A7BD81
:101800004044943E413CD03E63A0873EFFD4A33E7B
:1018100009DF6E3E5E07DF3EAB7E1CBEF3E0CCBD53
:101820000D0999BBE5768EBEB45E173C58112DBEEE
:1018300068D1BF3D692B6FBE8EA8AEBEF92184BDB5
:10184000E464793D0EDE67BEDC7FA3BE91AAA23DB3
:10185000C33FA03DD1B9AFBE2E7EBABEFA2991BE1C
:101860009765403E4F7E89BEF13A24BD0A7202BEA2
:10187000839ABCBEDA48B9BE19C5BCBEDC16AABD87
:1018800097561E3E31383A3E4FF784BC64F904BE89
:10189000DF3DB13DAE464D3E8857E53D58D150BD88
:1018A00010400E3EADCB3B3EE9280D3D1D13A6BEBC
:1018B00047BE0D3E83EF573E1E75ADBD1386963D68
:1018C0006884FBBDBAEAA93D225214BD3E5CF7BD57
:1018D0007938B33E90026B3E3B61CCBC2C1939BECB
:1018E0001B9860BE6041943E47208CBD606B56BE25
:1018F000E278873E4887163E4C5AA6BE8C67A13ECA
:1019000009B19E3D0156EC3EAF32D33B0A5A2BBE85
:10191000E2639F3E1D274F3E3EAAB2BD0C08C8BEE3
:101920006F5B563D7C58B7BCEC7E4C3E329EE63D2C
:1019300040695CBED19EA0BD69DA8FBD86BC7CBD0E
:101940006A3E223EC3996DBE0323923E21E19B3E37
:1019500026F70C3FF7D4BBBE1C9658BE717F853D61
:1019600040F786BD2C0F66BD42B3F93DB4C6D23DEB
:1019700094B4A93D287BBBBEDD1C01BEE57568BDE6
:101980003538BD3C663B9D3E84B167BECDDD8D3DA7
:101990009608D63EEC165E3ED1A24BBDE910F43D52
:1019A000D30D99BDA0D25F3E00A9BF3DBA3F013D16
:1019B000C404243E1FDD62BE6715FFBE6160FCBD2E
:1019C000FAB29C3EB1FD753D4405CCBEBC38B63D77
:1019D000776D1A3EC167A73E4413AA3E69F7363DAC
:1019E0008C7349BE278A93BEA32B5EBE94CF88BE5C
:1019F00069FF44BEAD94A53E6F8426BC3B6390BE98
:101A0000288FA8BD9D01B8BE5C79623EA13180BE21
:101A1000651558BE6C61C2BEC0692ABE7F8A963BFE
:101A2000442EB3BE069C1CBE592F87BE45C93B3E03
:101A30008D38BD3EF82C883E5F7F3E3EA6D75DBB0D
:101A4000EA2A17BEACA21ABE230B993E68C68E3D89
:101A500015FB813E03F49B3D0AA4C43CAA42A43E6C
:101A6000D6CDCB3C5E4EBDBDD9574BBE972AA6BE48
:101A7000CFF407BE5A3F10BDE4C5CD3B45735C3E75
:101A80001BD5993DF1CB613D7A264E3D9773863E3D
:101A9000B44E88BCD402B63C9FF691BCAB192B3E29
:101AA00056A5E8BD9F52B33E4F108F3CF40A8ABE44
:101AB000CE9C8ABEED1311BD1513B8BDC593D1BE22
:101AC00068A8AC3CFBC642BEA314513CBCCC983EBB
:101AD0001E281A3E8D6B143D137019BEA980863ED8
:101AE000F52100BE4E8AAC3E2181043E080883BE2B
:101AF000D8C68B3E0D11973E90A58FBECDA4CCBD10
:101B000030FD053CDAC6923E43524CBE45059D3D34
:101B10006FFBD9BC4BA578BA996D9D3E6C27713E81
:101B2000583684BD7AE89C3D8BC56D3E0D6DC53D34
:101B30001189B43E9F096C3EC550E8BDB55E83BEB9
:101B4000639500BE39B2FCBB7D11963ECBF6ADBEAF
:101B5000C34E493ED022ACBEA1219F3C587F48BE17
:101B60001316D0BD9634DFBDD04BA93D39CE5DBD37
:101B7000A2B6903C481EA8BE775B3BBE49C950BE8A
:101B800081647C3E2F19883E4D49CFBD2AB68A3DDF
:101B90009E78B6BD17357B3D8675C63D1827C63D78
:101BA000401A3E3ECF55353D766E493D40B915BD94
:101BB000A338AEBD59C851BED7F3D73D3B83FC3CDB
:101BC0006D9FD9BD3CFC71BE36CB4DBEE66553BEA4
:101BD0005C5B35BE03BCCE3E7E4BC23E1670B1BDD3
:101BE000F28ADEBEA97C703D9CC273BEA6612D3E0A
:101BF0006DBB56BD74ECB83E7C9762BD076115BDE8
:101C00006E169FBE7911C83DBF029BBECE08643DD3
:101C1000647986BD9C8FAF3D85A36EBD669B023FF8
:101C2000E78B87BE3FBE903EFC0AA1BE5F45F13EFA
:101C30003B8BDBBDE3D5653E4B592CBD6CA153BE40
:101C400067625DBE923FFFFF040000000048000095
:101C50007315623E4EA337BE253DDE3C155C4FBD7D
:101C6000E1FB1C3E72E080BD4D0C343D43BB313E78
:101C70000184A13DFEDE343A7693233E1973A4BD60
:101C800034CE803E2D7C12BDF82E2C3E2B0A323EE7
:101C900054C265BDABFAD03C86EF443DBFFB223D4C
:101CA000131B15BD21DBE83DEF09773CE442FCBD89
:101CB000F286873D6F422ABDFD40AFBDDF6878BE2A
:101CC0007485CB3C45FF18BE17F6083E2744253ED9
:101CD00093B5F5BDA399CBBDE68B68BE0D08EEBDEF
:101CE000B1025ABD4E9934BBB30FBFBBB4AC0FBDEC
:101CF000D6FFB53D2AA41D3E5A4552BE9C575ABE3A
:101D0000644932BEB4D2533D3E6222BE3E04C6BDDB
:101D1000A36D4ABD0D0F5EBE38368CBEC7DD75BEE5
:101D20004C6737BE3C05983D826D48BE66E352BCA9
:101D3000AFB6283DBC160CBCF1AB76BE54232A3D91
:101D4000899E76BEDB7A38BDC6D4283B6055393CC7
:101D5000D17616BE45351EBE79846DBE4978A4BEC7
:101D60000B9CACBE0624C03CE89B933D7AFED03D64
:101D7000D2AB403E2BDC673D9F9C52BE01BBC33CB7
:101D800088CF553BB05D8C3E9806CEBD17CB47BD86
:101D90002BBB143EEE5043BE8B95A73C5EF5A7BD12
:101DA000BC65413E7C335F3E93CF70BEC3BE833E75
:101DB0001AF54E3E79AB76BEE63CF8BDC536EABDB7
:101DC000F3E442BE0073953E77167DBE33611ABDC3
:101DD000443E4EBD7CA393BD7DFF273E063FBFBD65
:101DE0008FC7BEBDE19B5D3DF8FAA33CCBE01FBEB3
:101DF0003E6C3C3D19A22EBE7B11CF3D468BC93DAA
:101E0000E5ECF83D087C4EBC338C55BDF7E5C8BD0C
:101E10009778203EBBC5A8BDEEDB40BE8BE188BDF8
:101E20008443F13CB6E804BD770E6DBEE6E945BDDE
:101E300065635C3CBC3D733C0679EABD16AB00BEF5
:101E400012477DBDD6299CBDC5CF24BE81B2553C6D
:101E5000A6A60A3EA3FD573D580436BE802911BEF2
:101E6000D697893D42A55C3E029C04BDD1D8C8BD31
:101E7000F7970DBE2FB44FBEC7BB483EA0BF0A3E6A
:101E80001637F4BC37282C3E59113DBE62D0023EB5
:101E9000D89AF93C4D6930BD8C2CAF3DF1DC1B3E2E
:101EA00081860B3FD9CD963C1A2732BE2DA41DBE8C
:101EB0002F83883DF85AB5BD1A8241BE91E8A03CF7
:101EC0000382A53E2302633E17CA19BDD881EABD2D
:101ED000AE6C843D52E7293E95219C3D78079DBC20
:101EE000EF95BF3ED1D3673E4A228F3C54B3763D37
:101EF00012E8C9BD7BCDAF3DCC20F9BD13FC1E3E21
:101F00008E718B3E85926B3E8102113E9A1B943DF1
:101F1000E417C4BD167D32BE6A2DFFBD116C8F3D26
:101F2000D687AB3C84385E3E0D392EBE673D873D7B
:101F3000086AD13DCD5A243D14BD63BDB6258CBC85
:101F4000216AF6B91E361D3EAFB4F4BC59AB5FBD75
:101F5000478635BEB56FB13C3F1605BEFAE1413D3F
:101F60000C18473EF394E93CF25952BE2B7D97BDC5
:101F7000AB1A833CA474C5BDD7CF873DE6F1243DA1
:101F8000CBD73A3E30D17B3D51E9943D9F7462BD41
:101F900032A195BDD4EFFCBD70413A3EA05BA4BD1B
:101FA000317F1E3EF3E63F3D261C7F3CE1DEB23D25
:101FB000A6472D3ED1BBE5BDABE5C0BD00A41D3E8F
:101FC000385968BE24B7CFBDE45F543D7706A63DBF
:101FD0000BCB3C3E9C645EBED3B9173E5C4D293EA4
:101FE0009D4790BD9C283ABB3726A33EBE56303E47
:101FF000CB79403E4BD4213B12A83BBD7C278E3D84
:102000005B79F7BD3AC4B4BC48741F3EEFCB93BDB7
:102010005F0DB53D51BCB53D6FBE2E3EEDEEECBB48
:102020005B0202BEF2B5323CBF796A3EB932133E62
:10203000BFF983BDB597EABDBE7CD53C215C3BBEF4
:10204000638084BEE47496BDA181933EBE196B3C4F
:10205000F035CFBD356F333EED0200BE586DA4BDE7
:1020600045B2533D9095BD3D9CFAF4BD378C1FBEE3
:102070003F63023B4C29DDBD42D351BD856E0FBE8F
:10208000BAA76D3C8EE9B23D8834453EF1551A3E03
:1020900035DA653EA924293DF89407BD5514EC3C7A
:1020A0003B6F6EBE48D6293B5F0B4EBDE2F84B3C02
:1020B00008DE3E3DCAF428BDFC804B3EC6D4343E0B
:1020C0000563C3BCCE4704BED7E239BEC420733E0D
:1020D000FC5FC9BD015FE53D9EF72D3E9B39233D69
:1020E000EE0BC9BE7635C8BE90A8743E1FE1243EF3
:1020F00001A2A3BD5CBE243E83D77C3EF3C7463E0F
:10210000FBBCF63C19C5B1BEDD9CC2BBADB394BBF4
:10211000DF10663E1F4E613E0A328CBDFB9670BCDE
:1021200031DD82BBFF5F3FBE8A07BABC3C4B56BD68
:10213000311F16BD16B134BE4FED3B3E0DEFF53DE0
:10214000575C4ABE5B6D87BE66B2613E68DF003E8B
:10215000F9BFD4BDAC0429BB29EE04BE060545BEBB
:10216000560180BEC1D8B7BE0EA729BEF96564BEB0
:10217000694ACFBDBC77093E9EEFC6BDDA6D87BD0B
:1021800004773E3C19A0BABEA9A65CBECD04143E9D
:10219000B0174E3E678DED3C3866063E9D182F3CCD
:1021A000A42127BE6FD6C8BE2B3880BBE05CEABB3B
:1021B00075DF30BE6A0486BDF2AF4E3CE2003CBE25
:1021C00057DC71BDF62727BD665A01BECC29513EAA
:1021D0003B55EA3D1264D0BDABBA963B35871B3EFA
:1021E0008A6AF0BD725514BE1B03B03D09BCD53DD3
:1021F000484DA13DC2A5B13D67D536393E5834BDE5
:10220000231724BE606886BEB1FABC3C6D8B9A3C35
:10221000DB0311BE556833BE061A173EA1A0243E4B
:10222000FD236DBE7FC91DBE06E54FBEF3861BBEF6
:1022300082A8D63DE1B5BA3D326BBFBABC11F3BD41
:10224000A7E498BDBBF8063D8AC2FC3CD779093E9D
:102250003E89063EE643EFBC165B7DBECAF811BE62
:10226000182057BDB5C39EBEF19207BC9FF68BBD2B
:10227000EA7A953B76F9B23D19F78EBD3F3CF83DC1
:102280006FE439BE22CA8E3D1406CF3D7A7FD1BDA0
:1022900099B5153E111C13BD0E0B613D3AB5953D28
:1022A0003A9383BE256764BEB02ACE3D1BCDAA3DBE
:1022B000ECB58A3CE7A8C23D212E54BDCAF622BE29
:1022C0009FF756BE20687CBE8B00A8BD6A4D9FBD9F
:1022D00096998E3E1435CD3DBF8E1C3EF2450B3E89
:1022E00066D9C9BDFEFAEC3D7F8E103E22405BBE32
:1022F00068D1233D98C6163E7ED81ABE792340BECB
:10230000CF3AE53D00F666BD4DDE16BEFE51AD3D51
:1023100004FDAF3E712645BCF78610BEE84A7E3DFF
:102320008A4B133DF67521BE7C5E0BBE904DA3BD5E
:1023300014D0703DDFD106BDABD8A13DB1073FBD84
:10234000FC961ABE74C675BD5F8454BE3F176FBD40
:1023500019A83ABEE7EB5E3DEFEBC2BD8A05243E0D
:10236000BBE31FBE512B67BD9F9DFC3C5E0B80BC39
:1023700000732D3E01E4273E988701BE7EA137BE43
:102380000F7CB03D2ACD22BD474FC0BD38D22FBDF6
:10239000CB89823DAF9921BEE4E90F3EEA8E64BD50
:1023A000124D70BE4F64CA3D35E05DBD03B45D3E65
:1023B00072FFEB3D7242B53DF443313E8C65C2BDC8
:1023C000AAB612BEBBB7063E9B8AB4BD4AD0053E34
:1023D000DFBE69BEC537D4BDE1FAC9BDD1F616BDB1
:1023E000958C3B3E749B353E91DA19BE60104D3E94
:1023F000A1FB09BE3A0022BD8350A5BD8A6D23BD55
:102400000C7887BD9CD938BEDF0C3BBDB752FC3D74
:10241000A2AE0D3ED183393E894C153EB7441F3ED6
:10242000F8D70CBDE26F7FBD31550ABB686D88BD22
:10243000DE162BBEFEBC9A3DAB2615BEFB32BB3D65
:10244000F8BEBBBE57E7523D68E29FBD625343BD35
:10245000EB9EBA3C3AE0CDBD1F141E3D7A38063ED5
:102460001224D7BEDB68953C55E059BE20A5903EAE
:1024700035218D3D4463023E0EA4683EC8999C3DC3
:102480009B627BBE15D186BE0161583DDAF70FBE57
:10249000AA9639BDC8F94DBEA342F1BD0CEEA23CCF
:1024A0000B898BBE4D2B11BED4FA343DE2B04F3DAB
:1024B000BBEA20BE6589A93DD95005BDF6C0ACBDBB
:1024C00006930BBD0AE27ABEBD78E4BDDBCDC2BD8A
:1024D0003050063E0CD655BEC605273E0EC0E13C28
:1024E00021490EBD51E8A3BE73BA5F3B478BAABD1D
:1024F00017E83DBEE7DC053E6B36B5BCB80E023CC6
:102500003B7C65BEAE9BD8BCFA3D2B3D2B0DBEBDC2
:102510004A62EABD5AA00C3E8DBB31BD750737BE7D
:10252000B04982BE3DFE20BE069D173E00165BBC34
:102530001E960CBD4392643EB9E2D9BD05E3B53D9C
:1025400077F01BBDEAB9803C0B7FB4BD453E27BD8B
:1025500058EAA5BDB4C4363EAE99F8BC3A5828BE78
:1025600050C856BDD398803E18992ABD07446FBE07
:10257000DCCCEEBD3CB932BEFA75493D6B074EBEB0
:10258000F682CE3C18B149BC9977ADBD42B984BE44
:1025900005044DBE26FA8A3C930F473C8FD0C23DBE
:1025A0005F33183E8628483D652EE93C3B85313D2A
:1025B00085C467BE0C64A3BB03C8E03D619A143EAA
:1025C0004F48283E59FCA2BDB24BB83DA4528C3DA9
:1025D00052026CBE19FB2F3E6D74113DEB7682BE2C
:1025E000A030533EB6BC623E341FEFBD3DDDEEBDB4
:1025F000EDB188BE50D74EBEDB80273D6C6D8C3D63
:10260000686F02BE15A8F43C5AFC213ED04A2A3E0F
:102610005A8E3DBEA29A673D3F1588BD60A658BD43
:102620008C47763D83228BBD7C3D70BE635B1A3D3B
:102630002008FB3D9A7BEF3D841F5FBE1DDCE03D23
:10264000F0B7DEBC5987DC3D65ECF13B722B6BBE0D
:10265000969072BDF0006CBD29A47DBDF357A13CDE
:10266000BE3B543EAB8FC1BDA12018BD2EA44DBEB4
:102670000708473E24BD64BD3BA7003E218DAA3D0F
:102680008583ED3D18B92CBE7C010CBE4F984EBE23
:10269000DD18813CAE3305BE1658F3BB0FB005BE46
:1026A0006E71FD3D9B9F2CBED4C64ABE79818A3D8A
:1026B000F759243EDD93CBBD2D53E03D07AEE4BC7E
:1026C000038E1ABE65E00F3E91C19B3C17BAE7BD71
:1026D000B168223E6A7D76BB600605BE328A07BDC0
:1026E0002E93F9BDFB0460BEE7BE88BE804B20BDC3
:1026F0002984BE3C264BBEBD2F28B03D98F408BCB3
:1027000055A3DBBDC711B23A3C4B8CBDF440E6BDCE
:10271000C02BF1BD85952EBD46DA45BE724AF13D0E
:1027200064673B3D9375323DCC7A4BBEF051273EFA
:1027300045C90F3DAFBFA2BDB1E7BA3D40F22E3D46
:10274000047A233EDD240F3E8565263D510C0FBEE5
:102750001186BC3DE72F103ECC3E45BD1A301E3ED3
:10276000B9843A3EB33E8C3DA8D01DBEC9140C3A84
:10277000DB46363E92E208BE06491ABED05E1EBE59
:102780003683B83D1E7C9ABD0877EB3D40BED2BD76
:102790009F3780BE35F7EA3D22CFB73D6EFF91BD32
:1027A0001AF9943C5D01513E9FDE73BE73BE673DD6
:1027B00090BC933D16EFBCBDA0E81EBEBFF88BBC1D
:1027C000E01599BDD5710F3E69589ABE3CBD753C68
:1027D00069144FBCB67606BE369961BD2B8796BE8E
:1027E000BF3D8C3D00360EBED516F0BD0B465C3E9F
:1027F000BBF112BE2538443ED3DA22BD458901BE65
:102800008B20253EC4B7B13D900BA2BE0D152FBE47
:10281000400B9D3D1B441ABE90E196BCC26B1A3D15
:102820009CDBAFBD9DDA5B3E744341BE8DD1693EFA
:102830000BDC06BE9674833E0DB9E3BDBE5C3FBEA5
:1028400023285A3E7B8A7A3D69EAB23DC62709BEF3
:102850005A3964BEACACB5BC30DE303D851326BE03
:10286000DB11BA3DC9B5E73DC52889BB2045223DEE
:10287000E0A687BE948B40BDBDB8B9BD1F41A43D45
:102880005C7DFCB9EA64B6BDE79C103EE3FDFFBD8C
:10289000E5CF35BEEF36D6BCB03BBE3D07EF47BEF9
:1028A0009B9AE03B2883EEBC5BC484BD5CA1A33D46
:1028B000EF28A4BDB08D45BE71CCB6BD284AF23D0F
:1028C0001AE0C9BD87530DBE06596FBDB1E1E33DA6
:1028D0008C7F3D3C8C4522BE772AACBD4886FD3DB1
:1028E0006B3458BDEFCEBEBD3C4FBEBD00341A3E6A
:1028F000F87FB3BD6C98FABD29EA213E6DC1673EF1
:102900002CCDBABD3C6A01BD6E4041BE7E2A003E60
:10291000F93A673CB8C511BDEB791EBEF7C9323E26
:102920008DC2AEBEA2F60EBEDAA951BD8E674F3C77
:10293000577F853D284C34BE379D13BD06731C3E22
:102940009B863DBE4E8C2DBE9F6B803C7F052EBE70
:1029500005A7D23C759631BE88301A3E465E553C7E
:102960003F6B4DBEF6F1BF3D61A2B1BB2C5B52BEC9
:1029700008A517BEE78DB93DCA49CE3D3ED45CBE21
:1029800045038CBDF67B11BDEDDFD7BD3A331A3E52
:10299000CCFDB7BDA9B1D13D63C11CBE543ED1BC75
:1029A000F897A4BE3A60503D1860603CECC0003E11
:1029B00094B005BE682EB33D5C2287BE0CE129BEF3
:1029C00048F34FBEFE5E52BD1B54423D37BA353D03
:1029D000296DDF3DBC37AA3DAC4883BEE4615BBED8
:1029E00076B99A3D8E4541BEC232013EE56E993EB2
:1029F000646899BDBA02233D876E18BE5BEBA43DA7
:102A0000D61787BEBD846DBD00A6023E40B19D3D78
:102A10007958DD3C5EC8ADBD891A8D3D9BCC08BEA2
:102A2000E7B654BE0A5567BE1C5F3E3E65BF923E88
:102A30002F7F4CBEF37415BEE27D4EBD36D588BDEA
:102A4000CEB5FDBC707545BE42CB8B3DADE2583E68
:102A5000495EB03D6698A93DABAB183E312127BE1B
:102A60007C4FCABD20731DBD935C373EC136A7BBEA
:102A700043896ABDBF04DABDFA87053EC3144EBE62
:102A80008D888E3DDE9FCA3C18F5043E84540CBDF3
:102A9000C88C95BDBFEA02BC7CC6A53D42CB4B3D70
:102AA000F593E23D1A54423D78A6523E9D4984BDBD
:102AB0004A8C0F3EF7A46CBE034533BE0CC92ABE38
:102AC00093B02C3E9C2D63BEE3E2C3BD734B233E0B
:102AD000E245673E7C76833CEF35963DC7F7F63C92
:102AE0004A63EABD1DE40A3EFFC5673E7B8725BEFB
:102AF000AD4D1FBE14CF713E3720023DE5A4003D11
:102B0000FD4DEABE9F0B8CBE80C3E33D67229EBE97
:102B1000CAEF3C3D8981853D4861313E81F3D83C17
:102B200079DE6CBD5F2971BE388CDFBD460F0EBEED
:102B300044E7763DE3C6AFBDA586E2BC04DCA03D1C
:102B4000002F063EFDA95FBE868F6D3E75E0FCBD81
:102B50005A6537BE6BAB19BE5B4A0D3C03A67CBE03
:102B6000A84B5CBE94191CBEB3B0713D8912173ED0
:102B7000C684823A84A1EFBC15C0033E11F97ABD28
:102B8000AF7A503E6CDFCCBE479EE33C7C5768BDBD
:102B900026C8783D7953E43D97223ABC1B9244BD48
:102BA000DA5B1C3D4E446FBE065587BB8832B33D91
:102BB000759310BEEDB4D13DDE75833DEE91F6BC4C
:102BC000B645803D4767FBBE2E27053EBB17343E0A
:102BD000805E1DBD2144DF3D8D28ADBD19242FBC75
:102BE00070A50C3EA062F1BE9EF5163ECE8E6F3EE5
:102BF000F63003BC34BB44BEB3BD3E3E2875523DE7
:102C00008138813EB2069CBE4B1175BDC8DA7F3C4F
:102C1000424657BDA76EE4BD161F943CE53750BE33
:102C2000BA1A2CBFFF2593BBA287983EB87072BD1D
:102C3000550119BDAA83083EE06F073E8A89E03D31
:102C40008B75ADBEF73EDC3DF872B93C104F803E4F
:102C5000514A103EF35493BD60699BBD1F90D13D16
:102C6000AF847CBEE2C1B9BD96FD3B3C559316BE18
:102C70008E832BBE32ADD7BC206694BC87ADF0BD31
:102C800066802BBE1F1F2CBE5069133EDE58343D9C
:102C9000CAF7723C6E17343AEA85E03DD9DDF2BDE1
:102CA000D2F37BBE6EAD09BED5CE733D5C3922B981
:102CB000F53FEA3D403FB9BDB6B82E3E61CC2DBED2
:102CC000040FBF3DF2E71DBD282D0DBE8F42A33E70
:102CD000FB4D4ABE0B8CCB3DB8E7C43D0F8BF23D9C
:102CE0003DEF1E3D4D0790BB72F3D33DFA098F3E79
:102CF000261F823D3C05A43D5D3FD7BD11352F3DCC
:102D0000BCED21BEFB0F99BD1009C5BDABD822BEDD
:102D1000AD10333DD0F11C3E36B8BFBC996A463E7B
:102D2000FE4CA8BC063158BD0F056CBE92497C3ED6
:102D30002E82C33D440531BEB447833EE425223D87
:102D4000EA5FD1B906888BBD4380843CF3E39DBE26
:102D50006498033E687375BDB10722BE9C8F0B3E1D
:102D6000436D86BD9C9CA5BE9C828A3E36EB173E79
:102D7000CDB305BECBF79E3E0C5377BD970D7EBD00
:102D80000F360F3EF36824BE395DF3BD403C503D25
:102D9000479B89BD30CC193E42419BBBEBD1F73CF0
:102DA000E7D0783E0DBBDBBD3655B5BD8F29A4BD40
:102DB000CD7D093DF350FA3D5B855B3E4139DA3DFF
:102DC000C093D1BD0B8BB3BE0CDD37BE4465183E3E
:102DD000E544563D61F704BE3915843E5E32513EEE
:102DE0006B9E8F3EA42686BE10AE1BBECA42903D8F
:102DF000744FF53DB9D1EFBD31481F3EEA7F8FBD1D
:102E000019F8ABBD9C5CC9BCF62B8B3D6C3CA53C5A
:102E100097783D3D033753BE66125E3EC53BD33DBA
:102E200068266EBD0F2F18BDC003D6BDB8E060BDCB
:102E3000C54006BEF75C91BEE2FA93BDBB58D1BD5A
:102E400063F61FBE4AF968BE50203EBE519FF6BDD4
:102E5000065F82BE9DFA1ABEFA36E03DAE7C3BBDEF
:102E6000506EB8BECAD28BBEEA6D38BDAD6112BD20
:102E70008322893CBE67D2BDF34823BE65112E3E36
:102E8000A63DC1BEA4AF52BEADA794BBEAAA4F3EB9
:102E90008F27083EC400CF3CFD780EBDAD5D51BD0F
:102EA000675AADBB63AE3CBD6970583E9467343E13
:102EB0005C9DC1BD66E346BD2870943CE9E4253EB7
:102EC00028B4A8BD73BA31BE731EA63D8A43D8BDCF
:102ED0000DA28C3C256A313E72CA253E341233BDA8
:102EE000608984BD50FABFBD2B91C83D896AB6BDCB
:102EF0004448323E8AC438BC67EA8C3D246405BE2F
:102F0000FE5D58BE2F39D03D45FC74BCC126BC3D8A
:102F1000A062303E82DC58BBC76817BE9CD8023E18
:102F2000FA79493DB6D8C3BD5EA7D93D4DFFC4BAB5
:102F30002C6C713CCF56913DA80CF13CF44F2DBE4A
:102F4000C23859BD7D10093E07545ABE7F3E80BD30
:102F5000A3B8643E69F8D7BD81BA8C3D1606DE3D44
:102F60003DD717BDB22EE73D4F4FB3BD03BFDE3E89
:102F70003AF288BEADCCAE3EBA71B6BD7FE9133C25
:102F8000E5FA673E3E49053D67C63EBC49873F3E80
:102F90008EFD21BE6A1D2A3E94C799BEC3DE0DBEBA
:102FA0008D43253E69B570BAAC873CBE31ACB7BD28
:102FB0005C0774BDF08599BD7C180DBE866FEE3C34
:102FC0000498EFBD8A2D2B3EB62620BED6B40D3E0A
:102FD000EC322D3E30B435BE70A0F2BC5FD8DABD05
:102FE000E21B4DBD7D5E98BC589E0A3EC9EFE33D95
:102FF000DBFAA5BDC1DBAFBD3AE9173D243AA2BC5F
:10300000B009D83D58AD8A3E01EF163E2D961EBE42
:10301000DF88A23CC1153DBD8F2AE5BD415686BD66
:1030200075043BBD615C293E2A8FB7BDC617283D9C
:103030002B841BBECDA14F3D53AC383D0D516EBE10
:1030400018E9DF3D489B173EBF556A3E133B35BE2E
:10305000C1E984BC96D2F93D1A800F3E38B66FBDE7
:103060005E13823EAD8B913EAB5821BD38C2D7BDB9
:103070000934703DB713D73DC0BD393D13A710BE0D
:1030800064320E3E828D583EFB09843E5AAF0C3EA0
:10309000867DDF3D4B240BBE88A7EC3DBB60E83D41
:1030A00013F8173E0E5F4CBE927F61BEE09450BD98
:1030B0005CAF3F3E991312BE3E5F32BD30257D3D71
:1030C000DCCA0EBE6632723D96CCE03D07A766BEF6
:1030D0005691B43D8B5B81BD6075CD3DCA76773E20
:1030E000119A5CBE081B5FBDE2A6E03DE2CC833EC8
:1030F0003EFABD3DE2687B3D2A49D7BDD27A113EFA
:1031000041A480BE5EB22EBE8D6A3BBE5D49AABDA3
:103110003BE900BE4B8EE0BD773C863D1558383EFE
:10312000BAB52BBE967D56BE40B826BD26341A3E93
:10313000CD28133C1529D9BD70082C3E53C0DBBDEA
:103140005E9B6FBE364114BD7A480E3E272E90BE60
:10315000D284943D44E4123EDAA813BDC764B1BDE5
:1031600004CEE2BD9120223E9CADF4BC41AB103EAA
:103170007CC5623ECE31813C639335BE3F9D20BE0F
:10318000F9C913BE6B0188BDB917AF3D93389F3D98
:103190003C7137BE856F44BE967E4BBE2E8E52BCB0
:1031A0004855B1BE5863603CB428EDBBE0B35B3E0C
:1031B000D8C700BE859DC63C0D3A363E3A4356BE42
:1031C000AD4E1D3FFBE1093EFAB14ABED6EF533D7D
:1031D000D033E83CE092E43D3E8930BE29FCA2BDFC
:1031E00015EA813EACFF213EBE6093BEEDE9B83CDE
:1031F000653AAF3D25A2813DD582203E16624EBD87
:103200008D90A53E1C90473DA21937BE3BB8133D9B
:10321000A7C0E4BD27000ABED42200BE1F933B3ED8
:10322000A94F053E202D183E4AC2BE3D4B83283D86
:1032300084CFE43C4C8E143EAB490D3E8BFAB2BDBC
:10324000D0ADB63D8DDA153ED6639ABDDA7130BE8B
:103250007B68B43D3661A3BD9435C0BD3AB8D0BDDE
:103260001DD04A3EA659E7BC2590EE3DB3B9183CA7
:10327000F9D420BE24118ABC0DE962BDC070293E7C
:10328000FAAB773E4C12E53D71D19DBDE852D53C7D
:10329000CE68D4BC4C5480BDF6A535BE54840BBE5C
:1032A00019FB38BD48C3963D280C9A3E9D6AF7BD70
:1032B0009309EC3DE51B823D864D64BE1C53E9BD80
:1032C000FFE5873E043E01BE14DD82BC37FE5BBED7
:1032D00022FC9FBE6ACFC4BD44434CBEC7C69EBE3F
:1032E000D89AC2BE8875113E3030543D172CEABBC7
:1032F000BA5F5CBE8200393DF5E3163DA8D98B3B31
:1033000077EE76BE209B093D7CAB9BBD2B123C3EED
:10331000C9F6AC3D0286B13D68F7EB3D81C80CBDF6
:10332000BD294EBEDA75F43C3C98A1BEE5D20FBE75
:103330004A00DABD305C0E3D8F0847BE892CDDBBEC
:10334000E3285B3DD6DA173E54F528BD92A26A3CCD
:103350001B2B3F3EC0E389BCE86C3D3E5949A5BDEF
:10336000B11912BE459D253D84C280BEBA2AE13DF9
:10337000CAA94EBD47C457BE2065943C48750EBED1
:1033800011317FBEC5F5803E496B46BEF533AA3D7F
:10339000169FDB3D2712083E4F50663C850C40BE11
:1033A000962041BCB689143E23A88D3C88BB03BE41
:1033B000E072F73C62DDE53DCE1D56BDF0D8A33D81
:1033C0007A91383E0BE807BEB4935D3D8A65993E1D
:1033D00078DFDBBD868EEABD8D31BCBD621596BD42
:1033E0003858273E17924F3CC0EAC03DA710F93D20
:1033F000DDE73B3E8E4AF3BDA89823BC00051C3E8A
:10340000767DE2BD902781BE9092F23DB5FE06BE6C
:1034100022C794BD65A9C23D54E1443D8F6E933DE2
:10342000C4CA3EBDB6AC0EBE1A3D82BD2A6C42BEB9
:103430005BBDF03C70CBD23B63264B3E676A1ABD46
:10344000EB5158BE8F2E69BEF3E9373E20CA33BD1B
:1034500085569CBC81CC343E874511BE02EBEC3BCB
:1034600019CED83CFF5023BD748A8C3E3D270DBE3B
:10347000B77BD33D6BDD603EDEAE313E7B95163EC5
:10348000C1E189BD7A4669BE3676253E86991C3EE5
:10349000645D433DB4EC153E998F7A3D6BC00DBE23
:1034A0003AFEA73DB859933D811832BDD481FB3D0A
:1034B000282595BC71E52FBE016D4DBEE62DCF3D93
:1034C0002A212B3B7A05AF3DD3763B3E54D5503E67
:1034D000383E313D0E3F4BBE1672D9BD90A4B93D6A
:1034E000A60860BE73542EBEFF9FA8BD8A27F83D74
:1034F000E0FDB43E264A1DBECFA9693D3EBD24BEB7
:1035000014BDA0BD3EC26EBEC398103ED589053E17
:103510006D122F3E6F81213E85BC213E572E2ABB66
:103520006874B0BD57EEC3BE43AD37BB1310F8BAD5
:10353000E3DCCD3DBBA2F53D2F9106BDCAFB9ABD94
:103540002E6E1C3D1503DDBE73D8E1BD61DACB3DA7
:1035500054D581BCD3AB78BD2970003EC322233D36
:103560000DCB9BBDC13DA0BEC35746BDA1E1073EEB
:10357000B9E8F83C1518AC3D69B622BD69BF86BDF7
:1035800079BB3CBE2B8FD8BEF09C0D3E7E6F7D3E3E
:1035900007E230BE4F1227BE0E8E183EE561E6BD33
:1035A000CD8D1EBE302AD4BDD7FE113EFC66CC3D6B
:1035B00027A107BE327D683DD1FB46BE9F0B133E5F
:1035C0003DBE96BEB448A5BEC7F25EBDE8D356BBAD
:1035D000345F26BEFE7309BD002F393EE08318BD5F
:1035E000FF012BBC1A7FD7BD810DACBC72ED1D3E17
:1035F000B284AC3DDE09053CD8D79E3D3FAB313CA3
:10360000D4BC8DBEF17377BEFEC52FBE3B0B8B3D88
:10361000629E403E93EB803C4902B23D24D3783D0C
:103620003D6CC3BE8BB432BE8481F0BC7885B43DA2
:103630003DF949BD5A56AC3A735A2B3EB3D438BE05
:103640005A06FC3C932C6D3E3A9782BDAD300ABEC3
:10365000ACB192BDFBF9773D08963DBE52E369BD22
:10366000BF54A0BCFF11A63EBF2C253E7455FF3DA4
:10367000DEE002BE51DA9C3D8E47223D837CC93D8F
:1036800032C6333ECA899A3ED17E963C089CCC3DD8
:1036900029C1D83D7BF54CBE2814D7BD1F0F8BBE6A
:1036A00001B3903D1E0DBEBB4F59373ED9B5B7BDD6
:1036B000F56034BE50B821BE0CB763BE831C03BE98
:1036C000C58E0E3ED1CB28BD51232FBE5CC83DBE5A
:1036D0009F76B4BB473963BD8EFB153D2DB8D3BD76
:1036E000FF3291BCEBBD5EBDE215D93CE3F3F73C84
:1036F000D98A843D906E0F3E5ADF233EFFAB2E3EAB
:10370000F3FEAC3D05FC96BD0FE9CCBB1A22BBBD58
:1037100085947FBE4DF42ABE848078BD0C6DD73D64
:103720003E98813E83D7943E951F14BE866D7D3EA4
:103730007DE16C3C0D9DA6BD99CE723EBFE3B63DCA
:10374000A4C616BEAA5999BD9544B1BD247A633E5C
:10375000BB00923D9EA60C3D2FBC9ABE1A0DDEBD4D
:103760005992123EEE86F7BD7F8AE2BDD0FECC3D77
:1037700071725EBC2FA020BEC72595BE4F829DBA38
:10378000FBEDDEBDABBC193E8AABA3BD0B5E913C2D
:103790006DFF76BD32C8813D289941BECB51853C35
:1037A000350F713C6571A9BC2A488F3D19B8393E67
:1037B000025730BDC338523DDF9442BEE3739ABD19
:1037C00029848C3E97C09A3B8599153EFFDE0A3EC0
:1037D00015AB12BEDC33F9BB7B7118BEB81939BE0C
:1037E000EBC56F3EC6CD7C3EFF2D24BE7B2201BDC6
:1037F0007C9505BE10C4D6BC7F14CE3D402976BC56
:103800003F04AC3DC36A463EFE120EBEAA82E1BD35
:1038100067E38ABE9ED5723BD3550E3EFA7B54BDFC
:10382000C4A819BD0AE4D0BD876A04BEACC74E3C2B
:10383000E53A923CE06451BC55F4163EE413AA3DCF
:103840004BAFB8BD0FF192BDF626C93D983429BEE5
:10385000C27A92BD4F8E903E923B28BE4B41C8BD6E
:1038600002B25EBDC016A5BDC76D1EBC68ECABBC88
:103870002EA798BE7B10BA3DD9AF503D25351CBD53
:103880003966C33D730694BDFD2ACABDF8B225BE94
:10389000C7004CBECAA8353E332C7CBDF54E743DE6
:1038A0003D2A1E3CDE36933B6BC485BE2B5976BE4B
:1038B000D94317BE2A6E04BEAA41833E7EFB1D3E3D
:1038C000FEFC203E67BCA7BEDD3B94BE65EB013C21
:1038D000C93AC43CA26F923DE0D4FABD43E7AF3D84
:1038E0000C9D86BD7E8290BEC46CA23D4686A0BE65
:1038F000120670BE82D5073E6C48223ECED38F3D65
:10390000D067D6BD9B708FBE56BD1F3D3DD67A3D5C
:10391000F2A509BE7608F13D977454BE0682023EB8
:10392000F83947BEA045B73D3F65A13DDE00033EE7
:10393000D97F313E42AC483D9D5F423C7A5C69BED6
:103940004B42013D6AD4C73D60E50DBDC78A06BE46
:10395000698E803BD61826BE19C539BE9EAF0EBEF5
:10396000377F8B3DC881663DDB33853CAC62C73C0D
:103970004A1BB63BB2880CBEBF4A953C8F61F0BD76
:103980009325003EA54148BC870822BE3C8785BEE2
:103990009C1787BC85EF1B3BFF7673BED487A2BD07
:1039A000C51E0CBE910629BE0012D03D6C2572BD0D
:1039B000AADFCDBBE8D9963DC22B23BED65104BEAB
:1039C000A55593BED3FFDFBDC8D7E53C3B8EEBBC0E
:1039D0002CE027BE99FDA8BD8D93FDBDEF10B4BCB2
:1039E000813A16BE324A53BE289066BE2190323EBE
:1039F000ED8A173D00E89ABCE9A212BE3C1023BE36
:103A0000EBAAEFBD25932CBC0E8F57BE531E323E42
:103A100055E1F73D0E2657BC83FF11BE3F54F9BD5B
:103A2000C17F11BDA4ADA93DB3CE623DDEBF9A3DBD
:103A300043C005BE2DCECFBD24746EBB08190F3D0B
:103A40007BA3BDBDD58FFCBDE9B2673D2FF5FCBDA5
:103A50005633FB3C5F2BCBBDBEA71BBEA4600DBC89
:103A6000FE5D263E3CAA1EBE5D023B3E37DC1F3E8D
:103A7000BD0D15BD65AEF0BD61FA0CBC4D03503EE9
:103A8000236168BD1E6136BEDF0E403E5BD22E3E16
:103A90004B5289BE5AAA49BEA7B74E3D6B8ABE3D5E
:103AA0008BCFBCBD398A05BEEF15E73DE2A3843E4E
:103AB0004B6D23BE01CEF63DD4948FBE592111BE6D
:103AC000045483BC7E286D3E5D1FB8BCC6736C3E3B
:103AD000A38830BEA43B95BC7BD258BE465A9B3DC2
:103AE000D205AF3D393A21BEB82DD13C543C883C7B
:103AF000E3DD43BDE6D21CBE8469A23B3EEF1ABEA5
:103B0000A61D783D285D1D3E9DCEEDBD1FCD603EBE
:103B10002B1B0FBD9CD9B2BD322738BDDCAC05BE16
:103B200022F552BE4D66953C4AF8523D3B84153E07
:103B300043C0FC3C92A6243D9734DDBD3D4814BDF6
:103B40005CDB32BE5C18293EF374A8BEF1D4F73AB0
:103B5000C1C05CBE10FC653E4844B93DC5773E3EE1
:103B60006AEE19BE2A0D3F3E19F5EFBD07C331BEFF
:103B7000D05F0A3C2E01E6BDA6CDB83C06B126BEFC
:103B80000146DF3D6CCCA63D53DC18BE963CF1BC33
:103B9000684A02BEFD553D3DD8DBFE3DDBC3353DE9
:103BA000928851BCFA59673D594DEF3B6FDBAC3DF4
:103BB000E77A9ABEAC3C323D58918DBD7613043EF7
:103BC000A513943CE97576BDA5DC06BEF2EE7F3DFB
:103BD000F6743CBDAE38C73DE8C4EABBD54C25BE43
:103BE000F5941CBCD4E47CBC313B6DBE6633A63D71
:103BF0007BB861BE0713D8BC192C97BE84E79ABE68
:103C0000DB67193ED6002D3E48BD6EBD749FDE3D7C
:103C1000D5A115BEAFE0F13DD34A013D3CD84CBE25
:103C2000A5223B3E603C043EE02CDF3DC262DB3D12
:103C30002FACDF3DCE8F033DE1609C3D67F89ABD20
:103C400032B0E3BDECD8C43DA89260BD2E7AA73B4C
:103C5000D557BABDBD30C83D5CD398BE486D9C3DBC
:103C60004F97BABDCD73C13DCA7BA9BD4BE98F3D0E
:103C700075170DBE98A74C3EB679E1BD6A1719BC01
:103C80005782993D5448613E97D518BDC6AA7A3EE1
:103C900092845ABE7E9194BAAFEFA73D6B3856BE60
:103CA00080A42F3E80C70D3E1634163E443F773D1C
:103CB0004585303E24E101BEC216E7BC14A181BE99
:103CC000D7E3E5BDC63F053E5AC524BD8AE446BEDE
:103CD0004538BE3D462E2ABE49E485BE4F4895BDB7
:103CE000F79B1B3E3D3DA73E7EDC8FBD46EA53BCA5
:103CF000C51B933D32111DBEE27A9B3CC0DE40BA2B
:103D0000FE93363E1E31A2BDAF9F81BE41C752BD5C
:103D1000979D533E8A0B053E1303293E925CC53D99
:103D20006EDAFB3CD9A1F9BDEC20C73B64E7F93D55
:103D3000572335BD59410ABCA71D0D3E82DE673EA3
:103D40008BD56B3EE02EFEBD56C7273E3AE260BEE5
:103D5000396971BD90E0343E6ABD713EA6566F3D33
:103D6000EDA2DEBD4E9BB53CD422483E54F77C3DCF
:103D7000840C063EAAA1723EDCC425BE6BE30D3D59
:103D80008123A63DD9916C3DDBD145BE2E322D3D20
:103D90001B0D54BE25EB82BD9F325C3D68BC0F3CC1
:103DA000522955BE448EA23D78E7283E53F4943EF6
:103DB000F4C4513ED70EB23DEE7025BD99A0D93C5A
:103DC000778737BCFE55D9BD4C2E863D757A4EBDE2
:103DD000147484BD21D396BC74DEF6BC660F63BE3A
:103DE0004C1150BE26F2B8BD8FDECC3C248487BD7A
:103DF0004879AD3DAC12873D7C9385BE485474BE76
:103E0000121021BE2404F73D334F1E3E0B93E9BD33
:103E100049DBCBBD0AFA973D0EA7153E7FEFCF3D9C
:103E20002A5A59BE558A75BD5796113E02F71D3E56
:103E3000D4BCC0BC84B39BBC0E9B77BDD2286ABDEA
:103E4000D60CABBE6F14D2BDE871A5BCBBB598BD96
:103E500074150B3ED2DC25BE47C8013EC7F7A5BD91
:103E6000CD718ABE4EADDF3D83F2AEBDCC5B5BBD96
:103E7000251F373E968F0A3E7A84F0BD5DF00D3DDA
:103E80004FE892BEBCD3C03DBBB1133E5F7301BDD2
:103E9000D330A93DBE104CBEA44284BCB29446BEF1
:103EA000F89788BD43B772BEEC71313E96745C3EA4
:103EB00054FE02BE5EE5DF3D6D6B033EA5A7EFBD80
:103EC000F91C85BEFA460A3EE41D263EF437733DD2
:103ED000F9D9BEBD6A8E59BEC92C623D9AB8B4BC30
:103EE000275511BEB52C9DBDFFA8D3BDA2DFB73BA2
:103EF000BB0DC8BD206CE6BC8AB39F3CA6E3EABDFF
:103F00001030BEBD863F14BE92DA8D3C66595B3ED2
:103F1000269F8A3EC257023E3E78F1BBE22D923D7B
:103F2000976D62BE639839BEEECE013DB797573E9E
:103F300043FDA93DE45A33BD78DB6A3D2BBB8FBE00
:103F40009DB59BBDD6D357BC4BBAA83D8271053EEB
:103F50006B356FBE73FE34BE189203BE6AF8263D01
:103F6000044CBCBD94987F3E706EBCBD442D423E57
:103F70009392E8BDDF4DE73D1822D0BD75568F3DC9
:103F80003CD4D9BDE0BE16BD31DD99BDE950E53D5B
:103F9000E67C753B7EE421BC066404BD48CD0C3D47
:103FA0004BA124BE3BAE453EE329C33CAB491FBEFB
:103FB000115741BE671EB53DABB51FBECDAB20BE90
:103FC000AD028BBD154D01BE87245F3DC0F01ABE0A
:103FD000D00F89BCAEDC2ABE829127BE6B78593DDA
:103FE000415F3C3EB321093E263CF73D12E8EE3DE1
:103FF000B60479BC69D0D5BDEECB2A3D24B2283EAB
:10400000409E52BE481C1B3EDEEA1E3E70E545BD8A
:104010006B4F61BE2BC4963D15FF5F3E3D8B483E06
:10402000D2DFC6BD7EAACD3D0C10F63D9485C13DC4
:1040300089FF98BE1AB1983E6E7899BD038F10BE65
:104040006C9D4A3E1DEC8CBD12A2763D20D47EBDF7
:1040500036308DBEFB73453E2917BF3C540D97BDCE
:10406000C05B5D3CEB3B233E3C45AF3B983F89BE8C
:1040700025E464BE0BAD2FBDAB48D0BD474BF7BDAB
:10408000571DEF3D07B196BDE8B1D5BC0A2D41BE25
:1040900006B0A8BB34F9B7BD0D1205BE4DACA4BD2A
:1040A000C10E883DB58498B815633C3E0191B03D82
:1040B000601FB8BB80ADFEBDDB8A1ABE88FE56BE4F
:1040C0002B8193BDBCCA243EE93D15BEAA2D66BC1A
:1040D000AD7ECCBD16211FBC2EA5463D3221863DAE
:1040E00074CB96BDB7C64FBE77F3A53A1965843E2B
:1040F000DE0CDF3DB867443E1A6895BD906AEDBCA2
:10410000A9FC193E32A9563ED85C60BEEA5F35BEB6
:1041100078DAF33DC138B5BD67D3BA3CF591173EA7
:104120005B7401BCBD70383DEBE459BEC91EC6BD11
:10413000A547283E1513D4BC529769BD8028113E6F
:104140000BB9D13D13D4B6BDA2F39EBD4450AEBC55
:1041500022341BBDCD93793E8BAE623EF37F683E29
:104160004B049E3D47AC7B3D227461BE6D83AC3DEC
:10417000C1D84B3D46B78B3E33FF563D779F23BD9D
:1041800029CCF33B256F4DBEF0C498BEE1AE763E20
:104190004D27ED3B8F70933AE4AB87BDDE3DBD3DCF
:1041A000561242BDF44D35BE8DCE19BE703015BECF
:1041B000EC7F063DD364403EEBF1E9BDBF8B01BC13
:1041C0006E8611BE66F446BEAACD80BE2C1184BD9B
:1041D0000586023DE3C0953EA9B5EA3DB08006BE26
:1041E000CC97883E697D52BE60530A3EA5858ABD44
:1041F00066A8013E0035B8BD7F365DBDF46E3CBD9E
:10420000674B04BE0FCD95BEA8F798BD4927573D13
:104210008613BBBD6213D5BCC355363D8DDFE7BDEC
:104220006A25C2BC9F5C823D6A8E613DFACE97BC16
:104230005872863D28D8B0BC33FABDBD1E525B3DD6
:104240008202D1BDF64188BEF416B83D9100A2BEEF
:104250009E5E693D636183BE5922CC3D9E222A3E0B
:10426000B676143EEF7A13BDCFBF533E72F6B4BD9F
:10427000C268A5BD216EFC3DD12CF7BDBF6D72BDDE
:104280001102A8BDB1797EBE59C024BD656762BE6A
:104290007D5D4DBD08C2B3BDEE4B6ABE1BD8C13BB0
:1042A0002ED8A03E6960C7BDA638A63D57F249BECC
:1042B000E897163E015A23BEAE41EF3DA0AA3A3E12
:1042C000C3707BBD878137BEFFBB0B3D7A30393E63
:1042D0002D16153EB9EC55BEBC6CC43C4A7E4ABD99
:1042E00037EC3C3EF2C35FBE03F1AB3D565E753E1C
:1042F000D89708BEA2821DBE5C0AA83B566D5FBD62
:10430000DC71043D1C2023BE6946AB3D9D16133E67
:10431000EECD1C3C3D1A573E1A5837BE2658003E7B
:10432000FBA743BC9A98EA3DAA5F403DD1F44F3EBB
:104330002D3CCCBDE290B93D7E4A03BEBBFAF2BA39
:10434000B6F72E3EA53EA03BD2DC213E0485413E81
:10435000AA6E29BD03A614BD838727BE2445703EDF
:1043600036C2C1BD9F1BC13BB6F7593EB73D7ABEB1
:10437000E7656D3E9078F3BD1813633B192C443C00
:10438000C8027DBD6A8995BD3355083E5C6FCD3D41
:10439000988AA4BD60E779BD52BAD33D18E6D3BD73
:1043A000D9B1683E669CE3BD0ADA723E887B08BEDE
:1043B000143D84BED06C34BE42C1323EE3E99B3D25
:1043C0004CA28EBE7BCE41BE2C6FA9BDDB08143E35
:1043D0006003733DA44D67BE82A4EC3DB66B023E04
:1043E00098A2DCBDA178E3BD0571663E372D753C12
:1043F0002754B8BD6D9888BDC8E4CB3C31DAD5BD33
:10440000E176103E8AA846BE228D743DF271D9BD78
:10441000D1108CBE6528683CBF16C93D482C16BC1F
:104420001357523E366F6FBD6B260D3D70650DBE46
:10443000DA2DC83DE2E50C3D91ED58BE8D5D3C3D69
:104440006F52FD3CFC8B2C3D90A9833D9A1239BEE6
:10445000CDDB00BD4217843E6E7910BEF700853C6F
:10446000507AB7BD2B3A653C077819BE0CC2D93DCE
:104470001D47DB3D678D393E53B61A3E55982E3E9B
:10448000BDA495BDEF301EBE8A722C3DAD046B3DC0
:10449000F61044BC222F873D0096C93D9416413E3C
:1044A000970E16BE6522DB3D0DF40D3E00033D3E2A
:1044B000DC75AE3DA595C83C2048253E20A0273D93
:1044C0004760F03D3F4ADCBC9E2A12BCD6B301BE19
:1044D00044E9193EC318F43D3E42513EE63F1DBD3E
:1044E0000A519CBD58A3EBBE582B2E3D0C83A83D12
:1044F0000574AB3DCCF723BEC03173BD45132C3DD5
:1045000077688DBE1DA425BEAAD90EBDED891B3EC0
:10451000B4F2FCBC1C6850BDEBA4D9BC55DD833D96
:10452000DC4798BEFD5542BE5EEB63BD83DB2B3E90
:104530003D9E2D3D63E10ABEB5AE3D3ED79BB9BD64
:10454000F86C89BE9268BEBE891ADB3D0FB3A73DE9
:10455000EB30543D6E56463D07C380BDF4C6253D45
:10456000A144593DE9C6FABD52A2843D243E31BB67
:104570008E06CE3D56D418BE70D06CBD455D643DF0
:10458000E21D683D4A7857BE8BEB043E7AAB923E03
:1045900049D5233E81DB70BD0DB35ABE079D163E43
:1045A000315A6DBEEE0E5C3D45F03E3DACBB863DE6
:1045B0008ACD553C82B21D3D37CB7A3D8A30923D43
:1045C00092A00EBECDEEE0BD50A5AE3D59CCDE3C76
:1045D000728A82BDEC0D763D79C2A9BDF52A90BEE6
:1045E00003D891BE495792BD7FB56C3E00928FBEF5
:1045F000377F05BE3131343EEB91A8BEC1E590BE98
:1046000095EA843D285BA53E63D55CBDC5E5943E37
:10461000DDCB98BD1870E73DC2CFE7BDDCE24CBEF4
:10462000184FCB3C7A43CB3EA02067BE163ED63D0A
:104630006808043E5573B83D148417BE96B4CE3D49
:104640007FB9673E6598B73EF408B63C3419BD3D66
:10465000148AE33DFFB713BD21CC8ABCF1A9A4BCE9
:1046600015FC19BECEE5BD3EF30A143EE5B6BEBC50
:104670001D29173CD5095ABEFEA41FBE56E51E3E95
:10468000021EB83D4E47183E3FCEBF3D8D9FF8BD40
:10469000AECA1ABE703B5DBB2539353CE199B83CCA
:1046A000B39F1DBD3B82F23DBC7B19BD4CC98ABC8A
:1046B00003E8413D62F0CBBDE9A7D83DC40F723D90
:1046C00031E7183E3BABC53E5ECE9D3CD46E36BE58
:1046D000867FB93D1566C93D349FEBBDECE92D3EA3
:1046E00009A234BDB0089C3E2FF9053EFB002BBD4E
:1046F000EC5EA4BD8CE72DBDBC25023E9038B83DD4
:1047000052E4993E3338723EAD458D3E42278E3D90
:104710008242AB3BED2FB23D92B2E33D77A306BEA2
:1047200029BD4F3E3756623D45D787BD3D3C523D82
:1047300058B139BE0265AE3DB21246BE0357F43DD4
:1047400080D247BDB503953EF7039E3D7FDDF6BDA4
:104750001401863CE97DC2BD3828FCBD0C08863DAD
:1047600050A6313E7858A43D33C73DBC89B4493E7C
:104770005473393DAFEDA03DB7602DBEAFC1A13D33
:10478000598C6B3D1D1DB03E279021BE68BC1EBDDF
:104790003778A73D443D92BD67E0063D788B2F3EBC
:1047A000EE3A7C3C4598B1BC065CE8BD2E66773E8F
:1047B00076659EBCF580ABBC17D6133EDD01B1BD5E
:1047C000389FE13CA29E713E489D87BE1D5FF63D2D
:1047D00079201FBE3241943D82B8263E27FE58BC48
:1047E000D22408BE6AFC713DE92649BE7A5F833D4A
:1047F00004760EBDBCBC32BEB52C2F3E15FA11BEE0
:104800009A296C3EEB21203E2EB89DBE9C4F893DDF
:104810000193AB3D80EC59BE0AC018BE9992CABD47
:104820001682613DD9BA573DC662C1BD182C3ABE49
:10483000885C8A3D3ABA44BE8675893CE083833DF4
:10484000BC56C3BE46FCD7BE794B5F3D6E0F7C3E67
:104850006F1370BD1FC814BEF3151BBE1D15803E1F
:10486000AB2A2DBEE5F0F5BEDAEAF83DC45CE3BD47
:10487000920400BE88711F3EBB830FBE956DED3D57
:10488000F795ADBE32A8D5BE1988B2BC27BF09BE08
:104890002EE376BD1A2A73BD8682413EB23BC63DE9
:1048A000FF55143DE74484BE87F48ABCCC73C03CFA
:1048B000F104143EC1DA8F3D43DD683C61A1A6BD21
:1048C000135AEABD519787BC22361C3CDB72103D5F
:1048D000AE94153E1C3AD8BD8E2597BDCA9A8ABBA8
:1048E0000A93093DCA2E22BDB38BD63D51BC51BDA2
:1048F000218E6C3E3A5033BE10A2423D6A7AA73DEB
:1049000039FC863DB1FC2E3CA61F093E4E15393CB4
:10491000C010103DE303213E697288BD4833103E4C
:104920008ED7B3BD8D77E8BC33BC9B3DEEBD6A3CF2
:104930001AA40D3E45D8CF3D825DCE3C128919BEEA
:10494000BF4CD03C2B2A34BE3E91853EC7A32D3DA3
:10495000146A56BE55CD25BC963ED83D8DA5343D36
:10496000F3E6973EF8BA873D1E64A0BE29FC9ABEC6
:104970001DEABFBDE75E483E42F393BA149C043E75
:104980003BB6003E5594A03E7EA274BE247683BD05
:10499000A4E9943B81C2B8BD9999B43D1B83F9BD8C
:1049A000A5757E3D94326B3E4BC08DBEA4BC92BDBE
:1049B000E31029BEBE4E83BC3709ECBD2E4E773DB9
:1049C000B85BA23D2659FC3D31DFE53C684561BD41
:1049D0005F11A73DFBB5C5BDAE702BBD0756633D4E
:1049E000C4CE8ABCFAE17BBCB94D68BEC941DABC11
:1049F000F0A3473C75751DBEE23B173E885D6F3DD9
:104A000059EECFBD1A8A7A3E26BF4EBD17D3813DDF
:104A1000018E38BE691C47BD4465C33DE4D0FCBD72
:104A200075E3C43D60F8743E63CDED3B5A72A43D1E
:104A300041A6F13D34454CBECF6CC73D324834BE33
:104A40004B4205BC82C0063C918050BDD31F8BBE3B
:104A5000B1F2B6BD334B363D56852DBE8F4CEB3D86
:104A6000EA6F0ABD94E3583E36FCF9BC08D05F3EBD
:104A7000C7DF9DBD45FC243E31A3F1BD54EA80BD96
:104A8000EBC6A53EF0BE963E606909BDD4D0543E4B
:104A9000F73F74BEF0CCFC3D78FB9FBD546F84BCE7
:104AA000AAA6353E9C9B9F3C2113E0BDCFA9533E57
:104AB0001CAC60BE498341BCAA470FBE097E803D45
:104AC000CB8FBD3D7820263BD4F7DCBD7CCD833E2B
:104AD000B61565BE335D4D3CB5E2E4BD76EFF5BD80
:104AE0009D09443E0BECE53D9129C73D80FB9FBCF1
:104AF000FE9037BEBF5EE73CABA3ADBC8C7C673E8F
:104B0000AF55B73C6575863D38FB0B3DFA5622BE66
:104B1000B2FF1D3EA10C11BC2ED5063EB9CEBC3D48
:104B20003E1E163E0E2D843B7C010D3EF9F2B63D35
:104B3000856B183E147AA6BDE905FF3D6A6CC8BDB9
:104B4000892E9D3EEF7D84BDFFACA3BDEF79D83C9F
:104B50004F0C463ECF8F313EE08F99BBC479DE3C8F
:104B600027EC533E5FF2213E8617F53D265DA7BD3B
:104B7000472BB9BD08C9823D1348B9BD303F903CB1
:104B80005FCF913DEC56B6BD2BF183BE862CC8BCE1
:104B9000C61754BE407871BE7BC88ABECDC6CDBD97
:104BA0006CE488BEE8CAB13D4700FBBCB5FA3F3EA5
:104BB000530D3DBE83117ABD61CC2BBDA912BBBD87
:104BC0008F5734BE7BC2CBBD9077A0BE4E602E3EC9
:104BD0002B743A3E071B1E3E9C9507BEADE99ABD5D
:104BE000A926253C2449C43A3F531BBEA134E9BD44
:104BF0006F9827BE180D473E186FB5BDA330F3BDA3
:104C000073226BBE9D9885BBFE812CBE3825FEBBF2
:104C1000C5FBF3BD802E243E651E28BE974F1CBDEC
:104C2000A531053E598BAD3A8E14CB3CB830DABB7A
:104C30008EE6333C7B1DEEBD8CCAFF3DD4622C3E1C
:104C4000CA77853D1F240C3E4882053E6392E43DB1
:104C50006ED7463E915726BC2B85093EE37F8DB922
:104C600067C191BD5AF9873EE7C7233ED9EC933D12
:104C700023CE38BEF5AB66BEC30732BE223B45BE6F
:104C8000E066E73D9F476B3E20A5503E0DE11A3C94
:104C9000835093BDABEF0F3CA5B32BBE3AA4033EAC
:104CA00010C2073E2B73153EF1110C3EA9BCD33C3C
:104CB0003955573D889C9CBD85128EBD00CF57BE8F
:104CC00045349C3E4AE00A3EC2B34ABE734A2E3C7B
:104CD00043D6E23D9568543D41A774BE529EEDBD5A
:104CE0004F7D393EDA0C363E01FA083EB063453D51
:104CF000767644BCEEC021BE9AD71CBEFAC655BE1D
:104D000020F1623EE1BD083EC3D228BE9612173D97
:104D100054E82D3E9E101CBE525147BEC8806DBE49
:104D20003AAEFF3DE9F2413EDC41FABDF08D5F3D18
:104D3000FEA3FBBDDB8D5CBECA6350BE5441DD3DAE
:104D4000BB97063D004F933E77D956BB41C82EBD59
:104D500085FEBE3DF66A613C6F880EBEEB93A03DBA
:104D60000E3AAEBDC83F913EF3283E3E6029033D5A
:104D7000B23C133DEB67903DB19D223ECC54283EA2
:104D8000B4F4663D4AF0CF3E1AF9CF3D96980FBE77
:104D90009C08E93DAE0284BD07E83EBE1AD085BC42
:104DA00079AB69BE90E79D3E58EC293ED328D0BC34
:104DB00032A512BCF996993D7E84723E90D7443E4E
:104DC0007D8BD5BDE2D4F73E63DE83BD1DC8B9BC83
:104DD0001FEEA13E3D252C3EAA41943D5A93BEBAFA
:104DE000012F913E272E4BBEB51720BE436D453E89
:104DF0003D87473E8C3B4B3EF1C9BBBCB4268BBDC7
:104E00000B6A0D3CBB26CFBD1A4E1E3E557D07BE1C
:104E1000EE023DBE37FEAEBDBE5B873D4A378A3EE1
:104E200056002ABE50648EBC105F66BD4ECD0BBED0
:104E300094EF5B3E6588033D11DA54BD2B8D783EBF
:104E40005F68B8BD701FF03D87A73CBE9F9853BEFA
:104E5000B899C93B58E0843ED33C4B3D0F87113E87
:104E60004BBB61BE1BD220BE4903E0BD42F1BD3D3C
:104E7000ED246BBD404E1F3E7EDE09BE3428A93DA9
:104E8000FE30053B3AA98B3DE150E93CE5316ABD76
:104E90002524E53C704F943E08E017BC87382ABDB6
:104EA000E723A2BB3E7145BE6726393E5B4B27BE5A
:104EB0006521BFBDCE802D3EA819F1BD05074BBDB4
:104EC0005C16E9BCDEFA31BE0C406E3DD2AEB33D9D
:104ED00035A0243EAD1A383E322935BD234676BC76
:104EE000E0A3A3BD7A2E56BEA818553DFACBA5BEA9
:104EF0005F98FBBC041F28BD9187943D88112E3E0E
:104F0000467B033E33170B3DCB88A4BE73D312BD43
:104F10004D92133E090221BEB9EEF7BB2A52383E2C
:104F20008B04D2BDF26901BE4BF92DBDE0D367BE43
:104F300043E05C3D1581E9BC2C0BCE3D1354DFBD35
:104F40007D85BD3DD3480ABE807A973D08B0ABBD94
:104F5000983F94BED2372B3EEB53D1BD959C623C1B
:104F60006C7A9EBCEB20303D509291BE7B52F2BDDC
:104F7000359496BDD10194BD6F69E6BDC0B3B73D10
:104F800045C2343C318127BEB40607BE28D50D3E4C
:104F900060D51DBEFF566B3DF417383EF410023E3F
:104FA00000A120BEEC7D963DD0BB343CEC1E8F3D75
:104FB000523BB1BE825CC13CD4B7C13DF8D539BECD
:104FC00093F8B9BD3186B93D41DEE13D8D85DABC4E
:104FD00078CCA0BE00AC0ABE80BC5CBEBFA9993D27
:104FE0003C65F4BD971ACB3DB2FB1B3E942544B9FA
:104FF0005E7D993C7B9822BEF915003E99F33CBE3C
:105000001D9CE7BB336017BEEDFB0A3EC52BB1BC50
:10501000D04A6ABDC1E9AFBD5F78BBBD78D810BECC
:105020008D11923D418678BE939B86BE2C7832BD11
:10503000C3D2583D0208C93C64AA243EC8ED8C3D49
:1050400009C9DABD7C611FBDA1CC9FBDDFE1703D08
:1050500019DCEE3DE7B561BE944BE1BC3E29693EEB
:10506000FF46E2BD83F512BE4D450FBD3697063EA5
:10507000E5BC543D432636BE7AC28C3DB1979F3D78
:105080008DC71EBED66DB23D3C8E963D39AB0FBE70
:105090008905E2BD2AE3323C58790BBCDAD94FBD11
:1050A00056F0173E661145BE62D87FBDB6B194BCBE
:1050B0009B3AB5BDDD1ACC3DFBAEC1BDDDD4263E6D
:1050C000A8444B3E804720BD0E641BBEA47C163E08
:1050D0001B7DE23B977686BC7DAB04BE58BB12BEFF
:1050E000AD25733C2BBE46BDDF94593E586B13BEB5
:1050F00079AA52BED1B540BE625E583D831A39BD11
:1051000083FE613EF1A302BE3A54AB3DA8AA4EBD58
:1051100018ADD5BEE535FBBD41FA093D9F5D5F3E4B
:10512000494D7F3D9529BE3C331F2F3E1A8C983D3B
:10513000080F1CBE9299383E2D5DEA3D5C0AF93B92
:105140004884903D91FEC63D90A062BEFF476BBC77
:10515000746983BD6C4722BEC7C1E4BD075B6E3D69
:10516000D9ABB33D7BDBF53C99B659BE1FEBED3DAA
:105170005A60A0BD654EE73D97158A3DC0BE033E0F
:10518000DA62CB3C6732DFBD5D3623BEF6EF183DF9
:10519000CCB7073E3BF2BA3D96E7B6BD049218BEC7
:1051A000E716593D1DE4873D687EA7BD42A50CBEAC
:1051B0009C77333EEAF86BBD1CF6D8BD09D7E63DB7
:1051C000B9E748BCB6C5D1BD8B66143E6154793C85
:1051D000C1E2F03C75010A3EA651713E0E1E663DCD
:1051E00034A4153C0AE829BEFEEF8FBD9A509FBB40
:1051F0008C18AE3D97B6BB3D8700F13D396415BDB7
:10520000F70D9D3DD8B369BEFA23EF3D39DE42BEAE
:10521000E28EAFBD6FADA43DBE0F1CBE00C65FBC2D
:105220002F71C83DEB89B1BD1456433E46BD6CBEDF
:1052300063463BBE92223EBD513E66BE4BCD0CBC8A
:1052400094026B3CECFA3DBDB4F39C3E645D87BEBA
:1052500008108BBE5FB3993DD97898BD24BC7D3CC6
:1052600004F85FBE0CAF86BEFB58B3BD1A1F423EAA
:10527000A443DBBDF70D9F3D399AA63D3E260FBEE8
:105280004D82D7BD68F37DBEBB99A5BC8DF286BCAF
:105290008BF3223EBAE76D3D29C77DBE7E0F493DA7
:1052A00071087B3DB761783DDF4B51BEAAAAA4BD12
:1052B0008CA9FFBD6F4D1EBEDD5A43BE3A4FF33D74
:1052C00083DA5F3EF95DA8BD3B5A2ABED17885BD21
:1052D000D63AA3BD30DB4DBDB5C1A4BDA2E625BE07
:1052E0006FFF2EBD0DD983BEA04C803D2DB7CE3DA6
:1052F0002868013E468C363E786C06BE58DA283E59
:105300001A0A9C3E2EEB16BEE2AFA83D8A9CC0BD99
:1053100075EF003D9959F13CA22722BD3E96FABD9A
:10532000507DEC3BF17061BE7146B23CBED3273E6E
:10533000C92E4D3E91B9C73C54C4A13C8035913E25
:105340003318373C44DB5FBE92768DBD584521BE95
:105350007814AABD0087FA3D39A13F3E1D1A593E77
:105360003525A73CF9AE22BD86FBA5BD3C8ABABC5B
:1053700075B06E3E11429F3D8286B3BC5A4B293DAB
:105380008E0033BE7E77233EDE645E3E096C0DBE2A
:105390001C767FBD3A341E3BCFF30F3E3C2B093EBB
:1053A0008FB733BC88C9773E770EBA3D10A900BECF
:1053B00064D48DBDF0D377BD63335A3E41D2873D6F
:1053C0009EFDC4BD558B23BCE484443DB5631ABD2A
:1053D0006699B43D8BBEA0BD9834B0BDB2F708BE8F
:1053E00062FFE13DB180A53E0BCA203D28C01DBE35
:1053F000BD5260BEC95106BEF12C533E3A0D37BEB8
:1054000036ACC33DAD97943E62CC3BBEE0D8DD3DAB
:105410002230C93D94244E3B5D4911BE47F658BE2B
:1054200013CA653D147C6F3E4AE252BCB2077D3E12
:105430003D62FA3D31AF8B3D3B534B3E2DF0BBBD42
:10544000AEF6F33D86227C3E4E54A8BDDBA76FBC72
:10545000106F83BEE14EE73CABDFF13CCBF0263D65
:1054600000BD09BEFC8172BDAE9A5A3D4B72133E1F
:10547000D4C6153E672DD3BC807629BD61A5ECBD91
:105480001ED0A0BE18EAA93D55A740BE39C8323E7D
:10549000281427BDA48A853B5DF52E3E57B67C3D7A
:1054A00052A64E3EC9A9C5BD95B5933C4ED4BEBCCF
:1054B0002EEC82BE324D8D3E412D90BDF54E023E0A
:1054C0006DD1953DB42A69BE46D9A5BB3A38763D23
:1054D00064DC85BD029B5E3DAB56683E96EC7D3C30
:1054E0006C3280BD053A05BDE94E2D3DB875E63DEF
:1054F000EAEB03BD5448663EA3771CBD9C7925BEEC
:105500001F1EE73D3B54D7BDAA5E3C3E047413BE4C
:105510007AC4B3BD637BE83C3C09B93D2F3516BE68
:10552000D720843C583FE6BDD4ADFE3CA0BFF3BBC2
:1055300019F1143E581834BE8BB80D3EABAD01BE08
:10554000DA11B33D2945F8BCAE05F3BDFA820A3D38
:10555000F256A73D4EF47DBE6A8BCFBD425A4F3DF9
:10556000EDC788BD60F3AB3D7121DC3D5CDADC3D0D
:105570001CBE71BEEC3223BEC6D80ABD0F652D3EDF
:105580005CD1073D16F33FBEEF36133EA106FABDD0
:1055900091C963BE66B5C7BD421D01BEC7E69DBDCC
:1055A00059D6163E58882C3C0D4E6EBEA13C923DFD
:1055B000A0A4A7BC23D884BD3B953CBE1F11323E9E
:1055C000986EA53DB522553CC3A157BEFACFB73D55
:1055D0009197243E9BE8A2BDEAA450BDB318DE3DDE
:1055E00064BE28BE48F8473ABB6E29BE58CE60BE9E
:1055F0004B2986BD5B561FBE4938533EFF5567BDDC
:10560000B55998BE7F8104BD8866D1BD6DBE36BEDA
:105610009C8EBDBD8114AFBDA4A3203EC62441BE57
:105620008751DFBA37A4B13DB771583EB499CB3D2D
:105630009D9B14BEAAC4443EC9791B3E5C2BB8BDD9
:10564000ED8282BD35D782BD50224D3EF982E03DCC
:105650002D78B83D1392DA3D79AAA4BD2F9401BEEE
:10566000128990BEAB942B3E769A3E3EDA1ADCBD90
:1056700022ABD9BD02F4253DDDF4D13CF286163EC5
:105680001B1F5FBE3202C7BDC369293DEBD5063E75
:105690001E0D6F3BE5E13F3E19073FBC6D8F1DBE00
:1056A000E1289ABE429B62BD8C36083DAEC78DBDD7
:1056B0007FA7FF3DD8C08E3CD4EF70BE5C6CE8BCC9
:1056C00060FB68BE7035723E1987423E95F0ACBEF5
:1056D00073D65EBE408CD63D553296BD6325F03DF7
:1056E00023376ABEB3EA5ABD3E30B13DB28A06BE28
:1056F000FA614F3C99FE82BE72BCE5BD4B4B6ABE5F
:105700004012B0BE14EDA6BE89C2423E961FACBD8B
:1057100038290DBE9CA80D3CA996993C05310EBDBB
:1057200017222EBE178F18BE760072BDA6123F3EFE
:1057300021A10C3E24CAF5BB533F023E35DECFBD4E
:105740002B758ABE710A9DBDC28F263D0FBE01BE5C
:1057500099EF813D303AB1BC323E87BEB7A81D3DBE
:10576000BBB3A33D6FA11EBC4A5B52BE7EB6813D5A
:10577000EB00FF3DD02FAABDDF317D3D222D373D0F
:1057800045D160BE8C61BE3D47E808BDDEF1D7BDA6
:10579000B1AB3F3DC46B8DBD7F0261BD94DCF3BDF9
:1057A000C58D8BBE9E377CBE2501913DBAC1A23D01
:1057B000D91508BE379547BEF024313E64E9383A22
:1057C000ABA5863C0BF020BCA418433E01928E3E54
:1057D00023ABFC3DECD36F3EAE3B383EF0250C3E98
:1057E000C5338CBD291C4EBEACB9883C370959BEA7
:1057F000D34E5ABE165122BE1E42223EFA42813D6F
:105800009D3A8A3E2414803E88A770BD91B9163E09
:105810000ECF8BBDCB61A33D9CBE19BEE377C1BD4E
:105820003FBD773E41E6243D1C582F3D76C00B3DE1
:10583000E860813C46D0D93DE20183BC20AD1ABE70
:10584000199B25BD5486993EE2780CBED6EADDBD93
:10585000D6587BBB3341BEBD61355A3BB49B5FBE5E
:105860002673283DF8EF723EB7D05FBC259B88BDFC
:10587000E9EA86BD24C9053E152F523E505507BDA5
:1058800040CD6E3EB3C84A3EC476F9BD6264033E65
:105890006121143E3DE28D3B2AE711BE5CDE9EBDD8
:1058A0004056FC3DABA10E3E389A4DBE5466163EA6
:1058B000FADE04BECB1F08BDBCF7913CD76A693E37
:1058C000760A6F3EC552CC3D995F55BE8727F1BC25
:1058D000889B853D1FB401BE614CA1BC48FF183EAA
:1058E000CD7F473ED0C47C3E13CEB4BC921691BE51
:1058F000AE75F7BD4F841E3EE51135BE2B76F53DE6
:10590000B4CA803EFCB8533E51AB4B3E4582013E8B
:10591000A4CBEC3DB52F4CBE860C78BE240414BE3F
:10592000A1DA39BEFF0FB7BD0E93CB3D588A9A3C22
:105930008B3CFD3C3D0EF3BDE04E193E8C965B3D2D
:1059400049EF2ABED28D84BE7DFE083E7095473D4C
:105950009A7D813E6071DE3D502565BE0B6B1D3E1C
:10596000292B29BE777A04BEF48A803E0FA7AC3B70
:105970006453323E0CAF133E8B9398BD1DB44C3C28
:1059800021D101BEB44E5BBE9035DE3DA9C3B2BD90
:10599000A436B33DB294FA3CBE4F153EDE353BBE55
:1059A00017FF653D151772BEA2C18E3E261D17BD9D
:1059B000A22098BE769E59BEDE61E03DEC8535BEE4
:1059C000ADDB18BE122D0DBEE3EFA8BCD2110EBE8A
:1059D0000793A93CF61718BC4DE1E93DB04FD13D06
:1059E0001EA30BBEE41263BE403B8B3EAFAC9EBE1B
:1059F000F79F9FBDEAC4AE3C2218573D20B019BDA9
:105A0000D665E23DFA15173E7C37AE3DC080423E7A
:105A100064C2023E8757203E3FFDBEBD5CA9533D98
:105A2000D72B04BE30BC163E0A8384BD6BC3C4BDF5
:105A300058CFF03D9B0621BCFA8412BE078C0D3E68
:105A40004B86E83E9A75CE3D2FB8BBBE29FADCBC2A
:105A5000735088BE237000BEFA44C63D1DC4593E33
:105A60004413C1BC833B70BDAF2BADBE65298BBB5E
:105A70006F19FEBD80BBBCBCA42860BD8856F9BDB3
:105A800028A3933EB5F4D53D10590ABE808CFDBDC8
:105A900016C6A93DEBD3323E0CF05F3E2832223DC4
:105AA000017B013ECB84F63BDDCEEDBD54F1243EBF
:105AB00011197FBE86A6013D9165843DA885F63DFE
:105AC000B87537BC89EA703CDBD1D0BC1456CDBD6B
:105AD000FB49103E4EBBDCBD016D1EBE7C40343E1A
:105AE000AF7CD8BC7C1A943DF61419BE21C8003D89
:105AF000B7BB393D6C1A503E46D8A5BDA3FEF13D5B
:105B000061C7053EF1CC7E3E955A2E3DCAD89F3DD9
:105B1000022095BD8222B63C0AAC013DD101A9BC50
:105B2000964239BE40F06E3ED4FAA4BD6FACFB3D48
:105B300073A444BED5B2BCBD3E65FCBC08B32ABE4E
:105B40000AA9293EF9D6C03D8C64EFBD870FC33C3E
:105B500084D017BE81B5133EE84936BD59C13B3EDE
:105B6000CEAB47BD9894B13BCEA4293E108B05BE69
:105B7000788D57BE6A93853E68D2A53D197D8DBD4F
:105B8000BCA9023EC6731F3E72EC543D20560C3D2C
:105B9000A019FC3D8D40203E6ECAC2BC7643DC3C61
:105BA000A2745FBD72030A3E3CC2BCBD7CE40F3EE2
:105BB0002C0011BEF1452D3EC70A173D669653BE17
:105BC0003D7925BE466FEFBCAC94ED3D1A19AF3D53
:105BD0009A69943D32FD3A3EE3B0303E597911BEA8
:105BE000A93E9ABDDB73B7BC4783133D2FB105BDFA
:105BF000D2B4C3BC5D9F323EFBCD1C3DE016C13D1F
:105C00002D8F4BBDDC371FBD9DE79BBDF4D571BE0D
:105C100049762DBE502BEEBD233BB23DBC80DABC95
:105C20003AEA28BEC9BCA4BD09D506BEFBA912BE6E
:105C3000D95B203D4D3E2B3D62C0D4BCF01E4F3D94
:105C40006D882BBEAA7C463E87C627BDAE51CDBD12
:105C5000E45EE8BD1AA863BDD297053E6318D9BCBF
:105C6000301836BE1F361A3E167395BEF0E5813EDB
:105C7000440E86BD8E3228BEA4F5E7BB3868ADBDA4
:105C80006F4029BE74FF95BDF72CFFBD80A5893DEF
:105C90001FCF2FBECE3BA43CEA8694BD9E2A463E33
:105CA0004B35A4BE9F01103EF53C493CCFBF00BE22
:105CB00083EBCD3D6D26B23D26E0EF3D038C85BDE7
:105CC0007CE53DBDA9291CBE59E7A0BD744F23BE8C
:105CD0005037443E8026B73D302D06BEBED0CC3D69
:105CE000E047273C734432BDD8C97F3DB888DC3DCE
:105CF0005E98673EB0A62CBE2D0F6BBE120646BE48
:105D000036CD2DBED1FB093E31F93ABEEFD3CEBD23
:105D1000EC3162BE22D422BED496BB3C586C123EFB
:105D2000254C75BE97FE3339917525BDE823213E7C
:105D30002D3E653E1B3B15BC8CB3543D762004BE06
:105D400055A336BDC11E1C3E6EEB0F3DEA1524BEA9
:105D5000701B02BC5BC44DBD732781BE145506BDCC
:105D600029C201BE24FC373DB1E7DCBDEDB5793D6C
:105D70006FC55F3E3B45973DF10502BE507A40BD81
:105D8000159E2C3C79F2863EF95981BE8287963E5B
:105D900029C02CBE0BE953BD55BB933CBCDB47BCB3
:105DA0000B29C63D2E95543D398C683E74BD003E8E
:105DB000F6FC8FBDEA98D4BD0FAC06BE8EDD853DE6
:105DC00038CFC53DA8D9753E98E1EA3D6296D13DF0
:105DD0006F5D5FBD167A98BDE681333E5A7FD43D34
:105DE000C4CF23BD74EE7A3E9F4EFA3D218D29BC6F
:105DF00040E86C3D19F4DA3BB622423DDED243BEA8
:105E000003528EBE173A42BD6CEE10BE171DD83D30
:105E100089C8D53D1BABADBD22352ABE303C1DBE69
:105E2000FD5437BE5616EEBD477112BE9FA0653EAB
:105E3000B13C0ABEBF2908BE0270193E7CBC11BE2F
:105E40001D8832BE7FF04F3E316B023E5635783DA5
:105E50008A3522BEE8A06DBE21A5933C9B20A23DC1
:105E60000393D5BDC264BCBDA58BCDBD87D4ECBDAD
:105E70007068A1BD3D9D0FBE33F43D3E44BC3EBDA8
:105E800024790DBEE488383EED8136BD057A9F3C0D
:105E9000341B893EB030DE3DB1493D3EB3BA873E4A
:105EA000C1C707BEA182263EAAE221BD99042CBD2E
:105EB000502397BDBAF8363E4C9E37BE9F16E53B41
:105EC000F8E8EB3E985A463E74AEBEBEAD7F46BE85
:105ED000CBF6913E6FAC36BEA22088BC506ADC3D4A
:105EE0008B3EEE3DE5B2423E021449BE6E4643BDD6
:105EF000A131D43D24BF013E2188F83D8685513E25
:105F00000A2C7FBDB01CD73B9F52AABD1B627E3DB1
:105F10008F9B97BDF25C4CBE72B0D9BCEBE2C9BDA1
:105F20001B41483D79D36A3C82AFC03CE265573D96
:105F3000CA61EBBD6181DABDAC14B03D51092ABE26
:105F400043C3603DE3B00C3EA258BE3D2EB1E73DD9
:105F5000820631BDB008153E84C92BBEDEF52EBECB
:105F600025741E3E3EAED63D564693BD743E903DD2
:105F700018CC7CBD9A2DD9BD638F3ABE6581E83DB2
:105F800038F33D3EDF059ABDF1A291BB9110903DE3
:105F9000E6B698BD673D043EE022003D5FB0F33DAC
:105FA000ED3FAABD3BFD4C3E091A4E3D18D00ABE3E
:105FB0002D11ACBE472C40BEEFB420BD479753BD5A
:105FC00036EC9B3E6356EABC1FF2163E86967FBDBA
:105FD00088CD453D3AD1ED3DE8D73CBDE4C47ABB20
:105FE0004FDDED3C6BEDE3BE452A053EB59EEF3D32
:105FF000113E8D3DE026073B7B40A3BDF4F3D23D2F
:10600000028B29BE0A78E5BE050FB63DF683DDBAE0
:10601000B9A1D53C6FD754BE097D143C0ECE06BE47
:1060200050F6573E504A4EBE4F410E3B2701593D58
:10603000DF46BF3CBE96993D4F9E3ABE075E453D4A
:106040001FB039BE53756DBEEE07193D23C83B3EE8
:106050009FA93D3E5933BF3D676E29BED87BF13BBA
:1060600086B294BD9406B1BE1A10673E2479F13D04
:106070009CDFF83DC0F8523E09E4C13C1348B6BB72
:106080009D34A5BD2231D5BD07DB893EAC8A0F3ECC
:10609000569E133D1F0800BEEF61CF3D9A16343E59
:1060A000F4844A3EE7FEA6BEF5929E3D4DD8C83D1B
:1060B000B65500BE31A2053E608CC7BD2E32243ECF
:1060C0001318273D6CD658BE8D631E3EF92A0EBEAE
:1060D000E779A63D7046ED3D798E89BE24135DBEFD
:1060E0005C3757BD8AF82DBE0DAA1C3CA35872BE62
:1060F000DAFF1A3E6B06ECBD811723BE515983BEF1
:10610000A813283ECE767C3E64B2A73DEA6E613E7F
:1061100057E93EBD1321F8BCCF37773D7ED8B4BBDD
:106120002B2D5A3EF9AA8B3E5EBA78BDC1E8E83DF8
:10613000D238AB3C5B549EBCAD7457BDD739273EBB
:1061400018BF3D3E2E1F0C3EB7AD303E9D216E3E2A
:10615000306F103ECA0A1E3B332270BC3D5D2B3EA1
:10616000AE1C3DBEC63AA23E67FD9B3D4A38D23DBD
:10617000DF3ECA3DCB8D383D9FB2E8BC926CE53C1A
:10618000D74A6EBDC615903E92152A3E684A1F3EFC
:106190001A65BFBCDCDC313C6F63483C0AEFB13DA3
:1061A00006CD5CBEFC30D23C77822F3E8B2AF8BDF8
:1061B000DAD436BE564D0F3E4A5A3F3CC12B3FBD46
:1061C0007D8F89BE9C244E3C5AF7BEBD45B6A2BD0C
:1061D00077C844BD0A5CD83D17E10C3E92ACFC3C4C
:1061E000202E853CD32D373DE27EBEBB1947073EAE
:1061F00071381DBE5007073C8373A33D812D253D9B
:106200008154CD3CF0E1493E3CD2853E63FE9EBECA
:1062100073CEE7BD91A4583EAD604F3D96A93B3E7D
:10622000A53A4EBEBC1AB73C1F2924BD9A9BA7BDF8
:10623000CCE1C93D8F3F4A3E2A9ECA3D373350BD0F
:10624000C8FC01BE7C39693DB97C633D72EDADBCD3
:10625000D34D61BE188509BDAB1AFB3D2836783E8B
:1062600030440EBE5B2E883D968A0ABE66162A3DD5
:106270008EB510BEC42E87BDD499B1BDCB8CE3BD05
:106280006504133E5DA89A3E3AE85EBE99518E3C85
:1062900080B612BE800A0DBD4EB5313D43796D3ECC
:1062A000294C4B3B5CAE0E3EE1361C3CE971443D53
:1062B0003A28973CB58C6F3E5659833EF0EA2EBD86
:1062C0004092FF3C7966C73D2DBC8EBE88754EBEA0
:1062D000C4DF963D0902DE3D850FFFBDA70A0CBE57
:1062E00040C0823C981B0E3DB538EDBD262F0ABE3E
:1062F000039852BE364FADBD42C4083D5DFC28BD7B
:106300007C2B25BDE549C5BD937E733CB518473E42
:106310005C7530BE75BC4EBDC8D340BC951A483EB6
:106320004371DEBD79FA52BD729AAEBE34703B3E07
:10633000070A0C3D4C490FBE685712BE795D773E87
:1063400063F754BCB165B63C87A8DABD016CD53D96
:10635000D0233DBEB37B043E784412BEDCCDEABD03
:1063600077F4E33DD323E8BD4EC2223E5B3557BDF3
:106370002E71A73D2887FBBD4657853C7C2FDCBD91
:106380008E2DB73D185E343CF5881D3DCBB0CCBD9D
:106390007D4EB4BD70E84C3E36C79DBEF1E77BBD77
:1063A00018BD6E3ED59767BE92D6123E6AD70CBC1A
:1063B000DD3228BE64FF783CB5B2D2BDF269D4BDEF
:1063C000880F31BE4536183BFF75123EA74C0FBEF5
:1063D000544A893DD85997BDE1E2A0BED1229BBE67
:1063E000AF5ED1BD386832BD806677BEE759073EE3
:1063F0003894CBBD4A8188BCB4CC8D3C28D80EBE25
:106400001769383EB17CECBDCCF93A3CF6EA3DBEAA
:10641000A19713BEB42A473E6A4C17BCE5E6F8BD07
:10642000208F8E3D314325BE1644FF3D0E86D93C5C
:10643000EEECB33C3E48393EF99048BE5AD68EBE8B
:10644000EC8D89BEF680043E66470FBE3251263D74
:106450009E87FFFF0400000008000000FFFFFFFF11
:1064600048000000B287FFFF040000004000000069
:106470006B991FBE59B122BEFCBC66BD224B4ABE01
:10648000523C21BE80C53DBD2F0F4BBE246E32BE97
:1064900029F246BEA0211FBEE7A9A9BED39DDCBD3F
:1064A000BE528CBD91C75EBEF33DC4BD26AB99BD47
:1064B000FE87FFFF04000000400000005A8E23BE4C
:1064C000A93A55BEA7AC42BE30FE40BE5826D3BD49
:1064D00091BE39BE40E672BD0C5763BEAF100CBE14
:1064E000EBCA54BDA493BDBD94CD46BD43D8ECBD0D
:1064F00071B719BE053220BE193439BE4A88FFFF74
:106500000400000040000000AC825A3E3FC178BD4C
:1065100048D3AC3E8F33E43EC332BB3EDE2FB63EA3
:106520007268CE3ED0658D3D6745123FB2EF2A3F7F
:10653000611D4E3FB3999F3E52BE0F3F08E0B93EEA
:1065400073940C3F4BB0143F9688FFFF040000008B
:1065500020000000670EFE3F6E6FD1BEF02AC6BE5F
:106560005FE091BF1B66723EE037E1BF61E4373FF9
:10657000E3B7853EC288FFFF04000000080000006A
:10658000B6DC5D3E80B5063FD688FFFF0400000004
:1065900080000000FF4659BD661A243D6CFACFBD4D
:1065A000EDD1A83DEF8F993DCBE286BD4DE892BD80
:1065B0004663F93CAB68B1BD67C7393D5E8A09BE29
:1065C0001B85C93D8FC7C43D6CF8BEBDEE5506BEE8
:1065D0006CB4373D61D7643DEA55B4BD8AFB063ED5
:1065E00022DA3ABE52B522BE007A963D50F5943D6D
:1065F000FF6FC0BD1E6F513DCE2687BDBD89CD3D0D
:10660000B534FCBD8B15CFBD849C793D0AE3893D33
:10661000E21988BD6289FFFF04000000100000003D
:106620005C49813FFC97963F24D1BB3F563DA43F38
:106630007E89FFFF04000000000200001719853E5C
:10664000E8FB47BCC10F263DE47D04BE3FDFC9BC6B
:106650002C5ACF3DBF34A63C18945FBEA671533E62
:106660000B623FBED6ED6FBEC440A2BA8426E83DA1
:10667000D611BB3E2F4FAF3D8D4D003EEB3687BD53
:10668000B0932DBDF1A475BEF883083EB5753C3EB0
:106690009A5BCFBD77CEC13D36B2583E48121CBD85
:1066A000A6C25E3DF7ACD63D68B82ABE290635BE07
:1066B000B9C9AE3BDA0D99BCBC134FBE2FC8773CAD
:1066C000758E01BF81CAA43D23BE73BD408661BDE6
:1066D0003BF39D3DD7FEB9BDB41AD3BD74C4813D13
:1066E0000CBF95BDC256D4BD46E8CB3C70F1AD3D64
:1066F000664CE63C2CC1F23C624BB13D2595C83A54
:1067000073B20FBDE16EACBD1C97F23CEC01743D61
:106710003EE34FBD34D9BB3D926D843B63E5A2BDE2
:10672000CB135F3DBA0DA23D58CD55BDB681A5BD79
:10673000F03799BC7D7B3DBD0CD084BD5BC6DABC17
:10674000B041763ECEE0A4BD14E2123DA6BEAF3D00
:106750002DEA5ABDAA8BE7BC1D8747BC5D9A22BDB6
:10676000ABF4D83D4F46043D39C18EBD69EF9EBDA7
:1067700026098DBD9619E1BD2A539FBDB8EB233E76
:106780003F75E7BD18995D3D3C693ABDD59FACBDED
:10679000D1B7923DF1E172BCA176143D648FFE3D0C
:1067A00026F178BD6EBE01BED75A1B3E939F113EA7
:1067B0004B60743E52FFA13DA64A913D04EC0C3E55
:1067C0002B05E5BD5900BC3D45000BBE621BD0BC8E
:1067D000E9FF0F3DC77EE0BD29D40B3CCD7DF53DE3
:1067E0009A0209BEBF3E7DBD172E8D3D0EAC8C3D7D
:1067F0003A794A3DA7D9B13DB705253E996839BEDA
:106800005B4A7A3E789A94BC6DB3973EF941CC3D91
:10681000223D28BD2241323E21C2523EBA81E0BD16
:10682000B2FA323E42042D3EFF98153DC07DEB3A50
:106830008762B0BD35FCB4BD63335EBD8A8BFFFF9C
:106840000400000020000000BF62D3BF340CD53F1D
:1068500000BAD83EFC65BA3FB98AFC3F9D03DBBF56
:106860001EC4E1BE95EAEF3DB68BFFFF04000000B9
:1068700000080000304A81BCCDE82DBEFDDDEABD38
:106880007C4F16BD77A3EEBC34ED903DF420323C36
:10689000F15BFA3DCC19403EE6B06EBDDA2B683DA7
:1068A0009C8788BD5072653D76B3063ED69F763D87
:1068B00025ED153EBD0594BD6C922ABD1AF0D4BCE1
:1068C000E3F6EEBD5A7E3ABEEB7A39BE82039B3CBC
:1068D00089EE1CBDA8997EBEB9D0563DA07820BDDA
:1068E0000814113E7DAD403ED8BE0CBEC02C7F3E8C
:1068F000A277933C4E8F053D86FE3DBDDEBAA3BB1D
:10690000984A8CBCD8608DBDEC84D73D760C053D93
:10691000FE59843C510810BECFE7D6BD8717C43D51
:10692000475C103DAA96183C3B45B4BDE515E93DD2
:106930006590F0BC8FBFED3D7D7CE1BD021ACC3D82
:10694000ACBBBC3DDD952F3DB5182ABE2C7245BBB6
:10695000A354993CB793513C9C2B15BD5C57803C8C
:1069600016AFB83DE2035E3D2F307C3C1194F73CFE
:10697000F9BB3A3E1597B93D26A90F3E536F7F3DAF
:10698000752AB9BDEB28D2BD3C4498BDC58E23BC49
:106990004CA685BD72BA10BE21E0973D528ABA3C22
:1069A000A33EE7BDC1B78CBDE14A463D796036BD27
:1069B0008FDEFABDF15A033C73F17DBDCD270EBDCC
:1069C0006650D63C6C9E653DCC48AA3B3B718FBD62
:1069D000EABEAB3CA82835BD27D231BD0D7B34BD06
:1069E0008A61BCBC8F95BBBC6A7288BD06B933BDD9
:1069F000755482BD3E66A23D5BF3D63D960A13BE3A
:106A0000416D3EBE9C5B66BE7FF846BD8ADBB73DEE
:106A10007052853DF0E536BD4C99223E4F5323BE62
:106A20004239C53CD8DD083D6B0D57BD694CA63DCC
:106A3000ABD6EF3DE85C853DBE3A34BE64C243BE92
:106A4000AB8C84BD14D93EBD50C4463EBF77803D5B
:106A5000663C49BBD82D903DAE15773D56AABFBDCB
:106A600021BE1CBE6D1CD93DD7AF3DBC91E11A3E85
:106A70000B19E8B9F18862BDF8C4EEBCDC413A3DBF
:106A800037462F3D2F2AD93BAEA4653D97F1E5BB94
:106A9000026C88BD1F36563D8171F73BFD4988BDAC
:106AA000CFD08D3D83A834BD32BCA5BCCB139B3D5C
:106AB000BA33333DDE7D08BED6E6063CCB1B11BCA7
:106AC0000776433DAE4E08BD616BF7BCC020CF3C9E
:106AD000F80325BEB7ECD03DB8AF6EBD121C293C03
:106AE000AF728B3D1DBAB2BD0728C93D65A3EC3D11
:106AF0002B99BABC526531BD3B33163DEEBA98BDF9
:106B000089D72FBEEE3F68BC57C68A3D58FD153D5C
:106B1000549F833C513CC1BA48E1B33C351E0B3D08
:106B2000104726BD93611EBD6C43F3BD02501D3D51
:106B3000EE6A873D9A57A83DFA8AA83AADED1EBD88
:106B400031FA9F3DEA7D7B3D3E46B7BD12038FBDC6
:106B500015992DBD0DC313BEB37F01BE84B0E93DB1
:106B6000C8F6D8BD7A4618BEDB9053BD3D867E3D43
:106B7000D994ABBC70B4CEBD82CA213EBFB96D3DC5
:106B8000EDFE843DD379033E51B1D3BDCE52B43D29
:106B9000BFBDD3BC0B7F28BEA5EDC5BD7305A43C0E
:106BA000FF302BBE2279E43DBE6514BD9AB7FB3C95
:106BB000100BAFBC362E653D39A231BEB762993D90
:106BC000FDCFCF3CC5F809BD5593D8BCB93A88BDB7
:106BD00029DB2B3DAF9F083D486CA1BD4CA51DBDD9
:106BE0009998133D9213C1BD3AE0583D54334D3D41
:106BF000A43B8A3D2CA381BD95A9BCBDBE8BE03DC5
:106C000044BD8EBDAB20A03D2A6905BCAC80143EBE
:106C10005A5A123CADF422BEF813A5BD1199AD3DF0
:106C2000A83DBD3DBFCC90BD422905BDF237613DB9
:106C30000717BB3D4DD1A3BCDE6BD0BD9A2B98BDD1
:106C40005BA7BC3DB8316EBDE8BBCBBDE08AC23DA1
:106C5000DA52E23DD0B1043D7A9B29BC8D4D833D93
:106C60006A4ECCBDECC4BD3C14D9A33DEC94C9BC68
:106C7000CA64BEBD2731EE3D9278DEBAD4CD33BEB4
:106C80002795383EADECB2BBCAC441BEFB492B3D93
:106C9000DA9103BC052091BDA3C0A7BC427FF1BD22
:106CA000A541363CD16A87BE71DD80BEE583EE3BEF
:106CB0002A48133E51E1313C3592BD3D759E0BBCD7
:106CC0009D3997BD901B053DF3319D3B8D9A183C36
:106CD000D24D0F3D58F0C9BDC86D623D9F89883DBA
:106CE00011341E3DA15FC13D007EB83D6048413D6D
:106CF0009D35D93D3F06E23D703D8F3D4113053E38
:106D0000154BA8BD5C4C8BBD6D23B23C6CB914BE59
:106D1000F473953D3B987E3D4A8EFBBD1198933CA4
:106D200040D3D13A1A342EBE875BF33D20E612BE23
:106D300019AD3FBE7ACAD33C02678DBDF47E403D9B
:106D40001C2EE83C6ABD5A3D23159B3CADAC06BDEC
:106D5000AAACE43CB8793A3D47CCD63C837B89BDAC
:106D6000004C8BBC8DE147BDBAB75A3BDCC746BB74
:106D7000D8DEEC3C57C6493D88D8A2BD45D43A3D43
:106D80002F606F3D6F9CCB3C00A91ABB925315BD81
:106D9000708D173D4A851D3D2B59A1BB99A5BFBDDF
:106DA000848DBC3CA290273C2BED423D0305AB3BC0
:106DB00032FD873DB3CB35BDB5D9193D5076313C59
:106DC000CA04FBBCCD345DBCD18CDA3C788B493D28
:106DD000AE78AE3C95D608BDC175633D1A07883DB7
:106DE0000F5451BD5F7757BC4CDC673D15D9403B14
:106DF0000E93EFBBFEA265BD382AD33D44CB56BDF2
:106E000013902EBD6C2FFCBD05EE7BBDA3578BBD33
:106E100092ED0DBEBC6CE63DED94ABBDEAAD1B3E04
:106E20001618AEBD9C7D07BC06DDA2BD351617BE8B
:106E30002407A8BD9EDCFABC85EE88BD5A16C03C6E
:106E40004065A13D29F9EC3CF6A1BCBD8352993DBA
:106E50003789963DD06D603DED7783BC2E45BC3DB6
:106E6000977C59BD349B033D9285DF3C2EC50B3D7D
:106E70003025D2BBEEC209BBB6F737BDEC2021BE30
:106E80000FE357BD73511CBE8AA2233DC6BC963D7D
:106E9000FFB22CBDD04A48BD3F07B03D5EE8D53DAE
:106EA00031560DBCADF9D6BD6E783DBC1D2A8A3D6C
:106EB000E5869DBDCFC015BCB966223E164533BEE2
:106EC000BBA659BD720184BDA22B13BE3E11B33DBA
:106ED000818A1EBED8CE113EAEA698BDA8F037BDA1
:106EE000E190D7BC78803CBE0D785DBD7C6F233EC1
:106EF000C5FD853CA85992BD8AAF0E3DC029B43D61
:106F00008DDA7F3D2071DA3C6091A13D02CF043ED5
:106F1000D7A386BCBF97B43BF78B6DBE01E1C8BD5C
:106F2000EF54B2BDA199AC3DFBA9343DE21050BE77
:106F3000F7058BBE5395683D4D5B3EBDB3AFB13C8D
:106F40007FA4623D87044E3D10493ABD623D66BD57
:106F5000F78AABBDFA71083D1DE4433D70D7E73CAD
:106F600033FE363DB538CCBCDD0787BDC310253DAB
:106F7000FA484A3D0666D6BD3711C03DFE6DA2BD3A
:106F80003F1CC1BB29DDEDBC2F936CBDB8F0623D49
:106F900060E1063CA2A5A0BDA09CC0BD9F1DCEBCCB
:106FA0001A9395BDB0FE8F3D537001BE01E3CABC7C
:106FB000AA025C3D8F03393DD3F36DBDB12C7B3DFF
:106FC000F6E428BE8481223EF185693D08DE82BD5B
:106FD00085AD573DA8EB97BDB0B1C23DCF0378BD9D
:106FE000493C193EB2DFE53CC376713DB11C8BBD17
:106FF0006FFB773DDBD064BD4B6733BD1A3B5FBC95
:107000003841D33CB80F273D707B16BD46578EBD27
:10701000D1E8F83B892DA3BC7F74D4BCFF1757BDC2
:1070200022AC6E3DD786EEBC2B6F303C17E3A8BC7C
:10703000434F8B3D2650183D1C29E4BD42683B3D23
:1070400004982EBD7BBA3D3DD3E9603D76A28C3CD1
:10705000D397EDBDF102933D236E623D3630B9BB4F
:10706000A0CD15BD3F5EC23DA4C3393D2AC2E9BCD7
:10707000613B13BDC293FFFF04000000001000003D
:10708000A4F93B3E29C1853D541BE43D7DABEEBDDB
:10709000C36F243DCD8B463E605C1DBEDBDA2BBE4C
:1070A00099DBA5BDA51934BE594D7ABD2B52EDBC57
:1070B0003682443DBA2131BEE41B7A3D25D1A23B44
:1070C000494090BD6C2998BDEE02C5BDDCCC1BBE0D
:1070D000164F533E7B79383EE71DB2BBBA1C843D48
:1070E000BE61933C37D2463D211299BD1A065ABC67
:1070F000382EC33C0EE62F3D409BD63CFC13B73DDB
:10710000A76C4BBE907F073EF1AED5BDFACB073ED4
:10711000FE5A3B3E9FF126BE2988693E83605DBDD5
:10712000FFF89FBD2CC7AEBE0C3539BE4E1AAABEA5
:10713000AFEF99BC10140C3E778F00BFE54F733E44
:1071400041FFB03E7F888EBD32236C3E4171DABD77
:10715000A98560BDC39A5B3D636363BE9E1799BDFD
:107160000AF2AABEC7CB58BEBE7D8ABE7DA48E3DA4
:107170007F6B15BDE3673B3E3A9604BEBA919D3ED8
:107180003593333E7D808BBDACDD953DCC8C073E89
:1071900082FC613CF817613E48AC2A3E2622343E10
:1071A00033171FBEC9F70E3EF999363EFCC2323E78
:1071B000D36824BDAB81173E29E821BD394B953DED
:1071C000DEA33B3E611D253E1BAAF73BA1C6BEBC0C
:1071D0004C7299BDA985163E532F99BDF7466C3E5A
:1071E000F35D6C3E3456683D489F1F3E2A43C93BC1
:1071F00019F3493E0B48203EB3A34CBDE218EDBD48
:10720000AEC312BD8F63133E4C5B093E6DAFAD3E06
:10721000E00E913E2D49793D1CAA6FBEEC554B3DC9
:107220000708E13DBAAFD53AEB198F3EC2A5F2BDD2
:10723000AF91703D37B3B13EA0E6043E87812ABED0
:10724000BD90573DE149A8BD0897BBBDD287013E1F
:107250000FA7AC3C6EBF9BBDDAF75B3EEA0A543E1B
:10726000376D2EBE17E50B3EB6303DBEA6FBC8BD42
:107270008EB8AF3EC19915BECB8CB83EE6E2AEBC2F
:107280005A47893CCFEEEFBD5C2D4E3EEB1720BE3A
:10729000A430803D15E265BED69417BECF7ACBBD33
:1072A0003C6AFBBDC5B48EBE886202BE13DC893E5B
:1072B000ABAF9C3E2BCDE63D01AE41BE183DA9BE15
:1072C000ED3643BE981B88BE653732BD527A6A3EA2
:1072D000DCC5013E813E20BECC250C3E426B813E8A
:1072E0007F93793EE19681BE65AE28BE5E9262BE16
:1072F0000CF783BE6AA98DBEDADE99BD83BC08BED9
:10730000A6C3B73E26D2923EE63217BE58A2943E9E
:107310001BEB323D6B444DBD28CBA93E360295BEDA
:10732000FBEC79BE9A2C123E6C6602BE2CD08CBD52
:10733000B7197EBDE1906B3E4D8326BE2137D7BD88
:10734000D9C19B3D3C4531BE70D05FBE9C35BB3D35
:10735000C8947E3E40BA8A3E274D67BE09478EBD1F
:1073600024273B3D5868C0BDAAB0493E69430A3E48
:10737000BB6F52BC1B4CD5BDA4BE93BE8A19CB3D7E
:107380001EC75A3E21817EBD2F3115BEA6167FBE77
:107390003F8E5D3EEE1969BE2A308FBD9F081EBE2E
:1073A0009C6F2F3DA38A8F3E4824223C18670A3EDB
:1073B0006073A03E9A8E14BEA4C92DBE53C48D3EE8
:1073C0003A1357BEEE50B33D0351743E78B43EBC01
:1073D00008273FBE63681F3E7537073D93D6A53D1E
:1073E00020F9BE3E9EA50E3E9F8725BE801C28BE6E
:1073F000365B5BBEC12DEC3DA1A135BEEF8DC13C1E
:10740000D64E403EEA6DD43C125789BD5EF2293E0D
:107410003118403E2F2C413D800E3D3E871652BB19
:107420007B51A03CB8AFDFBDC58EEBBDAA46143D75
:107430000679A53D1CDE063EAEC3F1BDB006FBBD20
:10744000B393C93DCED971BCB05720BE2B595DBD99
:10745000B9DC7C3D35E89D3C1C146F3DF0BA083D1D
:10746000BE0EEBBDF67949BAD887A83C6FE7623EFD
:10747000DC84A8BC60E6383DDAF19F3B9495173E6A
:10748000A755683C1E30A93D1D6E783E54D41B3E66
:1074900074BE16BD33A9D63D7C9D8D3D798B4ABB0C
:1074A000FB34553CE5F408BD56F5F4BD763E1B3D76
:1074B000C570013EE78E1A3D0B55303E603D283DBC
:1074C000BE17B5BCB1A1063DFE770FBEA67E203E1D
:1074D000820623BCCEC3B03D359A283ED95DD6BDC9
:1074E0007D93163D843E0DBD7C5D2A3E3177863D01
:1074F0003746633E47683D3E08EDE4BD2A4A5B3DA2
:1075000036C10CBDAC48083E465BCD3D8C2F05BE58
:10751000A12D85BD979FA93CDA1290BD377E5D3EB7
:10752000A7551D3D5A8F3A3D1BC33E3EF5F9B73C6A
:10753000B9F4693D667DFC3CA7C6C6BD1E7C8F3E86
:10754000171E5C3EAA7197BDFCFD863EDCA7D13DAF
:107550001A85D8BDDDE0343E9BEE28BEAED830BDE6
:10756000C0155F3E47A84A3EA72DB7BD3D271C3E2C
:10757000F240B63D347A4FBE32B382BDE00E633D79
:10758000AFDD953DBD12DDBDCDE101BE2B902E3EA0
:1075900055BFB3BDCB80823E5662133EA405EC3B83
:1075A000FEBFBA3D661B9A3D180F703EB2E7153D0F
:1075B0006DBD853B78C522BE338C31BED2839C3EE7
:1075C000B177983E2F1641BE5701DE3D3482493DCA
:1075D0000367EEBDFFBBBCBD618EF6BC7E45923E2F
:1075E00016E53E3ED7C877BD6D69023E79F2B3BD60
:1075F0001A7F733C103E293EDA49DABD5E2BA2BCED
:1076000093995E3E7F5E29BEC0A6A7BDB4842D3E81
:10761000CC04B73D84A4453E99A9E5BDC38004BC14
:1076200042191B3EC9CF563CE96C07BEA103E7BD1A
:10763000AB109FBD0D8B543E4C47763EF3EC783C2F
:10764000051F273E50EE31BEEB5E74BDDBCFB73D6C
:10765000D1DE053E8E3E293E9ED4B93EF5D4203E75
:107660008B7E1E3E0B62EABDB791033E9AFA013C47
:1076700064D71C3E70CD35BD47D6F53DB45B153E95
:107680002205DF3D15F5213C9DBA99BB0AE5AD3ECB
:107690009881973B4139893ED03867BECF51983D9C
:1076A000AA56DD3CF291C1BDC099CBBDB4E161BE2B
:1076B0007CC0A5BD6E021FBD73450A3DBD6408BEFA
:1076C0006940583EE71E563ED7855CBE3A00F63DFF
:1076D00028C1643E6F1D28BEA5A8013EF50918BD4E
:1076E0001354023E1A9B303E33A6E4BD22FE623E96
:1076F000AF03F13C1EE5513ED633BABD7DF2933D5A
:107700001EC6F3BDF6F17D3D221CA83DB87FE13CCD
:10771000E530B33E94A88F3ED36641BE9404B73D96
:107720008C65533C4FEFFC3D14312DBC794BC03D73
:107730006CCD08BEF329C3BD249803BEC5B68D3DEC
:107740005ABA123E0CCC413E73D2B4BC5B6E343D8F
:10775000442F863E26EA0EBEB323A2BDE026A7BE76
:1077600085FDC4BD57B506BE447B653EED396C3D15
:10777000F80D8C3E1F149C3D278B4E3E47C73C3E68
:107780003D4E643D571F6C3D2E1982BE97D54BBEB2
:10779000B7A67EBEA0EE86BEBFFD07BE1AEAA43E17
:1077A0006D5017BE24BF8E3E9BFB093D8DC001BDB1
:1077B00098897B3DA7CC9EBCC76009BE7E2A043D4C
:1077C00074C461392627263EA0AF80BD4137783E7C
:1077D000A013653C04ECC73CA1A5603DFF489A3E60
:1077E00003AD8FBD8ADFD5BC09E089BEEB41233DE7
:1077F000BF798E3E433417BDBCE7BC3DD61D433C2C
:1078000076D7B8BD11A84C3E6FBB4CBEABB3A23E01
:107810000206FF3D1B678A3E796F18BEDCBDDBBDEB
:10782000D5302DBE94DDA9BDB63F373E58471BBDB0
:107830008C1DD1BD6ED78C3D971CAEBD45FF91BD53
:10784000EF92C4BDE023563DF638F43DF807A83E5C
:107850004503103D78387D3E4616AE3E272E97BD37
:107860008C1F603CE90D7DBDB576CF3C6614ACBD88
:10787000903D18BECC105ABD6C3794BC3B87143C6D
:10788000E5977D3DF2541C3DECAB553ED421873E3F
:10789000B49BB9BCFC0EBD3EFE8B293E133923BC04
:1078A000BCFD363EB07EA0BE5A1FE83D57DE333EDB
:1078B0006E428ABDB5444F3EB6B41EBD1BF4EDBD4D
:1078C00095D723BEC3750ABED6E8003E961247BEC2
:1078D000C3AA1DBDCD9769BDB6FF7C3EF9F91ABE9E
:1078E000DF65CD3AF473D1BD59AF663EAC3D163E6F
:1078F000FD8FB93B06BC653DC522E0BDC1E6073D35
:1079000048272ABDC10DD2BDB165A23EF7F6733B33
:10791000BE39A53EE7DE773ECC0F97BD4DEC003E6D
:10792000E320323E3BD7003D461E1BBEFECF45BE88
:107930001AD8A43D181EC13A60923EBEA0E105BD12
:107940004DF44DBECAF6133EBDC2033E72327C3DBD
:107950004C7044BD2424BEBD8DB2AB3D2FA82ABBC4
:1079600065BB943DCD332A3EFCC3643AD5855CBEED
:10797000E0950FBE20102C3E58A141BE5E08063E89
:10798000563A233EDEBFEFBD653F33BE40C2073EE1
:1079900020E2F5BD1AA7023D63D5563E4A65B53DC6
:1079A00051A91ABE7527DF3DCC5C00BD6C42143E68
:1079B000686A903E1EEAC33DE10EFEBC1712643EAB
:1079C000B756A73DEA4EE0BD5F88743E10D0C1BDFA
:1079D000A34459BD394C1A3ED50850BEBCD7483EC9
:1079E0004D236A3E8C80323E564F9E3DAE7F343EE4
:1079F0005F8B983D0DA90DBE5CF54EBCA10444BD46
:107A00005173033EAC9C8DBD0E62F13DA1A9A43D16
:107A100086BD873D61F07E3DFDA7E2BDF84A29BEE7
:107A2000BAF736BBCAB3C1BDE7702FBD8F11ED3DAC
:107A300095C3D93C51A5013EAB28A5BD1944B1BDA4
:107A40002A2BE0BC1D0962BDDA36EEBD10C9F83D37
:107A50007898673E177565BDC7FA383D358C62BDAD
:107A600085A3913D21B1FC3DB605593E4E3A77BD07
:107A70002C0E6B3EBF56D33DAEDCF93DA866C93D2A
:107A8000F3A8703D6A9C3D3EBAD0A9BDAFB8FABD1F
:107A90002C3F653EBDAA7D3CBD7DF43D9B476C3DC2
:107AA0003CA7E33C02A58A3D6D236ABC0B76423EAF
:107AB000E6B53E3E047445BC772233BD1285D0BB8B
:107AC0007B5B793E018F84BD2EA961BE1D6A403E5D
:107AD0003E4C113CD67C323E2AE02A3E29142A3EF6
:107AE000C6C497BD9135EB3D4C855E3D7DD8683A67
:107AF0005245BBBC109A9C3E734C323EFCED12BE0C
:107B00009C82A53C5609C2BD1C2DED3D4FED5D3E4E
:107B1000CD7C6FBDFD6ED3BD9199FABD60EC8CBE7E
:107B20006FF35FBEBECB73BE04F335BEDA60A73C15
:107B3000453934BE81AC3D3E6672173DAA8E48BEC3
:107B4000FD401DBD5DC7493ED0377C3D1953003E09
:107B500068CB92BDE1F4533E760892BBA572E3BDBB
:107B6000E45F62BDB82BF2BD0C92163D4A971B3EF6
:107B70008DA6663EB77AE53D880F28BE7FE5373E85
:107B80005979FF3D03181EBEB29A493EF45DA23EEC
:107B90008BE02BBD3944123DA63664BD6A50CBBD87
:107BA00068B22E3DF549FDBCE9E907BDB6083BBE0C
:107BB000B2757E3D1911343EB572373D89BA88BD24
:107BC000ECB4453EDBF1863E25AF213ED6BE753B8B
:107BD000E4EC5E3D59724C3EECB9B43D99E324BEF1
:107BE000E501E43DFFFF15BE30FF823CDC34483E3A
:107BF0008A0DEEBD07CD96BD2123883E61148A3ED5
:107C00004A57D8BC2A8790BD13C6153E275503BED8
:107C10002A035BBC48472CBD3FFF613EAF96ADBC1D
:107C2000F31650BC7AEE893DA40E7A3C00265E3EE7
:107C30006604893EC55A50BCC118863D61889B3E8A
:107C40007BE05E3E0E1316BEFC74233E801E4F3D4D
:107C500019891C3E89C5B7BD5CB1933D9893173B0C
:107C6000F04DE13DFCEF543E83A03ABD03A68F3EAC
:107C70003B1FE3BDDF36043B7E61FCBDBCDC6FBD5A
:107C80008F866C3E8F507EBDA0FAFA3C678D113E08
:107C90002C61D73EDE9ECA3D23C1AFBD2BBA3A3E12
:107CA000C00B493D8564873D5300DABDB50FA83C44
:107CB00085D156BEFD2E9EBCF261063C70F9353C66
:107CC0003B556F3E9075A63E6810443D4BDA033E2F
:107CD00041195F3E60AF0BBE7038D93C6E720DBE6D
:107CE000BE5C1D3DCD2A10BEFB5B513EC9C600BE29
:107CF000BCE6EB3D8E90B93C2ED42C3EF406163DEE
:107D00004A611F3DAE4D683EAA1887BD9CE7A3BDE2
:107D1000966F583E96BACBBDDF0F75BE043947BD8E
:107D200029C8E13DEDCE15BE5F791EBEF67055BC8B
:107D3000811D2F3E65BB62BE0998FB3D5D71E03D34
:107D400096D038BE4113FF3DCAE484BE57A474BD2B
:107D50004499523DF80D8F3E3BF1FDBDD6577ABE9A
:107D6000323868BEA559CF3C8C5D343ED9DE863EA4
:107D7000AC037EBE051A27BCE27454BEB9213D3E59
:107D8000DD1982BE59ACE53D6B9C5EBE1226CF3D2F
:107D9000A829663EC579963E9A95A63D0EA42DBEAD
:107DA0000596E1BDB6F03BBC7795033EDE6C1CBE8C
:107DB0009CCEBC3DE58659BE069D9CBE43E5463E35
:107DC000A0A63F3D6B680FBE31215D3E5EB2B2BDE5
:107DD0004CE12F3E6753DABC939C753E9F2547BE0E
:107DE0004B9E723E846F1B3EB25C283EE89705BEF8
:107DF00068C13B3D9D81AC3EB2820F3E6052AB3EBE
:107E00007325EF3DDD1E23BD5D1F1FBD35C7583EE9
:107E10008B390B3E62013D3EF9753FBEF9D6C53D3B
:107E2000BB68A5BD0079E9BD2368B63DE1E6BE3B70
:107E3000AA82EC3D8C41F1BD15DFFFBC76A6AA3DC0
:107E4000DB26B7BDBE411C3E763BFBBD63FE1CBDC1
:107E5000D5C2CBBD9DD86B3DB9F5843E668F99BD2B
:107E600078263EBDDD46BB3C4CDB543D4AFFDC3D45
:107E70009F5E423EB51D1C3DF71D533E8E59713D20
:107E80007991D2BD113D81BD9164323D43518FBD89
:107E90003B3F953E6D32493E45C02CBD66369C3D0C
:107EA000E8095A3E00E9023C75F4143E044063BD03
:107EB0004304A63D6ABCE53D490124BE8CE6CB3DAA
:107EC000CF689DBD12EE023E56E6983B7BF145BD64
:107ED0004D59503E4B1D1B3EBE5AB33D8850A43DEC
:107EE000BE983C3DFA05893D6E504DBECF377D3D75
:107EF000F1F1743EBAAAD23C288EA03D9602C7BCCE
:107F0000111C093E24F8313E4505B5BB6A309CBEC4
:107F1000707104BE9E647CBE167D1F3EE192383DAA
:107F2000FFB4BF3D1C5B48BBBC8388BE922596BE98
:107F3000EA2A4839570B1C3E1423973EE22DC13DD7
:107F40009E40003E88A6E83DE1B5D13D69013E3E38
:107F50001DD21C3E6C5B93BEA0979EBDA54D853D7A
:107F600061A759BE2C8A773D8C657B3DBFC494BD0B
:107F700079284B3E37CB61BEE3EFDABD0A441D3BA7
:107F800044825FBD4367BC3C49E1EE3C2CCA0A3DDC
:107F90009649813E3407163E653ABE3D77D4CFBD43
:107FA000A71E3CBE1161D1BCB43E0C3E428C3D3E8E
:107FB000E3919C3D8124403D83AFD8BC0C76A83E24
:107FC000BB79853E9E76CC3D05EA32BB90D32E3EF2
:107FD000A4EBCA3D7296C73C15F28C3EC75F6D3E5E
:107FE000EE0C9E3EABD0603E0225203E1EE7BD3C1F
:107FF000955CA93C12FF99BC87833C3E80F076BC1F
:1080000018858DBE2BF1D83CE52B3B3D991977BDEA
:108010004FB83CBECFBDF83D675BC7BDEC8169BDC5
:108020004526F0BCD1880F3E2FDF543ECE51823D15
:10803000F84511BE5AC3C63D3DE2BD3D7544E93D1C
:10804000121E853EA546353D5A07193E5E3186BD56
:108050007666223E995120BE00EF163EDCF4923E39
:108060005CBE843DED12DD3DF312873D8A461A3E2B
:108070009BB9D53CFE2EB7BECE58BF3D3D73A13E49
:10808000CEA3FFFF0400000000100000B1DA0D3E97
:1080900031452B3E36A5313E72DA243D46ED9E3EFB
:1080A0006516E9BC8A51C83D678B46BEEED41DBE3D
:1080B000651A8ABEF4F6E33D82FE9A3D4A20F3BC7F
:1080C000A8D5383E444D663EF925E7BC04CC993D21
:1080D0007ABE9B3E5B0D80BE0F1906BDEA18A3BD9C
:1080E000F6D0113E096B8EBC138DFA3D76348D3D72
:1080F000ECAC1DBD60FC703C44D138BE952D463EB5
:10810000D1E1663D9BA4E13CCEB51A3EEE243EBED5
:108110004D2E1D3EB6332BBE04B9D7BDCAE481BE79
:108120001B71F63DF98F353D39818CBD5832333E98
:108130009D027EBE8AEC293EEDB27D3DC100CA3C67
:10814000945F14BE528480BECF3B20BDC11365BE78
:10815000BBF1A9BEA3317BBEEF23A73DA6AF09BCEF
:10816000D6E527BEE434B23A58F536BE53A46CBE09
:108170008CAD35BE152455BDA96472BEC15372BE07
:10818000181AAABE150DEA3D29A1AFBD080966BCA3
:1081900086070DBD5A6D91BDC73836BDB05150BE72
:1081A00014004D3E698E543E56BD653DFF9B723EA8
:1081B000E499BD3D33E53A3EC1B7803C32CA353E15
:1081C000E69E93BE6730C9BE6BDAC83E8BAB563EA7
:1081D000005A8B3DA359D3BD47FFF73DF455ADBCC5
:1081E0001BDEE7BBAE7251BEB0C89EBD7EEBA03EAB
:1081F000B8F6AD3E79CCDA3D3E29143E8027C4BDA9
:108200009E045ABD434B5ABEEC0C83BD5DFD243C1D
:1082100055B1BCBD504A8BBE562F3E3C197128BE8D
:108220009B8D11BEAA227C3EC05ECD3D1C340C3E0F
:10823000F5E6823E963F4E3E6CBDA23D396EA13DB5
:108240002D9E01BD28F7C4BEC2F0E03C856E95BDF1
:10825000506AA23C41229A3E090BB73D9E999F3D30
:1082600063AC913EE2FD8EBEB92F1C3D5129CA3B45
:10827000080C1C3EBBC1F8BD5A0C4B3E43C2CBBDE3
:10828000877F913DE63F5DBE2FF51C3E866F6D3EBC
:108290002714DBBDF155F0BD8FA96F3EC4E354BD7B
:1082A000AF36CABD12023EBD0975FC3C1445B93C4F
:1082B000E758D63E3CF9AD3E62A3243E6F46C23E2F
:1082C000DF6655BE20249ABDCF07883E5530AC3EB0
:1082D000D08862BE7FB336BE82BBFA3DED634FBD30
:1082E0001514823E404B0B3D066CB63D60D91D3ED9
:1082F0002458043EF7DEAD3DDC7A30BE0945B2BEFF
:10830000DC4888BECA6A24BEABE78E3C85A8C83D5F
:10831000F2FC98BE9B4D9D3ED89C5E3E2AA9CD3E68
:10832000AD29563EEB2E903E5A56E9BE2D8AC93EE7
:108330001172FEBE2F0AD13DA8804A3D8AEC59BE7B
:1083400067DDA5BD28F7013FF4A866BEE57D47BE01
:1083500093D564BEFC05843E44D49C3E7F4325BE39
:108360006D541DBECAE7963E2D9BADBE275F233ED2
:1083700093FF92BE8540FA3C3BA78CBE896350BEFA
:1083800007C110BE9DC37C3EBD11B0BE4B80893E6F
:1083900021E2B4BDB4B1B3BC34E12FBE5361003EA1
:1083A000B4CF143E348E883ED8C123BE599FC8BD79
:1083B000292C05BE199C553E349F983D7C88993CDC
:1083C000F35D79BDB33E2F3DF318B8BDC46843BD1E
:1083D000FE5D9E3D8E1370BD462F6DBE6EF7B33CA5
:1083E00080F9493ED8C1443DF7AFCC3BA8ED6DBE06
:1083F000655011BE04DB053C8B93783EED24393E7D
:108400005AF903BC6C63933ED739FF3D421E723E5E
:10841000BA6C6FBD68EA273EF7ECCC3C21C6A93D9B
:10842000CB288F3E59E9313E4FD9B1BEBB696E3D75
:10843000F9F86ABE72B649BE8D9020BE6533003D24
:10844000DE220FBE0CAE113EF6DF3BBE5B3EFCBD36
:108450000D2D333DC107EBBD0B4DD8BA3CE01EBE20
:1084600005272CBE5924AEBC1012DDBDAD42313EF5
:108470005492AB3E453B5A3B32BC243E074F3C3DF9
:1084800092EFF53DA9049F3D3984B03CDBBA84BD31
:10849000F0CCAABDE3E3B9BCF42C86BA0D0B39BE0F
:1084A000B30E0E3EA510EA3EEA75CC3EE07A093ED8
:1084B0009D85813ECA428A3EF956EF3CAA05EC3CB6
:1084C0006291113E60B27BBEEBA6093FFBC1713EDB
:1084D00015E4CEBD04F73CBED70B6EBD02CC1FBE6B
:1084E0001987C93E3A4B5ABD9562373E0C721F3D03
:1084F0007BEC263EC3F40DBE2050BF3E885BBA3DE8
:10850000355516BE773FA6BEEBC36FBE56FB013E88
:1085100068259B3C38BB5B3D7B6C143E089A163E3D
:108520005EDC2E3E4F69593DF4CF0D3EE7EB31BD89
:108530003A1C223E6AE271BEEBF1003E5AF2BEBD29
:1085400063FC8D3D25A1DD3D825DB9BE6EAB90BD66
:10855000898D5BBDBAD10C3E252340BE3C88B9BD98
:108560006BA4FBBDBD73AA3E047DD0BDC74E81BECA
:1085700018748A3EDEC2693E55083FBEF99C723EC1
:10858000FB9EC23DE589F53DFCFE053E4BAF3DBD82
:108590006488583E607095BE3FBD26BE491462BED9
:1085A000296D64BEB74C203E2C547D3E29A505BEE6
:1085B000A1491CBEDDC7803ED9F15DBE949F2EBE91
:1085C00046D3B6BE9ACC67BEF924503E22492B3E14
:1085D0007DDA933E14B48F3E51998E3E8BB428BE03
:1085E000B1E71E3E0166B0BEA96E07BED12C37BDF5
:1085F000E94EB6BC58C3B7BEF301A6BD1C71C83D59
:108600004DF6B03B0A91F6BD65D8A43E5654323EB5
:10861000FCF5873CCB2941BE38AA66BEBF53C13D9D
:10862000EC9D6CBE416AB63D87BE963E9CD2F2BEC2
:10863000D78040BD243785BE618540BDD066B83D3A
:10864000D429483E641E81BDC1C80DBD192F8ABE04
:108650008931A8BE38DDAFBD0CE98C3C099A81BEDA
:10866000CED31BBEBF5B88BBDCF105BE68E459BD41
:10867000031780BE3271E7BD8C4ED43DC4843F3EAB
:1086800005D330BE5BE8A7BEC18114BD3E4248BEE3
:10869000FE033E3E0DCB823E8DCB3CBE9553353E18
:1086A00083C6A23E9F81E7BDB2BF6F3D97C098BC15
:1086B00057A9EEBE2CBD67BEC759E5BD03CA66BD4E
:1086C0002C7A363EA5FF423EC98F1EBEC15543BD22
:1086D000CF63E6BD7F7CBD3D3F16BDBEE89E41BC7D
:1086E000CFEC9E3C6F931B3E6A4D503D7B5FF93D46
:1086F0001DAC263EB1ACEBBCD66490BED8694ABD79
:1087000003F0AF3E51817F3EEC0F26BEC659CFBD70
:108710008A57883E9CF46D3EF5175A3A5AC464BC99
:10872000D073EF3D40DB24BE423CE0BD8AE7243EEF
:10873000CE2E273E5D6BA5BEE36194BE3FADA63D48
:108740001CB2483E48A0043E538E7E3DACA32ABED8
:1087500058DCEC3C28FA89BEFA99D03D9406213EBB
:10876000518895BEF95B5EBDC8F14C3E73500BBE9F
:108770000C6C053E54C3373E90E23C3E95C75A3ED2
:10878000E1DC233E4E71BD3D25863B3E4F07DE3C7E
:10879000A7AA843D88AFD23CDDF323BE0B7B44BE49
:1087A000F2D711BD779799BDD9BF113EDCDAC9BDAB
:1087B0004B4298BD1B65423E6FF658BD9B5BBEBDEC
:1087C000218953BE53036CBE3C21323E600B86BDF3
:1087D000086720BED0A9DD3DAADDD5BDAF5845BE96
:1087E0008A3FE1BDD44D5EBC850A633CCDCF153DCB
:1087F000A702F2BD7EC012BE2A56373EA48CD3BD5E
:1088000097A007BEEDEA5ABDB3E5A43D94194BBE4F
:108810006E1FA83C58F4DCBED7318A3DF9E09BBC02
:10882000AC40283DE469ABBDB824A83EE2BF13BF0D
:10883000DF5C5F3E36AF313ED672F73D1699823E21
:108840004A1DA03D6E16013E175072BE8BBE81BD03
:10885000C3ADA23C805BD8BC8049A0BD0819A2BEB4
:108860005A6F50BE527938BE9756AF3EE22BA7BD25
:10887000F65642BDD4098E3D0336893E054BD9BD1F
:10888000F55A38BE1979123DCCDE473E28621F3EAC
:10889000A8E8813E101AA53C266C8A3E379AC03C57
:1088A0005EC43BBEC0BE803CAB6F393D24591FBE89
:1088B00056988DBD8C6E7FBE22E757BD7A060DBEE1
:1088C000A074783E0B14B33E0CF23B3D0EC3EFBCDC
:1088D0001787393EF87EF03D175B3CBE47C8DD3D4B
:1088E000B10333BE1A5F10BE76DE63BDEE64303E68
:1088F0001A45883D5AB10F3EFE077E3C73EEC63DD9
:108900003A099B3EA9A6963D6D8B0CBEAB75A33D67
:1089100044CD1EBDBA1FB53DE829833E5C2C7C3E8C
:1089200050D5433E6B81093E867F8EBEDCD9473CE5
:108930002082603DAADD6B3C16D2073EC7392EBDB2
:10894000CBE41E3EE2D9103E13CE28BE6E2B3EBDB8
:10895000BCBD323E47888C3D54CF64BEF3F818BE90
:108960006A58303E6E8F603D8E9840BEF3CE3D3CDF
:10897000E009F5BC215FF7BCB9178E3DFEB3F13DB0
:108980001138893DE42345BD8194C3BDAB9EB63DFE
:10899000BD4C02BEE34AB3BD68B883BE2A7EFCBDAF
:1089A000CCA0FFBDF5C0BFBDBA91833DEDFC57BD66
:1089B000ADB6E43DAC3A813E8961893D92A9963DD0
:1089C0001762163E350566BEF455703E8BEF773D57
:1089D0006F4A1FBE5C25573E7C7FDB3D4629D1BDDB
:1089E000CCEE183EBB5203BDA112293E2A6E403E7A
:1089F000900A8A3EBA25F7BCA6149ABD16CFC63D8A
:108A0000C1B221BE34372ABE7F0D16BE8F80F1BDA4
:108A1000EAB144BE15CA80BE89849C3D290F83BD3E
:108A2000D26587BED111223E3CEE6C3DA33B82BE97
:108A30008D26903E3520543E85420B3D73D0C33E7B
:108A40002F1D303DF4EB9BBB497B73BDA42B603ED7
:108A5000110F7DBE6305E93D296C6C3EB5BAF0BDD2
:108A6000E89C013E6C4289BE17F6A43DD60F633EDA
:108A7000E68FEA3CBAAF023DF48100BE4BCF09BE9F
:108A8000723E3BBEDCAB5CBDE70B2DBEACD662BE1E
:108A9000653305BEA8D889BCE6F91CBE2BE16DBEC6
:108AA00007BAF8BD8BB05E3EB2092E3E3B9543BE81
:108AB000CCEA2B3E2B1BFD3D5036953E2D304D3ED6
:108AC000DBE7E33D1BEF17BE97A9083E48DE48BE33
:108AD000B7A7E8BDC3F8213E118C453E468D60BE68
:108AE000A9DBFABD06C878BE4165003E0C6B543E5A
:108AF000614DEC3D7A9DBB3DC8FD82BC37876EBEA3
:108B00005C6F50BD8D3D3A3D682E71BD596E763D0E
:108B1000928F0D3DDB9BF4BD83BB0EBD0787D53E19
:108B20007BA3293CC58FC5BEE885B83E8BF6E139ED
:108B3000F9D32F3E884A3EBD16E38EBE290AF6BD04
:108B4000CE4BE03E20453EBC1C6EEF3DCD24E6BC46
:108B5000CF3DD13EC44A23BC1732123EAA2FB73CA8
:108B600092D94DBE7F4C193FC5B4923EB3FA82BE36
:108B700056A4C03E163DA33A35A92ABE05B6163EF8
:108B8000554A8D3E10C63D3E38EB6F3E9CD30BBE22
:108B9000C8FB8D3EB1AE16BD87C9BEBC281B06BE44
:108BA0004F5D903ED2E9203D7EFB8E3D9E41A63E2C
:108BB0008664343ED40D0C3EACD00DBDC84C79BE9D
:108BC00012A9973ED789333E6FED623DF9BD4A3E0B
:108BD00041498E3E60BC46BE58D4813E0251B93DEB
:108BE000212EFABDAF75B03E01E7103EB9002CBE94
:108BF000950C3BBE025FCCBCB4854C3E2353A03EDB
:108C0000A1638B3E4B5387BD8D7C0B3DDF67783E68
:108C100060EBB93DDC11143E8B5B7E3EE1A1843EEE
:108C2000341150BD30E068BC7D8C81BE411BE73BF8
:108C3000A03A36BE7B8346BE390A37BE5F48283E1F
:108C400032CBD53DB602563EE0DF8EBEFD9FBA3D2B
:108C500089C7363D5C5865BD2E82F0BD894B353ED7
:108C60007FDE7CBD1835DC3D2B57FBBD3A2BD7BDD5
:108C7000CED8C23D62202CBDD4DC0D3D0FBD1EBD43
:108C800003DBA33D11A6B63DB649B8BC75FE9DBD3C
:108C9000A62C6B3E9F1A3F3D261667BEF402203D70
:108CA000AEBCD23B2F37C4BB63241CBD879C56BDD2
:108CB000AA44C7BD320E09BE16DAA0BE901B09BE7B
:108CC00053B6BCBD04D058BE63E3C3BDC16E90BEF5
:108CD000CC0B903C946445BECB606ABE8BDC9FBBE2
:108CE0000C426BBE66E184BEB6F8D2BE0896D6BD15
:108CF00090980A3EB2357F3C91A1D7BE0B49EBBD9F
:108D00005384053DA6F38F3A3A9236BE7298673E79
:108D1000457AA63DD687FC3D2E506BBE08CE0BBDD6
:108D2000DEF55ABC13EE8B3C1228333EECD2973D55
:108D3000A46FB03DD12739BD1D8F163E078D453E2E
:108D4000C6040FBEFD5B113C92764A3E9C40673DD7
:108D50005D75BF3D607795BDA81E423E52639BBDC9
:108D6000A731CC3D0A43A5BEEF04143EBFBFBFBC34
:108D70009B92A03D1BE552BEB4B90C3DE4C7D83C64
:108D8000A74C393D354389BED4668C3DD84F6CBB6A
:108D900062358A3E6E7F493EF2CD9ABEE07EB4BE19
:108DA000DFBF10BE25592ABED65930BE52484F3EAD
:108DB000414BB0BE821FE9BCAA6289BE1969AF3DB2
:108DC00020C293BE8D79F3BDC50001BE9E48BEBCD6
:108DD000ED6DA03C8982CFBE9A580FBE8F76693E5A
:108DE0001D0E5FBE64FB68BEECE17DBE3F818EBEA2
:108DF00007EE4F3ED3E63D3E709109BE0C58933EC0
:108E0000BC41DEBC90A0C83C5D881F3E04E7913E9B
:108E1000A5AE7EBE0B80FABE8A1C8F3ED092AE3BC2
:108E20007BB1BE3D82EFC1BD2013D13E11ABFEBE72
:108E30000DBD8B3E068789BE1663253C60CA6ABE9F
:108E4000333B193EF3632E3DFFB1A53EC05D17BE17
:108E50004A54013EB0070B3EC41BAA3EC1C867BEC0
:108E60002CC918BE3B6085BEF87FA93E22461FBEB6
:108E7000DA4DE5BE653CDA3D9B3151BD91BBD0BEBC
:108E800018D28B3D6ABCC2BEDA5416BEFF9E703E3D
:108E9000C0A9EA3E4BF8B43E6586473ED47882BE10
:108EA00033CCE8BDAACB9E3DB2102ABEB7936B3E31
:108EB000369ECCBD2471B93D8219D8BD8221FDBE3C
:108EC00019F09A3E1105113FB6ACA83B952DB83D5F
:108ED000B19371BE014098BD72E4493E6774823E11
:108EE000635F31BEE6A170BE808BA53EACD1A2BE51
:108EF000ABE19DBEB632713E0B8F803EA2E0F93CE5
:108F0000D53A1BBDCDD97A3E84DE3FBC48C6303E43
:108F1000DB942C3F2B734F3E7D0B323EEF223F3EC6
:108F2000CE15A7BD2DDED2BE8F46873E00CA8A3E33
:108F30005A233C3D1F91ECBE5B9F34BEC536FFBD3E
:108F4000F181A03D3447143FE364E4BEAB7F52BDE2
:108F5000A2AAFE3ECA94853EFD8A8BBED28DE03E1B
:108F60002A415A3E7EB621BEBBC2823DB8443D3E38
:108F7000E663B93D27A0443E6F2D83BE0524623EC3
:108F8000802E53BEE3554D3E5AA28D3DE3AEADBE9D
:108F9000F357F1BEB518CABE367755BE81B595BD3B
:108FA000F250843D124AC0BCBC686EBE1C7403BF44
:108FB00031D22E3EBE8784BD45D6CC3EA025C0BD55
:108FC000321C0ABFF22A09BF907D67BD1DB6D9BD0C
:108FD000110244BEBAE5A9BE2D7A243DFA131BBE88
:108FE00074F289BE357553BE94948A3E9D7BD43D00
:108FF000474BF4BEFED4F6BD9982A33EF962143D00
:109000008D04083EBB78FFBED8D9833DD0CE20BEAC
:10901000277438BDEED5DEBDE9398EBE3F8E48BE21
:109020007017513DBFC4ADBD4252813DA316C3BDB3
:10903000A7C0303EF7689B3EBA7E663EE199193E76
:10904000A6068DBE6832CFBD79E2C23BC150B53BAA
:10905000175119BECB6D643EB62B9CBD7C03853C7D
:10906000D844323C7B783BBE0FD53BBD30E31A3E43
:109070001F6AD1BC582384BDDDEF3A3DAC0E5F3D85
:10908000B6C8B8BDE31003BDDEBA8E3DDAB3FFFF4C
:109090000400000000080000DE9A233EC1858F3CDA
:1090A0009C0D903D9ADB8F3D757F10BD289885BD46
:1090B0002562CE3C4275463DCFF6C93C39AFEE3D08
:1090C000899DCFBCCFC89E3DEA95B83D65A838BD07
:1090D0003B7E24BD4B91EA3D3207DEBDBB65963D2C
:1090E0005BDB573D8D962CBD6F0EC83C42B2A93C50
:1090F0001A7A32BC4A8E32BE363B143E60BCB7BDD3
:10910000154E463C4BFF8A3C4D2F0FBD81072A3D33
:10911000BD10AF3C9F0020BEEF2F083DEA424D3D01
:10912000578028BDE7CC49BDB87148BDDEB03E3D93
:10913000FCCDD63C2E6C163D166636BD4FA22A3DA0
:109140002A816EBD2DC075BD953E22BD8A85FABCB3
:109150007AB8FB3C2EC077BDF3E237BED7568ABB48
:109160009D3B9A3BD65C80BD2A06FD3D03902D3D7C
:109170003AD1E33C3566413D275B603C5FFAD3BBA7
:10918000B992B33DB6C7063E949B9A3CA00706BE73
:10919000E69F43BC7C2F3C3D9DA95A3D2D78853DE3
:1091A000C8FFF03DA9663C3D27967BBD31D587BD04
:1091B000300D813BB26B5A3B833B973CCCA6473D7D
:1091C0008E1CAB3D660A07BECE19453DBCCECC3DDC
:1091D00036EFEF3CA9E9103D7A94C6BD3E388B3D91
:1091E000C914BDBCA98884BC572BA53DFAFCDC3D45
:1091F0008BA876BD00D3C43D0D880D3EAC9F013ECB
:1092000089E83D3EBCF3413EB308093DE0E02F3E16
:109210005F92303E881BF7BD4A6B02BDB0B43CBEC6
:10922000C1FAAABD50A329BD8A3131BE1857443CAA
:10923000E1F51EBED263503ECC94003EE1E1CD3D4F
:10924000D3E8423DC477963D899E8ABD2D1D2E3EB2
:109250000E6010BEC51646BE6A2BECBD0A37813DB6
:10926000BC019ABDE5FB603D6A050BBDC76164BDED
:10927000436186BD883DFBBC67E825BCF55AACBDA3
:1092800037C215BD45E6613D7406653D8ED009BD0A
:10929000E6576E3DE7BCBABB040E333DBA76F9BC67
:1092A000ADB8B23B272FD4BCD78D453C0B9CBDBB82
:1092B00002B5573C223E68BC8733F73C967AC9BC5E
:1092C000C3293F3D06F9003CE9C01E3DA1F60F3C15
:1092D0009803DDBCD292BEBC9E5AAEBDEF1E023CCE
:1092E000A95DA63C5D35C5BC1955A9BC0510E93C76
:1092F00064A0433D3D25D7BC56B1793D76C7D6BD68
:1093000038CEB5BDD746CF3C1134A2BD1E37B53CD3
:10931000DC860D3CBB28303D06FE4E3D1325A6BD28
:1093200009BD8FBC0058323D594D1B3CC4A911BE2C
:10933000392BAD3C3C7D17BC7964713D359D093DB1
:10934000A6DF8E3DF0A4B7BDBA1B893C3B7870BE4A
:109350009690C6BDC343C93C1FA68B3D8EB4913DBC
:109360002898893D5CE794BD0A4BB6BD6F01BD3DB1
:109370008E68EDBCBF1081BC6D808BBBA6D6D8BCFF
:10938000D59DF73DD0F1B23B90993B3C8D1F5F3DA1
:10939000C137543DECEE0CBE1A29CCBD211359BE89
:1093A000820110BEE4DB14BE9198543D67B7A13C26
:1093B000425B0C3EB60FA1BD86D2F43DA2F229BDA0
:1093C000CC19CA3D0B1D0BBEE13806BCDE3E11BDFB
:1093D000C321E23DCC99E6BD0D091B3D327AA03D8B
:1093E000C763D5BD865F7FBDEC7DC1BCC880D2BCE4
:1093F0009E44A5BD0080D53C81A11B3CBD6EAF3B0A
:1094000029078B3DAEF0CBBD021FBC3AD1BF54BD86
:1094100073C71B3D119E0DBE1E1134BDD6470BBC3C
:10942000B68ADEBDFF5AC73C98E4923CDB0BD03CC9
:10943000C9569A3C43709BBD0097D93B6F8D9DBC2C
:109440006E92C0BDDB98E6BBCC26AFBD24A5AF3C79
:109450005E6BB0BD25D32DBD7F75F1BCD663FABC64
:10946000146513BD71255D3D90EA3D3D05F5CC3C8D
:10947000DC56043D549EB5BD6ED721BDC77B4ABDA9
:10948000B96478BD4BF6E63C352D083DCFEA65BDA5
:10949000A177223DB7EC783D3CE6A13D2A91ECBC9A
:1094A000BE860ABE976FD9BD6B054DBE387732BDFB
:1094B000EDC780BEE34988BD452D89BEC89FCE3D1E
:1094C0001816763E978D313EAD5AA5BDB9398B3C05
:1094D000759C58BD29445F3E96D617BE8DF3C33D9B
:1094E000AB814D3DF49D9FBD282E81BD69D3A63D26
:1094F000BDE99B3CB55F20BD5A67A0BDCFCBC3BDC6
:10950000E12679BDF992943D0D4C1CBE4EB785BD48
:10951000466B80BD0DDA9B3C610C2F3C5E6761BCE5
:10952000D0AC01BE13C9E9BB496C94BD9995BEBDD1
:10953000CACECBBD2E576BBE0ADBB3BC5834CEBDF2
:1095400072C88ABDA939C93BFE00463D9999D13DF3
:10955000028E0BBAD60D113C4A59F33DEC200C3E5D
:10956000740743BE59A2F63D9B27883D8AE7B9BDE3
:109570005DE5ED3CE485603B02A91DBE8B56BE3D1A
:10958000107A503E98BBE3BDE103953C81A05C3D61
:109590003F1486BC6B30E2BCBD2EB7BC10A1163D9B
:1095A000DDF2923C1EBF4E39848A203DCA2BF7BDA6
:1095B000C42AF9BD0A095E3DA8803EBD4A4580BB6C
:1095C0001203133E7F5A0CBDD7A41A3DF628BB3BAD
:1095D0004C1C02BE62FD2DBE35F4CF3D1310DD3CA8
:1095E00078204F3D33CE823D4F7BB53D7909893D93
:1095F000E2B0CDBC87DB703D524F1C3E555BC23D97
:10960000C4D6393E30798E3C2385D83D236070BC6A
:10961000F9EB663CEB70EDBCE372863C66986ABD84
:10962000D0DA123C9ADE17BDE2D85ABBD5AFD03A99
:10963000516F66BCCF628FBCD3A87C3DAA33523D2C
:109640006077743D86BBFBBDF70700BCB7B26DBC4D
:10965000F1C8B73DC16CF1BCC1DA40BE93A64ABDAA
:109660004A45023EB3E2B53CDF8C1DBE7CFCCB3DDF
:10967000FF20213C5D7569BDBEC7313D94EFB33D10
:10968000D0C2CFBCE9946B3DE3F9A73D8B6EE33BC1
:109690004B763BBEC53EF8BCDDDF2DBEEEF994BD7A
:1096A000AA6108BE7D30F13D624E363E65E5BB3DA8
:1096B000210CC6BD241E313EE98AA3BE9973B6BDF6
:1096C00030B418BDC2FC973D3E907F3DDF3AFC3D73
:1096D000552E78BE0FFF023D498C06BD680D2FBD8B
:1096E000F8AFAA3DF14918BDA82B483D5DB621BD94
:1096F0006DACBE3DDD891FBEC7C31D3D28131B3C9D
:109700009BC10ABE8B37B63DCA822B3D5F44993C54
:109710008A481B3D3F5F873DBD6FDC3CA9F605BE17
:10972000A2EC003E1567E4BDEA74B6BDAB7F75BC24
:1097300039E464BE4321863D3FC732BE00A2F93DF5
:1097400054C91D3EA6A7F03D58CE3CBE4D6A9FBDF4
:10975000CC8B963DC6C646BE5D050D3DD0AD343CB6
:1097600072274BBEE4F3E33DABFBEBBD38EE43BDEC
:10977000625A48BEDB27323E52E628BE2C6480BCCB
:109780008491533EFE13B0BCC079843D85E1423BD9
:1097900070FD883DD98DD23D877AC23D9CA28DBD9A
:1097A00094B635BD8B1021BE559AC3BC27F1033E3C
:1097B0000A88CCBD36F9E93D4BCB5E3D18749ABCA6
:1097C0001D4F633C50FE1CBE8A12A5BD0021033E06
:1097D0009849CCBD8C5DAE3C61532F3E8DBD493D5B
:1097E00074ADCA3D34B786BE1DB8CCBD71F2EABDBA
:1097F000600A1B3E6EC7293CBE22823DCE700DBE64
:10980000FB211DBC82CCF63D3442CF3D2E0B143ED5
:10981000B8A3E23DCB7F13BDF350F73ACF9D93BD84
:10982000024CB7BD9E3429BC2FB8B13D03E9E6BD5B
:109830005FD26B3DE514883DDEF6903C6B25E9BDBB
:109840007698923DE016E43CC25AF33CAFE4333CD8
:109850009B6DA2BCAA4F0A3DD3926BBD913F2ABE1D
:10986000DD7F7DBCDF63803DD2CD61BEB01C22BCFC
:10987000AF459ABE915B0FBE401AE1BDA92AFC3CE0
:1098800090F1B13DCAABB03D9A0E823CAE2919BDF4
:109890005C0E8EBE00FCD4BEE6BBFFFF04000000E1
:1098A00000200000C6DDAA3A037BE3BB0B578FBB49
:1098B0009EBD99BB3D14183911FD44BA639FCEBBC0
:1098C0001A6D90BB497608BA972C0B3B4F7DC33974
:1098D0009B0C11BBAEA664B8F4F92F3BBED6133C6B
:1098E00029723D3B4974A5BBE5B323BBE6CFA1BBC1
:1098F000E170DFBBB903A73B5A4D203BE0B78E3B7D
:109900006769D93B1716B63A7F4F6A3B4C8EB73A18
:10991000D13095397E3709BAB24389390363E23AC7
:10992000781076BAAD3B87BBF8263F3C34500ABB73
:109930007169D5BAD3066139E02C953AE1822CBA27
:10994000E724FDB9293EDE3AA9C4353B38EC91BA8B
:109950009E421FBB136E7F3BEA1410BB4C5C9EBB48
:109960004538A2BBBC3351BB5AFF5F3C5BB5593B8A
:10997000784C99390BB52EBB80AD44BB22752ABB00
:10998000D91F24BBE6C5BF3B7FCC9CBA35EA583A09
:10999000E4BAC9BB5DFE44BB8C29F8BB9A0BC33A41
:1099A0002508803A5B721E3939E0743A991210BC6E
:1099B00019B6283B3812C8BB04DA11B76CB68BBB9A
:1099C0001A79B33B5EE5BFBA911895B9F45CA53A34
:1099D000DA1CB83AE5A2723BE7742ABB30FD123AB2
:1099E000CECFF439600F10BB27ED4DBB541BD839D7
:1099F0003D7C32BCFA431A3B5F7937BBE5D31ABBD7
:109A0000C9F6203B2B7ACE3AF1C568BB55B4D4BA1F
:109A100054AA8A38CBF0FE39F260EF3A641FC83B93
:109A2000514B3CBAFB268DBBF37804BC6EE7F5BA0C
:109A30003296C03A3014853B048B1E3BD8575F3AB0
:109A4000F7EE213BFF429CBBD97C8B3A595A033B32
:109A5000425100BBFA41DEBAEB68FA3A5B7FBDBA0D
:109A6000BA9A56BB52DCB33BAD5E0FBCA9404BB8B3
:109A7000051DC93B4FAEBE3B590503BB84DAB2BAE4
:109A80003E8236BB15CDB9BA14BF75B92648F33B33
:109A90005F35DABABD81963BD66CD83BF2E00A3B23
:109AA000F525B73A38DD573895270E3B3915C9BB30
:109AB00035CD373B1F74B13AE832DC3A7009713B5F
:109AC00064FEADBA2DCBF2B99777EBB9B6E0D3B956
:109AD00059B4863AAE54303A54D5ED3A38FF893B02
:109AE000E4BAAB39DF158A3B37EC1F3AA95E1B3B62
:109AF0003B806BBA27E12EBA4AC8C7B90902D13AEE
:109B00009216903A9C4CF6BA94FCD139BA366DB99B
:109B10004A9F53B9D9C26CBA258A4BBA052901BBF1
:109B20005EC248BAD0241A3A36D45D3B00FBFDBA77
:109B300076F03EBB0A2F073BF266DE3A502AF4BAB3
:109B4000B13CEE393699D4BADE08A1B8F5064BBA65
:109B50007A58883A39F9A23A83855D39A90CD53A01
:109B600003B4C7BA6F8E1A3941381C3C94F3BE3A1D
:109B700022CE213AB111973B97E1ECBA51769ABACD
:109B8000B7DD0DBBB8E587BA433A8DBA0872C03A63
:109B9000CB95BFBA6263EF3A1F2935BBB81740BAFD
:109BA000FEE5163880996CBA5AFEAB3A7D447FBB0D
:109BB000D2D97C3946E26C3B26E4A53AC19FE7BA8C
:109BC000E4A06C3B41899DBA4B200C3A7C6364BA9B
:109BD0007261BE3A2385503BBF841CBAE7A2F7BA34
:109BE000983D8AB9D673493B88514BBB914CD93AC1
:109BF000666302BCC030B1BA11A4AB3A7B61E139F3
:109C000013B394BA263D4F3A72BF30BA4F9F133AFE
:109C100035F050BA6E61BEBA18E9A5392B800C3BFD
:109C2000AFCA6C3ABDA2AC39F9A747BB339319BB95
:109C300000BB27BBDADD60BAC612C839826CE8B94E
:109C40005646A8BA35010ABB41F66DBA15A502BB46
:109C5000F67418BB5821F93AA717F0B9AAFF673A6A
:109C600077A4E4BAB8F9A2BBD268AC3B822A8FB918
:109C7000F7B11038D43039BABFB2ADBADC65FE3AAC
:109C80001A1AC3B9EA0050BA6F3202BABC46423B54
:109C9000D2197BBB68FA133A06AD80B9919FD739C8
:109CA00081085538247E8BB9E487F23A8B6BC53B2B
:109CB000AB14AB3AEBE6BA3AA38674B93AC2B439FC
:109CC0000955DE39E928073A0D9DCF39D721A13A48
:109CD0000CBF03BBCE1F84BAD64885BAE518A0BB1B
:109CE000F00D5BBA98F6AFBB9C5CC63A7CD33FBA2A
:109CF000A5E303B98096F73AA5F73ABACF97CCBA5D
:109D0000A39E8F3AF17CF53AA6C280BAF89E4DB96F
:109D1000C45B1E3AAFF181BAE87FB63A943C65BAAB
:109D2000D592FB3A076306BAABD76039EEF7A9BA0A
:109D300042E2F53A93FB2ABA81992B3B947811B908
:109D4000016AE23A132C00B91C471139F485A8388E
:109D50005BDF603A42CEDCBA9E63A3BA1DCF7F3987
:109D6000257C0B3A050E793B1DF35BBB61928EBAE5
:109D70000F22DC3A2FDB75BBB2A7943B8CA51ABB34
:109D80001C34493BE88609BB272110BB439D5EBBC1
:109D9000D337443B4F832EBBEE67993B9420B73AB1
:109DA000DA4BB7B9AB75103B9274163BD81B443BEA
:109DB000AAE547BB3552B73A15F40E3A670BB73AE6
:109DC000EE5E613BA341CDB94A325BB92C1FC73A65
:109DD0005C69A2B9E3C685BBD83DC6BA80652FBC15
:109DE000B08FD23A62A5B5BB3C94143BEB5299BA02
:109DF0008C29E8BA08715A3AD20781BB3DA5AA3925
:109E0000C73A24BBA23E773A793A02BBBE68FA3918
:109E1000696B6E3A5DE1083B18ADE8BAD8B4CAB9CF
:109E2000F37227BA5377FA3934D6B73B6B95883A31
:109E30004C2CF1BB5F0D1BBB1725093BB5F9123A42
:109E4000CACEB5B82A72EC3943FEAF3878FFF2BA01
:109E5000961E903A90515839CC312B3AFD40FBBABE
:109E6000AB04A0BBD345513B4B77763B2ED6CEBA45
:109E70007FAB973A78E4943999068D3A38E6963A6A
:109E800075FD7DBA9676813A027030B84FC28BBAB2
:109E9000E030A5B933845DBB0C6189BBA20C47BA25
:109EA0004EE43D3AD05EC0BA30C57CBACAD1653BFB
:109EB00074906CBA84001D3B41F780B9B9E192BB44
:109EC0003FD84EBAD2906039C1213CBB1FD189BA6C
:109ED0007D192A3920FD20BB02E578BA8C2C65BBA0
:109EE000460BCE3853F091BB1F63EF3AE1CBBDB9BF
:109EF000F58A433A1B961B3B814E30BA71BA503AF1
:109F000021AD763B4847AC3ABC4B3EBAD129B43A76
:109F10001B84C639435DB7BAFE916DBACE3591BB8D
:109F2000B231A4BAFD9B013AB5E3753BFC13D038BE
:109F300025771F3BC90339BB7EA2493A881702BB6C
:109F400096CD023A37D5A33A83560EBAFF2184BA8A
:109F5000A939123BA7D2C3BABE5F7F3A0138043B8E
:109F6000AECFDC3BF4DE043B2EE1EDBAFC9C093ABB
:109F70005E37D2BAE5326ABB4A60293BEE85483A81
:109F800001F1D2BAAFC5F73A79498EBACD7F40BB5D
:109F90006ACAE6B941B50EBB2297ED37F12640BA41
:109FA0003E8E603929D594B94749BDBA719181BBBC
:109FB000D538ACBA86ACA33BF4C911B958626A3B38
:109FC00023E4FCB91E1747BA252C9B3AC25FFB3924
:109FD00079359DBAA554B1BA278A13BBD9EA18BC02
:109FE000FB3A3A3B44F60C3BC76B01BA801221BBEB
:109FF00041E8E33B3C44B7BA62C1A83AFF8191BA59
:10A00000B81EFDBA7E599EBAA120E4B9822C52BB7B
:10A01000A9E31BBA8C5023BA6B8C0C3B4E1E4EBB73
:10A020006D982A3AA92861BB65BAA13B6A00B9BA02
:10A03000FE51B73BCCF13FBB2A9DD4BAC6FB3C3A9C
:10A04000E3C99A3A27A7AE3AB23BF6395FDA13BBB7
:10A05000E9CF713AEF93413B86E3543A8439F33ABE
:10A060009EEB783B984984BA2318C4BBE87EF2BAC9
:10A07000BB5C9E39ABCD4EBB7D9D32BBF6CEDC3991
:10A080005ADAF3BA36D92E3B2EBF013B947088BB07
:10A090003B811B3A0708C33A97739EBB2C05C73A0E
:10A0A0001FECB2B8BDA40DBB863B223A69BE53BBC0
:10A0B000A145223B6FCF5639E899D93A3005883B04
:10A0C0009181043AF5A51CBACD17323BC20F19BADB
:10A0D000533E173B4329A1B7BFFD38BAC49E09BC04
:10A0E0009FD18C3ABCE55CBBA256C7BAC5D71E3B14
:10A0F000B587A7381A59C2BA08B9023B218495B965
:10A10000860790BA20DF07BB519FCD372795D8BA75
:10A11000282F63B92992FAB93367053A87944FBA61
:10A12000DECF873AF7DA45BB94F4DE39C51553BB69
:10A130006D67A13B446109BBB21C36390504BE3AC8
:10A14000C7E43EBA66A626BBB251F3BA1BC309BB2D
:10A1500074EBA43ACF3F0C3B331C82BA9D4715BB2E
:10A16000E64268BB2ECCC5BB4CD9B33AE01A2CBB37
:10A17000933990391A6189BA95203EBB739C4F3B45
:10A1800005E239BAC24F153ADC25253A12ABDEBAE0
:10A19000E06DDBB9CE9F4FBB9B4DA43BB6C5283AC3
:10A1A00071959BBA2C0C7ABA9550603BCECD04BC0D
:10A1B000CB79EDB8A66010BB7A5CDC38D64383BAA5
:10A1C000FD5838BB1C661C3A5B0F9C3A43661EB9AF
:10A1D000FD49233B835A433B82C426BB8E0436B9D8
:10A1E000D8C4F93A3431C13B5A3F2A3BA258393BD3
:10A1F000A76A58BCED9A853A9B0B16BA3E73AC3AE7
:10A20000AE9309BBE6A750B90E6010B9B868BF3964
:10A21000C9E591B9F519D1BA38FFF43AC07A823B51
:10A2200079186FBAF84A0F3A34868439B73A22BBA4
:10A230005AA7333BB5864DBAA449B9BA2C3DF03A7A
:10A240003EED29B8E95AD1BA996000BBD4F3DEBA21
:10A25000C6C903B8EA5620BB75C0ABB9C47CB3BA53
:10A260001EC01DBB5EDA753AD4679F39075EB0B970
:10A270009E64883A45BCFA3BF220E6BA8B85F8B773
:10A2800085B72239730B643BEA6A383B27AF44BB7E
:10A29000234B8DBB4B731FBA2A8D153AEF8A3BB8FF
:10A2A00049A9A638D1BF2EBA9F30F0BAF25919BBCE
:10A2B000881835BA53D2353B5756013AC169C2BAEC
:10A2C000BF7C13BBEACD44BA22EBFBBA416E80B926
:10A2D0001706B6B8F92659BA6091463B7D8D11BB79
:10A2E000DF75ABBA1C43753BBE76CE3A26B5AF3AA6
:10A2F000C86795391EC3093A0F98AE3A447F3E3B72
:10A3000070870BBAFAF2FEBAAA88853A6047A1397B
:10A31000C96BD239D174C4B948538B3B598232BB13
:10A32000CD4CEDBA1A6349BB4F456ABB0449353B76
:10A330003FF44BBA2E9DC5BAE9F206BB396649BB5C
:10A34000117ABFBA8F3C6B39E41E1B39AF80D8B984
:10A35000A44A44BB3EEF58BA59152FBAB644B0B917
:10A3600074A3ACBB56B075BBAFB7B3BBC98C15BB40
:10A37000C05C273BBB5A363BDF1A8BBA51AEB538AF
:10A38000692F0F3AF9E7033A64CDDFB9A91296B8FD
:10A39000E551D8BA0DA829BA4E046339F57B5BBAEA
:10A3A000D2FF09BB86C6C73A5F0A02BB34452A3BC7
:10A3B000AEEA513A19DFB139AB11103BC3D9B13B09
:10A3C0007F82A03B04DBAC3A2B913A3B9D20B9BA8B
:10A3D00069257639F53228BB44992FBAF958EBBB79
:10A3E000836452BADF6475383B059CB9DA021939C7
:10A3F0007B232BBC9E86433A423C303B2732D43AE7
:10A40000DCD9C8B9F72BDBBAFD54A1B931B01B3B7D
:10A410008814CBBA60C60EBBFE397A3A958F873B5B
:10A420009EF164BA6CA1E939F5CF603B5D7BA93A36
:10A43000C90E9FBB2F7E893BF79C9EBA28239C396F
:10A44000FD6236BA9B8B163BEA9E4CBAA054C3BA47
:10A45000A9F428BB6C68293A7DD944BA84F908BBB1
:10A46000744DD0BBF4996FBBC977153CB4B96F3A42
:10A470002C63B23B033BB13B99DD8CBB5BFEDE3A08
:10A4800054B833BB16D2BCBA9D6880B99ED31A3B70
:10A49000483D433BE18E35BB58960EB94903AA3A75
:10A4A000AD8FBAB8A3B319B9BF50103BD0BE38387E
:10A4B000385470BA2E986DBB521F1DBB0FE5C7BB39
:10A4C000AE31CC3A402AF7BA0BF8803B40FA9E3ABC
:10A4D0003ED1EB3A57E54EBB1D60083B0CEB00BC90
:10A4E0008090003A6C2925B906501D3908C04D3BB3
:10A4F000E9AA6F3C4A47143B4079C33A414E8BBBB3
:10A50000AEFD193B762F6C3AA45A533A648BF93A54
:10A5100099A0BFB981AA3139A8AC0DBA08732ABB7A
:10A5200092B9ABBA8823333B426DB1BA0A561D3992
:10A530004892E1B8AA20D73A43FA97B967C82B3AAC
:10A54000BC5EDABAFEBF9D3AB1D650BBB796923A1E
:10A55000E4D8373BA1202CBBAE5D203938DF30BBBF
:10A5600096EBCB3B7B170BBBF9808C3B478D69BAD5
:10A570000311343B281F0B3B8905823B98351D395D
:10A580000604463BF366113BD2B4D63A9F882CBCF6
:10A590003547C53B9AA5BE3A6C922ABB19318FBA92
:10A5A00065FEE33A36655A3BE773D93A7AC54B39CB
:10A5B000610B8ABA2EA0483BB91F2E3BD5B04F3B4A
:10A5C0004C3B81BBA6A45CBBB69E203AE34DA23AAD
:10A5D000F2112B3B454359BBEBDC55BB5A8908BBF9
:10A5E000318829BBCF2C27BBB642AB3A1DD8E03A05
:10A5F000FA07D03B9123313BFED905BBC8CB943B36
:10A60000DC8A9ABB45AFC2BA30822C3B46B73FBB0F
:10A6100039917C3A6F1008BB43E044BB1E2292BBC9
:10A6200043BE3FBB8AC1E73A597AE3BB0E44A8BA9E
:10A6300007B513BC8C605BBB5051C2BA7ABA3FBB42
:10A6400094AD6E39717D993B6858203B702AC4BA2D
:10A65000CAF15FBA356DBE3AC88A59BBE6A29CBA48
:10A66000EFE50EBC26BF523BA110C9399366C93A2B
:10A67000C128C4BAD740DB3A9CACBB3B182792BB7D
:10A680006965DB3A398C103B70BDF33ABAD8C739EB
:10A69000F46EF63AE451AB3B074DBDBB8C2C2CBBA2
:10A6A0004949EB3AE0C33138BF3322BADA9DF7B9F2
:10A6B000431363BA421D9C3A16AD7FB950DA943AFF
:10A6C000E996203B71F05A394170263AC9FDBABA71
:10A6D000ACA7B2BA1038873A6C2106B9A9A590BBCD
:10A6E000F64B93BA6708D43A4287D0B9A08E05BB1F
:10A6F000E09B97BB81F5F73A11EC123B7CDA243BE7
:10A70000F25E4DBBF412ECBA0706813ABD4FA03899
:10A710000321B1B93109BFBAAB840B3BB8BCB2B9A4
:10A720005A9167BA7A4898BAC23E583B986F1CBA99
:10A73000D04C30BAC5F5AFB9AE70EBBA9D8D91BAB9
:10A74000B697CE3A27E4B4BAFCBEE4BAC791B53A9C
:10A75000D9B1CBBA8D2C153BCDEA4D3A05AC43BBF4
:10A760006B85953BAE6AACBA64E63D3B714CDC3A16
:10A7700079CD0EBB44493E3A940A1DBBA5F906BAF1
:10A78000BC20783A6A8D4A39FB75BE3A962034BBB4
:10A790008E145DBB37FE9F3A3796333BC2EB8D3A42
:10A7A0009738C2B9CA224ABA69287F3A2A7DC2B903
:10A7B000C530143B9C2D4A3A92C73A3BB176833B55
:10A7C00048E5683AFE5979BA88AE623A2ED3E1B9C3
:10A7D0005C46B939A026063B50624FB91E58873BEC
:10A7E000C292D63A1822203A1052D7BA8B478ABA68
:10A7F00032BDA0BBA6B6C53AC5EEAF3837BC943A59
:10A8000050D3EF3A2F5C90BA36BE323AD02B3C3A56
:10A810008F91B5B9770994B991D195BA9DD21D3A66
:10A82000CE597E394E35C8BA96D247BAE56C85BA4C
:10A830001358D5BA4A54C13A79F967BA869490BA8E
:10A84000F9169237A9E1093A856FAF3910FBA1B922
:10A85000615E2F3AB26243B9AD3EBFBA038928BBED
:10A860006BD271BB9C114EBB2FE265399FA0123A8F
:10A87000C73AC23A554F113B1253BABA48A493395A
:10A88000C22EC3BA058EA4381D1FC53A0020B2BA25
:10A89000548B69BB8140983ADEB7DDB88866D9BA77
:10A8A00050EFC4BA13DCAA392102233AC56299BB1E
:10A8B0003F04AB397AFE57BA909F6E3B4C3BE3BAEC
:10A8C0006BB6C33AF4A68A39E55762B90FE777BA8F
:10A8D00018B5863B163497BB1BB3A33B896E993CD6
:10A8E0002FD533BBF4F6B83A57F595B9AA24B93B3E
:10A8F000027AC1BB56214DBA2DD0C23A9EE94C3BDB
:10A90000BA58BE39BCC52ABB04F3BE39470D8FB94E
:10A9100068A605BB30BC06BB0459853ABC330BBBEB
:10A9200097EE0C3B378D4ABA3169E43AFD353B3A34
:10A930008635623BE5365E3B3D9CE4BA1BFDC9BAF9
:10A9400067D34CB811A12BBACDB59BBB552B56BACA
:10A950002C0114BB38196CB9515F82BA2706323BFF
:10A960007C7975BBCCE196BBF484823C2F00803AA5
:10A97000B31F863B7A49FE3B6B3DC7BB32BDD9BA9C
:10A98000181F383B5C489738AE11073B6F67663B32
:10A990006D128239ED9C80BB9B94C93B873AA8B964
:10A9A0006D9B1BBBD807043A3155363BB5C4733B8E
:10A9B000731003BB58614F3B076317BB4B60A5BBCC
:10A9C000CE5D2D3B4638213B519D9CB9B602AABABB
:10A9D00036B7A1BA547A4B3BB1F05B3A6FB3D1BBF7
:10A9E000C7C3FE3A900783BB3167E7BA2E947DBB9D
:10A9F000D69333BCBACF183B69271DBBC9E162BAF5
:10AA000035DCA23BA832A2BAE0D78738797CA238DD
:10AA100073D2893AEAA996B9FF8497BB6C382F376D
:10AA20004CBCBE39D74A263B82CE95BAABE0E73A5A
:10AA30005B8BA03A10CDCEBA255B00BB9542A93AFC
:10AA40003A5A04BBD75AF0BA838A0D3A13D76439FD
:10AA5000F036BCB9EA993EBB92EFC93A4CAE693BBD
:10AA600083DD733A9C262D3957F7133CA7F61EBA9F
:10AA70004F78893BED406D3AD4947D3B31FF07BA66
:10AA8000FF4519BB71CC25BB5E90433A374D813AE7
:10AA9000778C50BB8EDF84BB3346963B169293BABD
:10AAA000C87FD4BAF88ECF3949F447BB54CC8ABB9F
:10AAB0000C944138BF0B5D3AEDF1FB3AF73B1E3A7F
:10AAC0001677003B6055E3BA0EE5343B921A89BA1B
:10AAD000D96E6EBA5F99413B5CCC8A3967122F3BC5
:10AAE000AD4032BB82D708BACE4288BB5254913BAC
:10AAF0003C8AD1BB7810A0BA026AACBAD4FB563BF0
:10AB000049FEB4BA7A9CA9BAF7E1B53A4DEED2BA89
:10AB10004331573A8C92E23A44474A3BE1814A3802
:10AB20006632123B0E9B8EBBBECC27BB6FDBF5BAE9
:10AB3000646B72BB6161833B38A6FEBA1A26FDBA0C
:10AB4000DDCF33396FEA67B7852118BBC8E30E3B09
:10AB50001083CDB9BE30A03A2B1C1BBAC93924BA18
:10AB6000A866993B8D00D1BA6B27963943E021BA8C
:10AB7000F4710A3BCA0CBA3A78499ABA3D8715393A
:10AB800093BB38BB64760C3B442028B92C4387BA6E
:10AB9000A289F0BAE0CB32BB6C9F6EBB3249FB3A64
:10ABA0008B93953A6A6D04BA9E591CBADF26E0BBB6
:10ABB0001D41983B2AEFD13ABBFF233BFFA70FBAB9
:10ABC0000E0547B9E2B3A3BA18E61EBB61590ABA2B
:10ABD0006FF8B33A16EBC8BA266A333BC106083C95
:10ABE000772FAFBA1DC0013C72AC39BAD47E283B76
:10ABF00024140BB823FF1E3A31D1843A4B3F973BC4
:10AC0000D61DB2BAC547E83AC7C677BAB87AED3AA0
:10AC1000256960BA325894BACA7067BBE29EAE3BEF
:10AC20003E9B05BAECE1B6BAD5E9FBBB893AAE3A30
:10AC30000EAFB539CECC11B9839E1D3B7ACB36BB56
:10AC400007279F3A04418E3A3872CEBA723F90B8C5
:10AC5000A6EE56B99F4B08BA4DEC7F3AF4396B3BE0
:10AC6000F7FE7A3BE1FD59BB96B1AA3A5ECAB2BA89
:10AC700070E29ABB7E79BA3A4BA07EBBDB0459BA2C
:10AC8000ECAC38BB6C264CBAA6177F3A5630AE3BBC
:10AC9000282987BBFD3AF6BA63B892BA9C383A3A8B
:10ACA000A6861CBBD2FB10BA44078CBA319A9EBB55
:10ACB00093F30E3B70FC9FBA21DF053BA43700BB2A
:10ACC000BFC1BA3BD912893A2C7007BBDE53B2BA66
:10ACD0007EAC2C3BCF43673A82D4FE3AED2ED13B7B
:10ACE0008FA698BA2B98E53A8043AEBBDE35E1BA21
:10ACF000A9B085BC24365939F711E1BA99E4A6BA4E
:10AD00007EB726BBCC0CB13A15B315BBBE1E823A3A
:10AD10006C1E42BA1DD9C4BAC98C46BBB495B43BAB
:10AD2000C518123AC6F91FBB4D9DD2BAD55D88BB76
:10AD30000A5286BBD1A17C3ADE249B3AA796953A6B
:10AD40004659EF3A5BAB42BBE8A2C239D437F43A7A
:10AD500071C5E6BABB0D8DBB613CD5BA6BFAC93A79
:10AD6000F60BBBBBAA37CDBAF583803BA24A7DBBAD
:10AD7000F8E6A63A9A6604BB11AFECBAC3550B3B92
:10AD8000B7EB89BB61A4BDB8D741DB39B28BA23B1D
:10AD90009B9402BB42AB733B1B4FE8BB391F3DB9D1
:10ADA0009F16203AA1E7A23B61658C3AE28F7A3B7D
:10ADB000E7F54D3AE1725E3B6F564ABBE80237BC9D
:10ADC000241EA8B97E8687BA69AB66BA5C1410BB2C
:10ADD000EFFA96BAD2ED993B8300DF3A21D0863C58
:10ADE000F9A5C83ADD56FC3B128EE5BA3DF5A5BB88
:10ADF000202B94BC3CF752B88E872F3B3108A9B961
:10AE0000B473DB3B08DE33399261993BD113A83B25
:10AE10004C35C1BA9C4246BAD55C5C3B0D5C4C3BA0
:10AE200071FDBC395258E93B2D8873BB8F8C08BA31
:10AE3000F0909E3BCE2605BBA6ACB5BB87A0F0BA72
:10AE4000E9455B3A8AC79B3BC459C43AE16A643B13
:10AE500045B732BB4CA9073A3B42F03ADF7828BAF3
:10AE60007C4981BCF26E843BAB4C44BBE9080DBB12
:10AE700061A6CF3A9C82C7BBD4BAA7BBD0A728BBD8
:10AE8000403E853BF72E06B9EBE5F03A177BC9BB90
:10AE90008858403BCA057E3A29941ABCCF79073BB3
:10AEA00080EC73BA86A182BA1482D5B9047ADD3AED
:10AEB000F1FB83BA39EBAB39189D12BB1B06043B7F
:10AEC0005351963A9835413A3EA2B63A923E8A3A62
:10AED000B6B015B9E52323BB7F52A5BAD690C2BA46
:10AEE000D785073A4D071BB9C2D15D3ACD3BADBA04
:10AEF000ABAE9F3B495087BA4E60803A271D41BB9D
:10AF0000C1D3483B6BF2D53AC42550B9261E853AC9
:10AF10006642F3B90E2050B82FD4643A6F934EBBFB
:10AF2000D7F2273AFB65E83A535F1A3BA14289B949
:10AF30007FBA30BBC12CCCBA33EF103A5CE9B43ADB
:10AF40003EF3D9B8ABF5C9B96AF5A5BAF2AB97BA71
:10AF500090FB0E3A16B586BA788B7BBAE092313BFD
:10AF600077AC2ABB205933BBE313BF3A9759D3BA06
:10AF70001D3F49BBF999CFBA35974E3BE168CCBA32
:10AF8000B846FF3A0A19A33AF8FCEFBA28984CBB26
:10AF9000398A683B8C54813AFCAA143BE8E113BA25
:10AFA000A338343A2C4D94BABC650CBB7A179ABBC3
:10AFB000F02D05BA301D453AE1C58F39826179BB64
:10AFC000FE38D83A2E118EBACA6AA23A1011B0BA17
:10AFD00011C8E63A516259B88A0AC2B97064663B30
:10AFE000C05AAF3A4298DFBA87BE29BBE3221DBBE5
:10AFF0001EEA7ABB2935D73A334FE5BA07B88A3803
:10B00000E18F85BA6AB8273ABFBBA238FC5ED4B8D4
:10B0100098AB873A24A118BBFE2EEE3AAFE1EDBA09
:10B02000803D36BA31CD78BB2865673B758047BB1C
:10B0300052178F3AD47232B9ED4F5DBB466559BB9A
:10B04000A09DE8399C91683A0019FBBABA892ABADE
:10B050006CF815BB1355643A344E2C3A9213443BAA
:10B06000681EBD3BAD8548BB399EEB3BC668443B83
:10B070002B11553B28D60A3B7BB548B70DE5023B63
:10B080000F661E3B83D205BAD060963A68E3C1B919
:10B09000CFA767BBE20402BB9045F2BA42D1C33AE4
:10B0A000B78FF6BA85EEA1BA9095763BFE63AFBB3B
:10B0B00067B45DBA2180ADBA9818E03A48BE97B936
:10B0C00097FF623A8B5FECB9670F3C3BB0E47EBA06
:10B0D0005DDDE43A52E8E0BA0CB8F7BAC4551F3C5B
:10B0E0002D9852BA4A3AA83ACA47CFB99CE2003BD7
:10B0F0009E57EC3A324CA53A0DD3F539362E40BB6B
:10B10000BB2FA03A549F683A4B7732BB7ED3E23ACA
:10B1100043E04A388B2984BAEF5A3EB98BD64E3B6E
:10B120009324ECBA9F5085BB6DA964BB040C49BB4A
:10B13000A3A9D5BBD8550A3A93E701BAC7B91C3AB7
:10B14000A13152BAA3DA0EBBBB9B37BB218FCBBA5E
:10B150006190BB3A2BCC4A3A1048B639A61A093A44
:10B160001881CB3B80B30C3B9632C43B26E24FB9EF
:10B170001958A0BBD66612B99DEB5F3A2F33ABBA14
:10B180002D8F3EBB51032CBAC0AC223BDC6DCABB39
:10B190002990573B7FD9613B2C38DAB8B8BD29BA22
:10B1A000C1465E3A0908773A2BCADDBAC20030BB05
:10B1B000773FF73974FD9939E704153B6701A5B965
:10B1C00027CFB43A29ECB8B985E57F3A8AEBF4BACF
:10B1D000602B16BAFA90E2BA7EFEFBBA2B70C03B27
:10B1E000EAB43ABA0FB9953B6F286BBBFF2F5E3AB2
:10B1F0000CC34CBBF75BAFBAE79449B9E32FDF3A16
:10B200005C9CEFB9B723D9B916E02DB95F808B3AB2
:10B210003CA73F3A9F5988BAE303A03A0F248DBA5E
:10B22000981EC9BA186B95BB089E33BA558164390C
:10B2300067BD173A1E35323BFE3E3EBB5657FA39C4
:10B240008855EA3AA51D0B3A10128F3928675C3AE7
:10B2500043AF0EBBA98F063BA033733AC8C45DB899
:10B26000FBBC55BB8B8876BAEA8B4E3B3E8EE0BA70
:10B27000C4481EBBA940533B0999D4B9CB5CC7391C
:10B280002176C8BABA3BB63AAADDBB392087863BDD
:10B29000FBD3B6396D2D5939DA64863BBFF298BAC3
:10B2A000FB46C3BA5BE2FA3A317E093BF430A0BAFE
:10B2B000D800F339B4887BBBC58C9ABAC0463FBB73
:10B2C000B0D4033BB035263A8076293BABC8BDB835
:10B2D0000F950BB94EBE45BB60A27F3A180EB2BAAD
:10B2E0009FF29FB71FA5703AA14C5E3B74C9DBBAB1
:10B2F00017B7E23BDE743CBB53AB64BB5244B23A7B
:10B30000CF5744BB65FFB739FB01ED3A6E8B3A3A34
:10B31000B4DBA8B9CFB3D7B938F19EBBBE5369BA75
:10B32000BFD3183B4E4D2839F733853BD56E053BCF
:10B33000883D8CBBAFB2833A0287803B9F94F8BABA
:10B3400089DFA33A7E2D313BEC5DD73A1950B53AEF
:10B35000A5D6CCB998375BBB393E1E3A9A18CABA03
:10B360001F7323B854945E39D35831BBD0C24B3BC2
:10B3700009BB47BBB394E7BA8A6E97B94AA981392A
:10B38000FF73333B79B0923A6FB2EB398113913A44
:10B3900068142F3B90CA3BBB37B52A3BD6F6213AFF
:10B3A000609446BAB1C08BB8461B4F39CD3E8C3A3B
:10B3B000938EA239D7C9A2B9DFD1C1396284F8B955
:10B3C0002E0A843A1BCC42388A8ADABAB21A37BAC1
:10B3D000F7E81B3A8C132FBBC091943A080C45BB7D
:10B3E0008859A6391E9674BB8CE3D1BA9118413A9C
:10B3F000666F0B3BA64BCE3AF7A5F5BAF4C89D3A5B
:10B400007923A1391C58AAB9A27B843A631D23BAB7
:10B410005A758B3AFA446E3903C454BA7E583ABA14
:10B420004D311D3A2BA3833A5665383BBF4D1FBBA8
:10B43000579CB5BA37F903BB3300D7BAB7DE45B965
:10B440006186003A6C1E223B52D825BA73119E3A8F
:10B450005F119EBA4C492FBB5580BAB9C749A43A6F
:10B46000E4D6223B0A686FBA8AE3883B365C1A3B13
:10B47000E5BB10BB3A13B4BA23B43FBA1FC108BB33
:10B480006944973A5B7DA7B9F27D4D3A1DF20B3BBB
:10B49000F6CD233A325740BB48D93FBBC6F10E3AEE
:10B4A00078DF89BA74B6183B78AE243B0E37DC3AA5
:10B4B00096F1F239808E95BB2151B13A43A0D4BAAE
:10B4C00078E519BB0056383AD19E2C3B0BB5EA3AC9
:10B4D000615EE6BA630E8F3A64504D3AB9D674BBDA
:10B4E000C171C5BABADDE93AD606F33A4DD53E3B4D
:10B4F000B8BB78BAC2116DBB5A46083B827D2CBBE3
:10B500007337F1370E114E3A63227FB918D720B83E
:10B510000268D53A24D3FCB9ACFF14BB535C93BA90
:10B52000043A803A0BBEE13837E29B3A2BD4283BF1
:10B530009D5F1C3B1CB87FBBCEA3BB3A1CDDE3BAAE
:10B540006DDF08BBF820F0B90FE90B3B185D063B37
:10B550006A1814BBABCAF0BADA6BFB3ACD7F7C3BFE
:10B56000AE5CA43AE29BFFBA3CD705BCC38819B9CC
:10B57000A9C1BE39E85989BA1EAD303B76D8EE3A3A
:10B580002E53C6BAC71BCA3AE93BFABA624F793A98
:10B59000BA7E9F3B154D76BB32516C3BD60F14BA29
:10B5A000A6A82D3BC93900BAD19FB7B97812BABB4A
:10B5B000DC3383BA0CB8983A0A520B3BD848A13B0B
:10B5C0009B81EABAA3EFAEBA7C59B039437EC63A42
:10B5D00035C049398A3373BB9025CFBAD2BFEABB95
:10B5E0005DABA53A7001283BFE5C923A0658CC3917
:10B5F000E157F83B4C90943A1B40FE3A52451D3AB5
:10B600008680013BE697C03720B13B3B6E487FB94F
:10B61000A4BE3AB7D45A673AC220283AB61BEDBA4C
:10B6200095F98FBA607AB43A07AD68BAE6CFD5BB60
:10B630004FF753BBC5A136BBA7B9173BE73D453B09
:10B64000716974BADE486538ADA52EBBC34F233887
:10B65000C3BD773A3FE2663B6211C93A9E68173B29
:10B660005C5C9A3B0BE9B8BA8FC363BBFCCD22BBD1
:10B670006745F5BA7C81FC3A65D3DB3A4F360FBBA0
:10B68000E929853BBED01D3BFB10E43A79552FBB21
:10B6900064187B3A2471893ACD5F9FBB6C58A13AFC
:10B6A000AA56193B16E3193BF7C57F3AACFF463A59
:10B6B0008EF2F63A3A5B91BB8A570E3A66CB103A55
:10B6C000DD1C93BB4C98C53A0A21923B7A2C97BA61
:10B6D000533371BBD0FE683BBB1CC5BA51659CBBE4
:10B6E0003CE924BB2C92EE3AD1347EBB59AC663A8D
:10B6F0003890623CCEF478B90060A73A2F49F7B988
:10B700003325143B463122BB3605D5B9BE82B0BACB
:10B71000C764EFBAF5360EBA80F1ECBAE49184BB97
:10B7200078AAF8BAD911163BE189083A2E39B5BB87
:10B73000C2818BBB94AC8EBA44AE18B8B1A3593B4E
:10B740004D750A3B34518DB86D2FB43A01D14BBBC6
:10B75000FD814C3B2E19EF39274AA4BA2C1B89BB1B
:10B76000F70A893B257CBD3B325D273C7C4D92BB73
:10B7700027F1BE3BF9595EBBA591843A7FB342BB2A
:10B78000BED6943AB7A65E3A700D723B07E0E4BBB2
:10B79000D8859BB7F8DE733B51C5B43B28AC0B3B57
:10B7A000A80488BA41BD1D3B8D55F7B9CB3B19BCE8
:10B7B0002B4D703B1A5C353BFA14BFBA76340B3C08
:10B7C000BE0891B98472113BDF6EF5BA05E953BA30
:10B7D00015563BBB1827F1BB796A703B832AD53BD2
:10B7E00011B3A1BADC7395BB8360ADBBF7C93BBB9A
:10B7F0006849C4BB26292DBBB48D2B3B7584DEB8AC
:10B80000F5E2A4BA144BB23AEDF4BEBB634A693B0D
:10B810005B265A3A9FC306BBE4AF123B2875F33A46
:10B82000237C4B3A40133EBB569C53BC0AF6B7BB35
:10B83000005A7C3B94B69B3B6F395FBBBF4B49BB07
:10B840009D9E06B906FA723B79EB6EBBB98D9D3AA7
:10B85000D906583B0254833B55B611BB0BE58EBB52
:10B8600065E33EBC7813C73A448ED13CB28782B9B7
:10B870001A5BC23BB7FCA8B97514013BBE9E843B62
:10B8800028DDA5BAD11672B95C5AC4BA4670BF3A5F
:10B890007E1734BAEC24C5BB14EDBCBB99BFF13A9A
:10B8A000860228BBF2DBFFFF04000000002000003E
:10B8B000C7EF003B6DF0C33A5482DBB7E5B9CB3A32
:10B8C000140B04BBF1CFCFBA2C7219BA951962BB15
:10B8D000DDEBAB3AB681083BB720FAB99711D1BA84
:10B8E00007A9CC3ACDDA44B9AB7A02BB42A37D3783
:10B8F000B19F3DBB60F6A13A60105C3BE9BF64BB01
:10B90000C2DBAEBA23F0A33ADA1CBBBAD86C15BBC3
:10B910003CE397B9EE2DD33ABC12DFBAE88D9FBA5B
:10B92000C75AB0BA721E09BA153FD93A7493123A7F
:10B9300031900ABB4E20D63B998B6739440D3ABBF8
:10B94000D3E1C6B969DC12BBA6A228BB8426C338E2
:10B95000F23D73BBD56E14BBC013203ABC7B113AC9
:10B96000262E8C3BD0A4FABA3839B0BA636CF3BA3D
:10B970008C0303BBB856283B04C808BADF4D0B3B09
:10B98000F0F1A2B9A0CB473A85BD41399EDF48BA54
:10B99000378B78BB0CF5883A62162B38CD3A46BB0C
:10B9A0005B7C973B060E013B92A2353AA90A04BB89
:10B9B000C85A44390F36493B0DA2343B6C76F839EE
:10B9C000ACC35FBBED3205BB53CD353BCF26ABBB24
:10B9D0001DE5E6BA65E053BA3F7E0CBBD06927BAD5
:10B9E000C17B973B4A1A86BB111149BCE2CB32BAE4
:10B9F00073D81DBB4F837CBBD004A13B85FBEB3BC5
:10BA0000B928D5BBAA2D21BB034C5FBB827957BB9C
:10BA1000C57AD0BAE6C0D2BA82EAD5BA047010BBF1
:10BA2000D45207BB1AD53A3B4218C0BBDC2B0DBB26
:10BA3000F9D1063A678AC2BBE06F803A5CA2863AC7
:10BA4000564EAABAD877C9BA849A00BBD949ABBABC
:10BA50004EC4A3BBA449873B58A743BB207A54BB21
:10BA6000931203B9FA0A2EB97E19F9380723C9BB14
:10BA70006399E4BBC27B893BF7F40CBB695D22BBD5
:10BA8000F07CFDBB736740BBDC913B3B6765463B8D
:10BA9000B284EBBAE8B90ABABA95433A412FAE3A42
:10BAA000603FE03A7831053C126F863A56A21A3A66
:10BAB000EF01713B5CEA0EBBDC055C3B02B52A3B47
:10BAC000BEF348BBDDBA09BA140489BB3DDF1CBC18
:10BAD0007A77323AAC7485BBFACADABAF98690BB87
:10BAE0004CC0D9BB0C7A79BB2D0F86BC483179BBD1
:10BAF000C0CC1EBCBD77A2BB2F1C3E3A116481BBDB
:10BB0000A3E007BC9BF17B39C37CE4BA19B65D3B6B
:10BB1000BB31BF3AE27783BBB774CEBB379439BB36
:10BB2000B822A0BA9D25043C6ED7613A132C28BBDD
:10BB30007324AFBB9CA011BC88AEF03AFABF9CBB8B
:10BB40007AA1D73A9C38FB3A9F00863A0C6634BB00
:10BB500095F1AEBB5F8902BBDC281FBBF02D0F3A0D
:10BB60003276D33B65EABEBA61B684BB8201B1BB13
:10BB700041018DBB0877983C2AB27B3B1F1EA6BAB9
:10BB8000D1981CBCE4BF743A54E02CBB37F547BBDA
:10BB900084FF7DBBDCF6B439D11D933A6A4EBA3AC4
:10BBA000D0F9023ADC4BB93AA47B54BB4537483B49
:10BBB000717C983AC31B13BB90FD65BAE7AA293B79
:10BBC0009EB9DAB9FDF18A3AF0DEBA3B138053BA76
:10BBD00080B923B9B63EE03A4D6400BB3032DEBADC
:10BBE00080D7EC3A4AF9563A411A9AB92457A53AFD
:10BBF00072F6393A175E50BB612C98BAE475F63A82
:10BC0000975FA0BBDB1F233B4B83313B024DC5BA83
:10BC1000AC1ACABA2F20B0B8F069B73A074CD1BAFB
:10BC20001D5BE5BAFE3D803B33D36239A6B486394D
:10BC30009356893AAE39223BAD04913B9D16E33AC7
:10BC400062FDEEBA0D10E6BAC3F103BB8D885C3914
:10BC50000929FDB950E2F13A6AB123BB15358DBA15
:10BC6000109CC4BA7D2C66B95C928F38DCDC21BB99
:10BC7000E9EA96BB2327363C1CBCF03A0A9D9ABBE6
:10BC800032AF203BC79F2BBBE7B01BBAE887A0BAF7
:10BC9000330152BBDAB47D39ADA26E3B5EB4E23AF9
:10BCA000B716823B6A6105BBDA718CB4B0B4333A23
:10BCB00047372C3BA5D875BBE8B4E93B80BCFD3ABF
:10BCC000A2923ABB3EA75D3B4ACD0F3C0979FFBA31
:10BCD000CD9D32BBB28C8B3BA3F0813A90DD5A3BB9
:10BCE00036CEDE3B5354923B2A1B07BAC262123B4C
:10BCF0007C9F143CDB190B3B0C7B81BB851929BC59
:10BD0000BBCC4E3BEC024A3B1700B0B957A252BA2B
:10BD1000DE29723B9BB1863BFA199B3BB755CF3A64
:10BD200079A33BB9966C15BA1656893B1882803AAE
:10BD3000032F1F3B5EAAF5BA7514FC3B5BA3E4BA64
:10BD4000BE6FE53BA979A2BB9A94B7B92249413BA2
:10BD50001FB7F8B934B632BB9A3E043B0B743ABAFB
:10BD600038EE71BA0C55523A36F605BBBACE043AE3
:10BD7000E750313C0CF7ECBBC9671A3874A1CEBA56
:10BD80005431153C9452F6BBC7134B3B6655CBBAA6
:10BD90009BE5C2BB034A75BAB761B4BA00C6D33AD1
:10BDA00040F0CE3B66FD02BC2F8523BBDFFE83BA8D
:10BDB0000829F2B9AE1FAEBAF0A070BB3AE6B73AA6
:10BDC000CE454D3A6AD1163B2981D03B3882BC3AE8
:10BDD000ACCFB9398F90F4BA88E4723A8263433BAE
:10BDE000999055BA9A0F13B774086FB99796D3BA4A
:10BDF0005CF28E3B28FB2ABB42477339ACBA11BCBC
:10BE0000834F2CBBFF05093A4866053A0A1814BB54
:10BE1000E8FCA0BA9CFCEA3A5BBD0AB9AF6F6DBA08
:10BE2000BE17C3BAE5590538C155763BA202A5BA7B
:10BE30000B262E3A7F1D2D3B7D106BBA969918BBB1
:10BE4000CF87AD3B74BF3A3BDA77323AF1DE3F3A07
:10BE5000719196BB6F473ABB81220E3B6D90E5B95D
:10BE60004F22BDBAE3F88E3AEB2F0ABBFA7E15BC1F
:10BE7000769A31BB1B37983B0C0C8FBA18F0123BEB
:10BE80008BB9E83B53E6DBB9854C83BAC992BFBA9C
:10BE90003DAD3A3A0D60923A22D3403A763F18BB14
:10BEA0000C5D6E3BE143D5BA67EA09BB804997BA9E
:10BEB000A6D136B96AFF9DBBA18A3E3CFC818E3A71
:10BEC00016BE423B317A60BBAF8A1BBC3C1F30BB05
:10BED000938297B94C83FDBAED2526BB069036BBFD
:10BEE000BF9F3FBB6E0ED13B19D69DBBD170023BAD
:10BEF000937D1EBB574FD43BF8A4A43B55C034BB25
:10BF000055B160BB01B5373A1678D739F5335F3B89
:10BF10001C45F53A8B4521BBE4AC40BB435CD6B82D
:10BF200033FBCDBA016BAB397D389D3B441E5A3A89
:10BF30002237993B04C109BCF5B7D43B0816893BAD
:10BF4000D79210BAB014CE3B867CEBBA7812CEBA38
:10BF500013DCD73A6BFA813BC6DF82BB09F2F9B733
:10BF6000B7276FBB69F8D3398E41933B5525E93B21
:10BF7000D163B13B3AB22DBCC378913B1CAE933A2E
:10BF8000E3E3A33B42A9B7BB3EC5A8B9F570323B7A
:10BF900083FFC13B0752973908F260BBD43836BBE8
:10BFA0009C2B38B869EEC53B3A77C53A8719D0BAA9
:10BFB000D4788FB9D01ED6BA247F853BA0E1BEBA13
:10BFC000BCA1D5B8F751053B13FFAB3B44B7033BCE
:10BFD0006A7ECC3A7CF091BB306A36B96C20F73A75
:10BFE000D2BD5C3BF8717738BA7AF9BB1654E93A9E
:10BFF000A312E0BB4E0F3C3BA915A8BB2FA9233CC5
:10C00000E43A73BBC24471BBA41377BAB1DD3FBB42
:10C010000BA9123BB852E6BAE7E5523B0812A5B9A4
:10C02000A1DDE4BA10A8D2BB8F66D2BB0964A13AE5
:10C030002D9F96BBCDFDA53B9662D43BFB5917BB0C
:10C04000A6ACB1BBDA80813B0701B9BBE623DD3A80
:10C050006BF76F3B0E4C9ABB9D1E34BB1DFD26BB80
:10C06000283CB2BB796C8C399E0C103A9A5B2C3C04
:10C07000CA602A3B3F53FCBC8A60423B04A4E1BB3C
:10C0800000FBDA3B6B919D3B71DE2BBAFD1FC6BAFC
:10C09000380BDEBA4AFA723A3BC9EF3AF7D3E93BBA
:10C0A00081599B3B22F07C3B0A2426BB5BB9A53A15
:10C0B00058548EBB391C49BBF6277EBB94287B3B6A
:10C0C000415A80BBFB58D63ABE380739C7AC583BFB
:10C0D0004D0A88BA36EB54BB60E1383936AF0ABB3B
:10C0E0002DFCDD39E271803B8B2D3C3C84263FB931
:10C0F000381DF93B60AAEB3B44E8F5BB9D0A74BCD4
:10C100005B2F3D3BAE2282BAF2C924BB8B53A739C9
:10C110001DA91C3BB4751BBBC38A0EBB3FE9693A22
:10C1200020BA0ABB381D1ABC82B587BAC26C4E3B16
:10C130007C88EE3B3C320ABC62C1C5BBAED2C33B7D
:10C14000BFC6A2BB2F81433B0303833B89FF68BA71
:10C15000D1AC45BB19FB5A3B17C375375FDE703A4C
:10C160006A384ABBF9DAECBAB7E8973AFAB1D2BB07
:10C170003016183CBEE1DD3B4AC2C5BAE8C0AFBBD1
:10C18000B978803B7DC545BA80AAB9393985A4BB49
:10C190005DCD553B2EA9B83A2A6BFB3B8DF1C9BB4F
:10C1A00084908BBAD728E8BBBB2204BAC8FF8C3A6C
:10C1B0004D6C82BB5892EA3B996A39BA4FAA65BB6B
:10C1C000E6206EBB0A30933B8254F03AA0428A3B91
:10C1D00064BA123BEB6C9CBBAFC90D3B656E703B08
:10C1E00058F1CD3B8B2ECA3BA7641EBDACB7ECB754
:10C1F00092ADC3BA499E0CBC0ACCA43BBDA30E3B76
:10C20000A1AEA23BF6A89FBB1F3614BBFC0A9F3B06
:10C210009CE8023BD28588BBECC169BBCC044A3B9D
:10C220002B085BBBFC4D0C3CA2A81CBCB5543E3B90
:10C23000094AE33866DA663C76BDF43B9911593A0F
:10C24000D00C49BA185E4739CED9FFBBFD4E143B1E
:10C25000A1B4A9BB5594483B3D1B4A3B14729DBBFE
:10C260009AB6053C2B1347BB1678EF3A048ACA3BB3
:10C27000386DEC3B8A8E0ABDFFC23BBAD34C30BC52
:10C28000322B67BBD3E6643A6E20AF3B7D68F83B48
:10C2900036E605BCE4E252BB978E60BC352F063C07
:10C2A000D36983BB69C2D3BB77F1303B48EC9ABBFF
:10C2B000CA76E2BAC9BFD039D179133B51F32DBB4D
:10C2C000FBCEF3BBEB15DD3AB7CB873B80FE6DBBF6
:10C2D000DDE414BB5BDBAF3B2C18063B8617813BD0
:10C2E00082428E3BCB3617BB8F3138BB8EB998BBA1
:10C2F00013DD01BC46259BBAEFC593395F860F3C21
:10C300000200BFBB252B6EBB256A9C3BA3220ABC47
:10C31000658C093BE0CA983BA23997BB493325B9E4
:10C320002E807ABAD1E04F3A4497DCB9C5C138BB08
:10C330009088C8BA68CABABBBA55FDBB6C4231BB5B
:10C3400014871ABB868013BBF297C638B92562BB27
:10C35000C5DA543B073ED6BA114BA9BB732DC13B7E
:10C3600005A698BAC7A07C3BCF306ABB058AFF3AC6
:10C370008C98593B0A7E953C0FF37EBB786D843BCD
:10C38000E860DC360C22B63BCDB44EBBBFC6CD3B1D
:10C39000CCB9213A147BB73A1AC0FE3B82DE823B0D
:10C3A000552591BB3B8321BC61C782BAB76A043B68
:10C3B000926DEB390F126B3B5A54083CAE44CBBA2A
:10C3C0008E1786BBF9DD373B3B85EC3BEF2BED3A17
:10C3D000FFE5F5BAB154AA3939D4BF3A0B092E3A60
:10C3E00004B845BB8495373A99C0EEBB68C6B4BA69
:10C3F0000CE36ABBD839E5BB51D0B93BDC91183CA2
:10C400008009673BA2D89ABA7AECB63BA054E3BB4A
:10C41000A58FE839B1C816BB38C240BBA0F0393A85
:10C4200079412E3BB4FBEEBAB267C0BB7CEF0FBBC9
:10C43000C1D2AE3B006085BB850AABBBBA074E3BA1
:10C44000A416863A9A89E23A5199D03B007B48BBC0
:10C450000C30CE3BDCF8B73926041CBAEB56F93A5F
:10C4600011163E3B60B14B3ADD0C163B6A8B043C27
:10C47000DA617C3BDD10B4BAEF369DBBA002B3BAE3
:10C48000FA7777398991B03A2E10D5BBB9083C3B81
:10C4900062FE1CBB720E403AE19B5A39108F5A3B28
:10C4A000D0690EBBEC7B233B99BEA2BAB09B5EBBAE
:10C4B0005147EA39F3F5853B2EEAE73B7C2898BAE9
:10C4C0007034383B14C3793B79E8BE3B2CBF8D3ABE
:10C4D0007FA8B93AF041E83B5B1A6C3A0E137D3BFA
:10C4E000D94408BCAA73ADBABF00B4BBCFE094BABC
:10C4F000AA6E7C39308DC3BAF160233BDFB8903C23
:10C50000117A06BB3AEFEFBA14A958BA98B0B63B05
:10C510008A1F40BB95FEAB3B1675AABBDF8077B97F
:10C520001052C9BA6338BB3B6039CF3B925C423B87
:10C530004CFFEB3A6282823C2AB92DBCD36A44BBE1
:10C54000B727EB3ADEF897BAEB73F1BABF6C7339E1
:10C55000B787423AA819EDBA208F35BA0262943BE8
:10C560007A27133CA8709C3991AA843B8F486FBBF3
:10C570006B86F5BBDBE08F3CF19BFDB9B4BF9ABB8A
:10C58000D86F793B14DCB0BBC33D613B877FFB3B7D
:10C59000BB38823BBFFEAA3B95529B3B764503BB13
:10C5A0007023CBBBCAAAC9BBC3C116BB075B3E3B4A
:10C5B0007E0D103AE2C27A3B89DE53BBDE522DBBC0
:10C5C000482AF53B770774BBB68829BBD458F1B924
:10C5D0004D75BB39C61735BA0FCF65BACC36D9BA47
:10C5E000664A9A3A927A0C3B88CDCABBDFF43A3B52
:10C5F0001939D9BB611E92BB685D983A382C2FBBA4
:10C60000DC47ACBBEFAC563BFE4AE63A14A5AB3B6D
:10C61000ACF323BBE5EF91B9ACD63EBB66E7063978
:10C62000BA7A2ABB9922833BD428003B44EC3CBA1B
:10C630003840083BA89BB2BBB7C9B0BB16FA073B52
:10C64000608C96BB8622B7BBF1A2F2BA52273BBBE5
:10C65000C754E6BA3DEC913AAA2D97BBF016A6BB9B
:10C660006633393AC39CEEBA4F6294B95787933A0E
:10C67000A81C473B7020083C222E40BABB2AA4BB12
:10C680007CE4EBBB3748883B8505A03A76E4DEBA0C
:10C69000C8F7173B7D0AFBB9A28CB33B8D2C263B18
:10C6A0003F45523B8233683A0638A1BAC30D18BAE7
:10C6B000FFC0F2BA110744BB23AB4C3BE30C7CBB7D
:10C6C00071821F3BE34B943AB8FC61BB3F2C98BB93
:10C6D0002491D5B949E2433B41EE5D39860805BB5B
:10C6E0001D64513A57A0AD3B07E246BC7B5DDF3B82
:10C6F00001B1BF3963FB8EBB056AC0BA67118EBB3F
:10C700006EC94FBBA125063B95B7DA3B2291A83BEA
:10C710003D849EB98999B63A0AFDE6B90061C4B96B
:10C7200048A91C3A344E023A81A1003A50C68ABB4D
:10C73000C9B1F4BA20FD833B23A99BBB33A69A3A27
:10C7400051F82F3BD0A415BB4861B53BECF58BBA33
:10C7500069FF963BDB35223B073B59BAE63D1ABBE6
:10C760006D86FBBAA0A4B939F7A187BBE335823B3C
:10C770004BE2C1BB42FDB83B14F9053B36A44BBCB0
:10C78000DD458D3BA94EB9BA673A4BBBE379383AE0
:10C79000EFD0873B04E1B9BA9FF4843AF73D80BB00
:10C7A00040303C39A275A8BBB9D7C5399CE1E739FF
:10C7B00045DF1ABCDCDFEFBBFC9388BCE4C688BB5A
:10C7C000DFC918383C51D5BAFD5742BCE4CD37BC5F
:10C7D000FCA22C3B3D93C73BC90B5E38E97F8CBA6A
:10C7E000F3E9B539A0943A3AFB0CD5BC6DC8C7BB88
:10C7F000102A75BCECFC973B2D4AEABB06E3053DCD
:10C80000E453CFBABE7CF43B5DDD41BC1F77D0BBA7
:10C810008A30E5BAC1D8ED3B4ECB50BB179685396F
:10C820004459513B45ED613C0CF7ABBA3BCB83BA65
:10C83000440DC5BBE77EF23981053ABB31DC6A3C69
:10C840006DF6963B2B0D443B5C370E3C186720BBC6
:10C850009541BD3B963784BA8EBEF33BFF5F7FBBED
:10C86000B9FA2D3AB7651C385F9DE83B9A65DB3C09
:10C87000A10C053C9A7E793B9B08C839579BD1395E
:10C88000873434388B10143BD648E4BAE484523BE6
:10C89000B9BCF8BB8C19D6BA4D05BB3BD988393C1D
:10C8A0005ABD423C146D6EBA98E59DBB21C6133942
:10C8B0002D801D3B0310ECBA11AF323C9C79B93A84
:10C8C000C1ABA2BB664BE3BA74D5C6BA276AF43AC9
:10C8D000242C54BB51A6FEBA3150913ADE9D883BC0
:10C8E0002F65ADBA26303B3ADC8B8FBA4CF37E3BDA
:10C8F00039AB39BB86573E3BF006AC3BC3CE2EBCB2
:10C90000C59EFC39547C103B40D0E5BAAC4B9E3BF5
:10C91000A77064BB6B65ADBB3EB0833BC8552D397A
:10C92000A767AC398A13E5BBF84A543B94E2D33A83
:10C930009FC482BBC75B223BF57738BB572541BB01
:10C940002A3CF83AAC5189BAFE1EE5B975DA86BBC5
:10C95000C437A23A7E3B70BB988CC0BAD42218B8B8
:10C96000CC7769BBE211753BAC91B43B3B689B3B18
:10C97000A8EC94BACE824E3C54CBF0BAEDBC503BFE
:10C98000DED7D8BB0C95FABA4F3DA33A6BD99E3B84
:10C990005F4EB73B5F0518BB92CE73BB5DC0A73A35
:10C9A0005648ADBB0A270A3BE4071BBBAA4AB8B9E5
:10C9B0006891B43A39D726BB388886BB312C103BF6
:10C9C000A4C453BA4CA5403B8D4E443AAE73A13A31
:10C9D0004CC8CD36013041B8E70CC0380B8AE33A79
:10C9E0009E6024BB681A5BBADC33AB3B814482BADD
:10C9F000E31E213B067ADFB9A831F43989F999BBE6
:10CA0000E3F0923AFB4957B853BF693BF1BB5E3A3A
:10CA1000B420E1BA71121A3B3465BF39530C2DBAF8
:10CA2000E143F7BA123AF439D71A133BCB7A2D3ACD
:10CA3000C9CE99BA5D7F95397351E73A0F67BABA93
:10CA40001EF2573B8CD64FBB88CF87BA08AE273B28
:10CA500096B978BBC90407BBD05CECB9F6879D3AA0
:10CA6000F037603AA499323A5489863AD584DD3B4E
:10CA70009A8284BAEA992B3AF56B59394596983BD4
:10CA8000528DD0BAFAD1D6BA561B053BAFBB4CBBC0
:10CA9000C88C2F3BEB815EB9E6AC9DB9640183BBCA
:10CAA0007045913B73CE8D38D0E28A3A2899E8B927
:10CAB0005E75B1BA00E1AD3A6E46CF3B73392EBB1D
:10CAC00023E14ABBCDEFFAB96DA35CBB89D5723ABD
:10CAD000C01BCE3A7BBA7BBAE687E4399B16083A8C
:10CAE000E8A40E3B74876539FF4814BCD419833A17
:10CAF00007C4DEBB312F363B94B789BAC064D33B41
:10CB0000CDC28D3A19B4F9BA36795A3A4FF11DBBF4
:10CB1000D3A0963AE7DC133ACB224339C4B224B906
:10CB20000CF17CB90E0E14BBCBF20D3B3F73CC3A2B
:10CB30001ECB913877C328BBCC2F27BA13568ABB9C
:10CB40009E257FBA44B7143B63F0B2BAE786603AD9
:10CB5000BE93343A51C21FBB2E238FBA3DD0BA3A8E
:10CB60001C30EF3A0EB20E3B7C8DA2390D6FEFBA3E
:10CB7000E7269A39089509BC3159323A2EDA193A22
:10CB800037B0B8BBB4122D3B0817A33840859EBA06
:10CB90005DF1233950833D3AFCC72D3B1FB7B43BB1
:10CBA000D7BBA9BA24D081BAAD4E003BD444A83A31
:10CBB00009B88EBAC592EB3A580C163C9161AA3A64
:10CBC000D87E56BBE32B17BBFA6C64BBBA2B133B66
:10CBD000663F0C3B441287BA94AA06BA28A2193BB6
:10CBE000ACA853BBBD94973AD216FDB892BDFAB922
:10CBF000A3FF25BB7B9510BA919C22BB0A8A3D3CC2
:10CC0000A95212BB220F78BAE1A2B0BAF309813A55
:10CC10007B302E3B7C812BBADE6F19BB2040733AF0
:10CC200025A64BBACA5D0ABA58B42BBB9E5102BBAB
:10CC30005DC74EB9AF08E83908D2663B3BDA1CBB8A
:10CC4000D8531CB77FCF263AF934B33ADDE30CBB97
:10CC500077E4193B878B1E3B3340AABAE78D0E3B26
:10CC60005C47D13ACC7BAA3A8DBDB73A7A8E9639D9
:10CC70008FA6943BB09748BB39B4623BCF4AD3BB35
:10CC8000BB44A3BAC234693AEB7BA4B719E8B83AFB
:10CC9000EBFCDA39432443BBDC4F58BB7310E3BAD7
:10CCA00014CD3E3B9E576039357491BA64D603BBB0
:10CCB000AE64B53A7B68F43B0400D93BBFEC7FBA65
:10CCC0008D74EBB8985EC93866B6C33BB3D938BC2F
:10CCD000FD29D3BAF2141D3B24FA04BA73671DBBB5
:10CCE000AE6EC93B9ABF7CBA610B43BCFE3D83BAB2
:10CCF000BA66693BEC64F337D6DBE03A219600BABA
:10CD0000D7CBC83A6D1C09BBC82D61BBD599193B5F
:10CD10007D49EBBAAF0CC0BB35F99D3ABB4737BA7A
:10CD2000CA55063B96220B3A2E593BBB8F077BBB5D
:10CD30006710963A9532AABA2CB0E43AF998BFBB7C
:10CD4000419AADBB713DAB3BDF3F893B94E747BBAD
:10CD50002248773BBED452BAEF3910BBC0B9B3BA40
:10CD6000AD0087BAB4BDA4BA92DFB0BB023590BCA7
:10CD700089B6D63BC807113C2977C8BA97D668BB95
:10CD8000894E653B5548363B95B99A3B3900EBBA1D
:10CD90007BF514BB3A5424BA9424A83BB567C8BAAF
:10CDA0000A387BBB0D87C63B36FA013A8FE254BB8B
:10CDB000980A963BF629973BC8A021BB058BA23B5E
:10CDC00049D2C93B247C3DBB7C125F3CEE63A4BBD3
:10CDD00030D705BBEB4C293B61DC93BB4778A6BA47
:10CDE000B48FD6BB2F165D3B1FB94E3C7A4497BB20
:10CDF000462959BB9B7AD63B68FADFBB1336803C89
:10CE0000560918BB95ABE53A3CEF08BC2E87DC3BD6
:10CE1000FE4AF3BB022239BB077394BB184DA23AFA
:10CE2000E5AB883769087FBBF15F2B3B35C9E53A35
:10CE3000F4753CBB9050A7BC3D5532BBA275063C77
:10CE4000A8860F3AFE856F3B90AC143B9374463B2B
:10CE500059F6C6BB9706853B614C74BB014FED3B51
:10CE6000570626BBDC1C97BBC9C4C6BB929B89BCBA
:10CE7000FA39BC3B431E223D14456BBB46A980BB1F
:10CE80004CF417BC675AD33AE26D96BB5B22F13A79
:10CE90003EA35F3A984EFDBAE296D23B2B7ED8BABB
:10CEA000F23471BBEDBF7DBB1DBEF43A581EBC3AD7
:10CEB0008DD3C33AC167F53A346CF2BBEC6F783A64
:10CEC00083BEA53A338A143B84715EBBC39FAF3BDC
:10CED000BF463EBAAB8118BBDDD08CBAB14F133B15
:10CEE0006A94863B1931613931A1BC3B15D49FBA94
:10CEF0009874E039A9C56FBBEA5BA23ACACBFABB0A
:10CF0000CB4121BBAE28E63A832FBF3A01F581BB66
:10CF10002D24093BF943BDBADE2F213BFB81EE3ABC
:10CF2000EC4EE43AE7D5133BAF96813B5011293BD9
:10CF30000E151C387B4C8D3B5CECFC3AF7C0433B38
:10CF4000394DD03A249C8EB99F0976BB7204A5BA9C
:10CF50003236D7395E1C02BB0677843A7DFFFB3A36
:10CF60009DD4493B56BD9BBA5A15ADB95D01C83B2E
:10CF700069FDFC3A6256B9BB372B61BB35942F3B38
:10CF8000FA1A923BEF383ABB5961E73AEB2F45BBAF
:10CF90002A16AB3A8EABC5BAEDACA9BB6A2C01BB65
:10CFA000C2B5C13B2CC5D73B1A8F59BA476E103B4F
:10CFB000A99A0B3B14F0033B7B7FA03BC1993CBB80
:10CFC000EF5F8BBB895E73BABC3BA5BB0EE089BB30
:10CFD000DE11B3B84131273BCA728A3883D325BBEF
:10CFE00061DDB33A843672BA09B714BCD9AE663A79
:10CFF000EFDA9B39E436593A034E463A4090C13B4A
:10D0000002070C3B3B7596BB537C39BA8216E73A54
:10D010004931ED3A0D213F3B8EAE183B2753B93ACB
:10D0200006CED0396F803E3B642212BBF48CA9B986
:10D03000688C98BADD84223A7756A3BA8F66ADBB66
:10D04000581196B86B5804BBF3338FBA99F836BBB6
:10D050002C7AB2BA75BBF13A8F507A3A009D2CBA4D
:10D0600048F5C3BA9A7D683AA626833941375B3CB6
:10D070003EE424BBBBF546BBFCA8CBB99BEA34BB62
:10D08000FA9E0D3A85D185BA0CFC053A1B213E3B30
:10D0900032E31A3B156D4C3AB03FBDBA6E336E3B6E
:10D0A000D0411C3A42ED33359A6243B8E956093B08
:10D0B0000ACC133BA15D8F3ADC68C23BEACC9F3AB5
:10D0C000A1D42BBBF93502B70F46CDBBBA7893BBC1
:10D0D000B3166239D3C979BA83D1143BAFDD71BBC2
:10D0E000EFA61DBB561B163A11A01B3BA3335D3B9D
:10D0F000A78D27BCC2B6A8BB522AAE3A8DF0FE3B24
:10D100002E0EC8BB772566BB9BA976BB1986803BD4
:10D11000E697B83ABB2A12BAED50283B226212BBFE
:10D120000FB9F9BA7CF02ABB86FB7CBB38511F3B98
:10D13000A045113B8A6087BB5DEBB83BC9ACEDBB3A
:10D14000D6F263BBEBF5F8B7E636553B819111BBE0
:10D150008288923B09A68E3A30CB06BAFFE9AC3BF7
:10D160002DE90E3BE9F8F1B86AEA80B99A78983A65
:10D170000D7245BA002F853B68C13FBA4DCE2EBA1D
:10D18000D67D6AB9D79BFFBA4FEC93BA5FB17E3BAD
:10D19000C3BDEB3ADA9472BB40196B3BE170DD3BE7
:10D1A0008207243BB673393B406DA7BAE01594B9AA
:10D1B00043219C3AEE5A2A3B84C682394F9C32BBAB
:10D1C00079DDC23B3D06C1BA3116ACBBC260A7BB1C
:10D1D0007A5DF7BA9721B9BAC023D33A1892B0B999
:10D1E0006F57883AA6258ABBDF41C63C3D90A8BA56
:10D1F00022D5CBBA750BC73BB1001B3B95A57DBBB8
:10D2000020B1923B68159E3BFB2C1DBA5FDC103CA5
:10D21000DE143ABAFD26A8BA5F04B03B029039BBCF
:10D22000206E013A4A114C3B2EEE823B9BA9FD3AFF
:10D23000A4809A3BA6568FBB6EEEA43B793E52BBB0
:10D240004FED4F3B3490903B70C7EE3AB68A543B5B
:10D250002B7DA2BB46597D3B007A093B899E8A3BC8
:10D26000E1AA1DB9D4693F3BFCD45ABB7B30D9BB82
:10D270006BADA03B0A6A6F3BE3011ABBE7FD93BBB2
:10D28000EBED323C5AABD63ADBE768BBF25F1CBB36
:10D29000B247F839C51D21BAA900BA3B9DBF9F3BD3
:10D2A00059AA573B55AD78BBD87DFABAB766593BFA
:10D2B000261E0BBB88E0C23991929FBBC49A67BA05
:10D2C000D49CE23B1071FEBAA458D13A598296BB65
:10D2D000F8FEA3390C3B6CBA67F860B81D3BBDB9CA
:10D2E000514188BBA178A8BA71870EBB92C55D3B3E
:10D2F0004646493BF2D8EBBA0F1758BB4A6452BCBA
:10D30000B3A479B9A2B9D8BA8046243AB77607BB94
:10D31000F04793BA482775BB7538FCBA4BE95F3ABA
:10D320009C9AF6BA776EB9B9566A4A3AEF85973938
:10D33000BBBD42BA106316BC76A9263BC682073C29
:10D340005E53B9BB395EE6BB0E68B8BA468455BBBE
:10D35000B5E0753B9CFA1939D505E8B91DD88FBBE6
:10D36000C8E090BA287AA6BAB27F85BB8A9A17BC61
:10D370007437653B405CF93AD83338BBAA80BCB8F7
:10D3800040E7F7BBB45E8ABA72CFB4BA8AB1E3BAE7
:10D3900025FEA2BA86F21CBB12DE653B02DECABACB
:10D3A0003D6809BB824C10BCB511063BF5980839A5
:10D3B000B01626BB1FEDD2BA8DF9DE3BEF2125BB9F
:10D3C0009E3491BB16CA583B28211BBC96ECCDBAA3
:10D3D0004CB8573A89A46F3BE150903764A99C3808
:10D3E000DAF55ABB87B0BCB9FDF375BC964EBD37B4
:10D3F000D62DECBB081E9CB80A077FBBD862B7BA13
:10D40000B4BE7BBB6C606338F3B1C7BB79A2C0BB51
:10D4100040C4DFBA2BBD403A0FD959393362F4BA50
:10D420002A46443BDDB51B398D9F74BBFA4C26B8A8
:10D43000DB54293B3D3FAEBB77CCB73BA9BB383B68
:10D440003B3EB5BAA0B2853BA339CEB935F54FBB4B
:10D4500045CAA0BAD42502B8FD1891B9D141BEBAC7
:10D46000142D43BAC182E33AA59C543B5296553CD5
:10D47000FC3E9CBA1444B3BCC4A47B3B19683F3B3C
:10D4800061079FBB7AD54B3BED4BC13AAFFE2B3BBF
:10D490001A731A3BA51C05BB9FC3393BBA83853B56
:10D4A000ECCF26BBE36EB6BA04C612BB0A540DB964
:10D4B000A4C9193B5A9EF13A135D4BBCA113813BA1
:10D4C000FEE69C3B31A788BAC1B5C63B57630B3C0F
:10D4D000EA46E23A56CA02BB5E547CBAECAD74B975
:10D4E0007F07A9BBA9E32CBB1E8F133C59695A398E
:10D4F000C7139A3AFB755FBA79F6993BD85A08BCBC
:10D50000ABF36E3BB88EC83906F1DFBAA9CFF3BBD7
:10D510009ED095BA1F44F8BA28566F3B8FDB97BA56
:10D5200069E2F838EF35C23B426866BB829A96B929
:10D53000C9FA8CBB41D6493CC4CCC7BBD88B853912
:10D54000CDAD983BA9CA7DBBCC0F0B3B175A353BE1
:10D55000266993BB3F7F88BB4EB41BBB8E33ED392E
:10D56000C60D92BAF6E5173B144C10BBB286803B51
:10D57000BA0F083CE9E86ABBAAA5213BAFB38BBB55
:10D58000EADC0BBB0EAD08BBF1DC923A426C5BBB34
:10D59000B814803BE12703BB6CA5853BE573DE3AFD
:10D5A00094B7573BE12B4CBBE4429BBA7A4F3B3BD1
:10D5B00069FCE53A13C5E9BA023D803B74BE18BB6D
:10D5C0009AAC51BA85B35A3B9FA814BBCD7872BBB5
:10D5D000AB60463B3AEC4E3A1D870DBBA10D8D3B2F
:10D5E00029ED67BBFAFA493B2BF78DBB9C66FD3AE8
:10D5F000B05DAABB16F9F8BB799C863BF296B7B82A
:10D60000459685BA4203C5B776B1233B3C0ABD387F
:10D610004D6A9A3AE64D17BB333F443A61D298BA05
:10D6200098BBB43A74D2B33AC46383BABE2D16BB66
:10D63000E6FDABBB5008063CF3A614BB3BCFAC3BAE
:10D640002194833B97BB06BC703098BB4F69BA39B5
:10D65000FEEF70B947D5B0BB2B76EABA15B8FBBA66
:10D6600026A4BD3A0878D33A60EFFEBA325E51BCC8
:10D67000744948396FBD173C2E80653B3775593862
:10D6800084B379BB8CEBE438E9BED03A79BA80B97F
:10D6900072F665BB6CC34839C1BF353ACB3FE23A3D
:10D6A000599AB7BA4EB98E37F46C4ABAE3F2F137E9
:10D6B0001B9560BA9C1DB7BBA0DD89BBE7D52DBA11
:10D6C000E419ED3B6CC234BBB7A3D7BAC00A043C23
:10D6D000791EFA39A5EE1F3B6BC1253B02875D3BE6
:10D6E000EEF8FEBB0C0CD43B481DE13C5DE634BBC0
:10D6F000537221BBBA3AF6BBDEF00F3B9B27ACBCA2
:10D700007A5EA8BA5CB47C397BC83C3B95ACC3B8A4
:10D7100036353DBB83CB833BBB396ABBA62BC1B936
:10D720007C3C893A82E4C33B131B233BBA0E18BBF3
:10D7300053BB593BEC698ABA10182ABB527BCD3BCC
:10D74000C87735BB87FAD0BBBD8BB4BB347EEF3A0C
:10D75000BAC097B9065052BBC72460BB3C40C7BB98
:10D76000770AA6BB65E2193B605BB13934DB32BC9A
:10D770005C50083C74EBBCBA69447B3BAB5E15BBA8
:10D7800037AF823A5799B5B94512FC3AAF356B3B82
:10D79000DF21C03A191ABE3A38CA0ABC491D84B9F9
:10D7A000016C853B2C5F5ABC1CDF1EBA6E02823BAB
:10D7B000EE2BBBB8FC3C03BBA72C75BC4E0CD63A79
:10D7C000F979233B841D953AF0E818BA663DE33BAE
:10D7D0003F363BBAB4A644BB8C379C39B4A28B3AD3
:10D7E00040A9DB3B18CF51BBF11D9FBB63EAD03989
:10D7F0006010D8BB4CF8C5BBDC23B53BB1372B3C24
:10D80000FCDCA03A83F95D3AD4A74E3BC7B824BCF0
:10D810006DCA8CBA4AFBCDBAA1539EBBB1E5C53ADD
:10D8200041AC19BBC436A4BB431CBC3BE37A7D3B73
:10D830001B44C83A3E4DDF3BEC5587B90556FFBB4C
:10D8400087D44B3A195E29BBB85E62BBEE2253BB4C
:10D85000D8C2A63B5583D73B03C8143B5F5717BAC2
:10D860001D1EE1B9E41E973A3CF738BA9B89833C08
:10D87000D160B6BA89D3DEBB2EE6A73B0463473C32
:10D88000DD16C53BE718903B44ECC53B1E47BCB9D1
:10D89000702658BB22253EBAF1948B3B1F3167BBE3
:10D8A000BFE0E83B84447D3B1ACB843ADCB96EBBD5
:10D8B000FEFBFFFF04000000800000009E789FBE7A
:10D8C0008F925A3EBD331EBEB8AD79BEA308B6BC1A
:10D8D000D4DEEFBC0F49CCBD6BD92EBCB4B4F1BDC6
:10D8E00047E123BE3E463FBD94DD143E23C7C3BD82
:10D8F000A17FEABB3A4F65BE51DA25BE8D955D3EEC
:10D90000312311BF144E88BD3C7D74BD3275183D66
:10D91000E71F87BD37AB19BC0E42C8BEA6FE7E3DD1
:10D920008BE082BE0C177B3E664BC2BC044D3D3D76
:10D93000F746ED3DBC594D3D279D42BD8AFCFFFF9A
:10D940000400000080000000CC668ABE0D11183F64
:10D95000D39FAFBF3C9197BF85CE853F4D3CA5BCC3
:10D9600053C3CDBE37C03BBFC39F81BF807E60BF66
:10D97000F5C652BFEB7DB7BF44631BBF7C873FBF7B
:10D980001642B43DE760F5BE473942BFDDCFD4BE95
:10D99000F22883BF535433BF4E129BBFC93C8F3E06
:10D9A000C45A87BFFE188CBFDC6B8CBF8F7B643E74
:10D9B00086063DBFC6D22BBF89E094BF53F5E63C37
:10D9C000229EDCBFDF553BBF16FDFFFF04000000B9
:10D9D00080000000464E50BFDAB30640A3F9FCBEFB
:10D9E000FA57ADBE464020BF188AF3BD11EC07BF01
:10D9F0003D9093BE7FDA8ABF869320BF85E6553F70
:10DA00000826C83F5E78C1BD54E11FBF23F7293FF8
:10DA100056473D3F8C41EEBEE00D67BFFD2768BE17
:10DA20007FD1043F437BEC3EE71BB5BF62CDB7BF60
:10DA3000D189C8BE92782E4061E413BFD3CFC63FD0
:10DA40002841883F5D6A1FBFF26C7BBFA93B4B40FA
:10DA5000AA18C93EA2FDFFFF0400000080000000DC
:10DA6000853FD9BE49E84F3DDB2C0DBD9DA511BDBD
:10DA7000978F37BE27F628BFB48442BED31B9DBD07
:10DA8000ACEE2A3C6D36A0BDFD1D3D3D3A8DB3BDCB
:10DA90009547923D4A90933C5F103ABC52BE88BD78
:10DAA0002F27E8BE8F50863D8A9FAE3D3B8D9EBEA0
:10DAB000DB80423DC2B303BF90B023BD88B014BE2B
:10DAC000DBF914BE268845BD488C50BEAC4D62BE05
:10DAD000D402A3BE534229BE782CE2BC0AEFCF3E4B
:10DAE0002EFEFFFF04000000800000009C64DFBFEA
:10DAF00023323E403632883F2D8D2E3F00C8ABBFCB
:10DB000059A710BF5505C2BF23785FBFF08D8FBEE8
:10DB10000CD2BD3FAC0A2DBD1B8B623F937C0DBF69
:10DB2000AD090BBFB0A6FB3E7DE9883F4304113F22
:10DB30009825DDBF5123AC3F3CFAB03F92FC184022
:10DB4000D6257B3EAE89D3BF5A0172BF14D3C33FE3
:10DB500010574B3FD39967BF68FC04C040A28BBEEF
:10DB6000491D59BFCA8B49BEBB5314BFBAFEFFFF44
:10DB7000040000008000000014E1BE3F4F3895BF54
:10DB80002EE48ABF570FA33E70389E4001CA1C4046
:10DB90000AD1AABF1C1F143FAE8F85BEDBA0E33E97
:10DBA000ED604CC014AC0FC088DE04C04A202BC00E
:10DBB0004D5353C054EF1FC0C6C9B7BF40E3144014
:10DBC0008FFE96BF540102C03D1294BF79E440C05D
:10DBD000834E9B40D18B8DBFBAFF13C068AD3340DD
:10DBE00026F527C06FF4FBBFD17D4140F67C09BF0D
:10DBF000FF26123ED7BA094004E8FFFF08E8FFFFFE
:10DC00000F0000004D4C495220436F6E76657274D0
:10DC100065642E00010000001400000000000E00EA
:10DC20001800140010000C00080004000E00000092
:10DC3000140000001C0000000404000008040000A0
:10DC40000C040000040000006D61696E000000001B
:10DC500011000000C8030000840300003C03000022
:10DC6000F8020000BC020000840200004C02000028
:10DC700014020000D80100009C01000064010000B3
:10DC80002C010000F0000000B4000000780000004B
:10DC90004000000004000000CAFCFFFF1C00000060
:10DCA000000000091C00000020000000030000002C
:10DCB0000000060008000400060000000000803F8D
:10DCC000010000002B000000010000002A000000FD
:10DCD00002FDFFFF1400000000000008100000001B
:10DCE0001400000001000000F4E8FFFF0100000044
:10DCF0002A000000030000002900000012000000BC
:10DD00001100000036FDFFFF1400000000000008B5
:10DD1000140000001800000001000000AAFDFFFF31
:10DD200000000001010000002900000003000000C5
:10DD300028000000100000000F0000006EFDFFFF33
:10DD4000140000000000000814000000180000008B
:10DD500001000000E2FDFFFF0000000101000000E3
:10DD60002800000003000000270000000E00000053
:10DD70000D000000A6FDFFFF1400000000000008D9
:10DD80001400000018000000010000001AFEFFFF50
:10DD90000000000101000000270000000300000057
:10DDA000260000001A00000013000000DEFDFFFF47
:10DDB000140000000000000B140000001800000018
:10DDC0000200000052FEFFFF000000010100000001
:10DDD00026000000020000002500000022000000D4
:10DDE00012FEFFFF140000000000000810000000F9
:10DDF000140000000100000004EAFFFF0100000021
:10DE00002500000003000000240000000C000000BA
:10DE10000600000046FEFFFF14000000000000089E
:10DE2000140000001800000001000000BAFEFFFF0F
:10DE300000000001010000002400000003000000B9
:10DE40002300000019000000140000007EFEFFFF08
:10DE5000140000000000000814000000180000007A
:10DE600001000000F2FEFFFF0000000101000000C1
:10DE70002300000003000000210000000B00000050
:10DE800005000000B6FEFFFF1400000000000008BF
:10DE9000100000001400000001000000A8EAFFFFCD
:10DEA000010000002200000003000000210000002B
:10DEB0000A00000004000000EAFEFFFF140000005A
:10DEC0000000000B14000000180000000200000019
:10DED0005EFFFFFF000000010100000021000000C4
:10DEE00002000000200000001D0000001EFFFFFFD8
:10DEF00014000000000000081000000014000000E2
:10DF00000100000010EBFFFF0100000020000000F6
:10DF1000030000001F0000000900000003000000D3
:10DF200052FFFFFF14000000000000081400000072
:10DF30001800000001000000C6FFFFFF0000000104
:10DF4000010000001F000000030000001E00000090
:10DF500018000000150000008AFFFFFF1C000000F1
:10DF6000000000081C00000020000000010000006C
:10DF70000000060008000700060000000000000185
:10DF8000010000001E000000030000001C00000053
:10DF90000800000002000000CAFFFFFF140000009C
:10DFA0000000000810000000140000000100000044
:10DFB000BCEBFFFF010000001D000000030000009B
:10DFC0001C000000070000000100000000000E001F
:10DFD0001800140010000C000B0004000E000000DC
:10DFE00014000000000000081000000014000000F1
:10DFF0000100000000ECFFFF010000001C00000019
:10E00000030000001B00000017000000FFFFFFFFDF
:10E0100000000A000C000000080004000A000000D4
:10E02000080000000C000000010000001B000000C0
:10E0300002000000000000001600000001000000C7
:10E040002B00000001000000000000002C00000078
:10E0500024130000C012000060120000181200001B
:10E06000CC110000841100003C1100009010000051
:10E07000F40F0000A80F0000580F0000140F00005C
:10E08000C80E00005C0E0000B80D00004C0D000032
:10E09000A80C0000500C0000C00B00006C0B00002E
:10E0A0001C0B0000CC0A00008C0A00002C0A0000A7
:10E0B000E8090000A40900005C0900000C09000048
:10E0C000B4080000C0070000E40600006C06000071
:10E0D000D405000088050000E004000050040000A2
:10E0E000D803000040030000F002000070020000AE
:10E0F000B801000000010000600000000400000002
:10E10000A2EDFFFF00000001140000001C00000051
:10E110001C0000002C000000340000000200000081
:10E12000FFFFFFFF0200000034EDFFFF19000000B9
:10E13000537461746566756C506172746974696F4B
:10E140006E656443616C6C3A3000000002000000B0
:10E150000100000002000000FAEDFFFF00000001D6
:10E16000140000001C0000001C0000002B00000038
:10E170007800000002000000FFFFFFFF0200000027
:10E180008CEDFFFF5F000000626E5F6F757470754D
:10E1900074332F62617463686E6F726D2F6D756C6E
:10E1A0005F313B626E5F6F7574707574332F62619F
:10E1B0007463686E6F726D2F6164645F313B6F755D
:10E1C000747075745F6C617965722F4D61744D75F3
:10E1D0006C3B6F75747075745F6C617965722F42FA
:10E1E00069617341646431000200000001000000B5
:10E1F0000200000096EEFFFF000000011400000086
:10E200001C0000001C0000002A000000900000001C
:10E2100002000000FFFFFFFF0400000028EEFFFFE8
:10E2200074000000626E5F6F7574707574322F62D7
:10E23000617463686E6F726D2F6D756C5F313B62D8
:10E240006E5F6F7574707574322F62617463686E7F
:10E250006F726D2F6164645F313B6F75747075749C
:10E260005F64656E7365332F4D61744D756C3B6FE4
:10E2700075747075745F64656E7365332F52656C69
:10E28000753B6F75747075745F64656E7365332F5D
:10E2900042696173416464310000000002000000C3
:10E2A00001000000040000004AEFFFFF0000000131
:10E2B000140000001C0000001C00000029000000E9
:10E2C0009000000002000000FFFFFFFF08000000B8
:10E2D000DCEEFFFF74000000626E5F6F7574707596
:10E2E00074312F62617463686E6F726D2F6D756C1F
:10E2F0005F313B626E5F6F7574707574312F626150
:10E300007463686E6F726D2F6164645F313B6F750B
:10E31000747075745F64656E7365322F4D61744DF2
:10E32000756C3B6F75747075745F64656E73653280
:10E330002F52656C753B6F75747075745F64656E94
:10E340007365322F426961734164643100000000DB
:10E35000020000000100000008000000FEEFFFFFC7
:10E3600000000001140000001C0000001C00000060
:10E37000280000005800000002000000FFFFFFFF1F
:10E380001000000090EFFFFF3D0000006F757470FB
:10E3900075745F64656E7365312F4D61744D756C76
:10E3A0003B6F75747075745F64656E7365312F5261
:10E3B000656C753B6F75747075745F64656E7365BD
:10E3C000312F426961734164640000000200000063
:10E3D00001000000100000007AF0FFFF00000001C3
:10E3E000140000001C0000001C00000027000000BA
:10E3F0002800000002000000FFFFFFFF20000000D7
:10E400000CF0FFFF0C00000052656C755F353B613E
:10E4100064645F31000000000200000001000000A1
:10E4200020000000C6F0FFFF000000011400000003
:10E430001C0000001C00000026000000700000000E
:10E4400002000000FFFFFFFF2000000058F0FFFF68
:10E4500054000000657870616E64322F4D61744D18
:10E46000756C3B657870616E64322F4269617341EF
:10E4700064643B626E5F657870616E64322F6261C6
:10E480007463686E6F726D2F6D756C5F313B626E79
:10E490005F657870616E64322F62617463686E6F5D
:10E4A000726D2F6164645F310000000002000000A3
:10E4B00001000000200000005AF1FFFF00000001F1
:10E4C000140000001C0000001C00000025000000DB
:10E4D0005000000002000000FFFFFFFF10000000DE
:10E4E000ECF0FFFF37000000626F74746C656E65BE
:10E4F000636B322F4D61744D756C3B626F74746C3D
:10E50000656E65636B322F52656C753B626F747418
:10E510006C656E65636B322F4269617341646400A0
:10E52000020000000100000010000000CEF1FFFF1B
:10E5300000000001140000001C0000001C0000008E
:10E54000240000006800000002000000FFFFFFFF41
:10E550002000000060F1FFFF4D000000726564754F
:10E560006365322F4D61744D756C3B7265647563E4
:10E5700065322F426961734164643B626E322F627F
:10E58000617463686E6F726D2F6D756C5F313B5295
:10E59000656C755F333B626E322F62617463686EC7
:10E5A0006F726D2F6164645F310000000200000033
:10E5B00001000000200000005AF2FFFF00000001EF
:10E5C000140000001C0000001C00000023000000DC
:10E5D0008000000002000000FFFFFFFF200000009D
:10E5E000ECF1FFFF6400000070726F6A656374698C
:10E5F0006F6E322F4D61744D756C3B70726F6A6532
:10E600006374696F6E322F426961734164643B6267
:10E610006E5F70726F6A656374696F6E322F6261CC
:10E620007463686E6F726D2F6D756C5F313B626ED7
:10E630005F70726F6A656374696F6E322F626174A6
:10E6400063686E6F726D2F6164645F31000000005B
:10E65000020000000100000020000000FEF2FFFFA9
:10E6600000000001140000001C0000001C0000005D
:10E67000220000002400000002000000FFFFFFFF56
:10E680002000000090F2FFFF0A00000052656C7548
:10E690005F323B6164640000020000000100000082
:10E6A0002000000046F3FFFF0000000114000000FE
:10E6B0001C0000001C000000210000007000000091
:10E6C00002000000FFFFFFFF20000000D8F2FFFF64
:10E6D00054000000657870616E64312F4D61744D97
:10E6E000756C3B657870616E64312F42696173416E
:10E6F00064643B626E5F657870616E64312F626145
:10E700007463686E6F726D2F6D756C5F313B626EF6
:10E710005F657870616E64312F62617463686E6FDB
:10E72000726D2F6164645F31000000000200000020
:10E730000100000020000000DAF3FFFF00000001EC
:10E74000140000001C0000001C000000200000005D
:10E750005000000002000000FFFFFFFF100000005B
:10E760006CF3FFFF37000000626F74746C656E65B8
:10E77000636B312F4D61744D756C3B626F74746CBB
:10E78000656E65636B312F52656C753B626F747497
:10E790006C656E65636B312F42696173416464001F
:10E7A0000200000001000000100000004EF4FFFF16
:10E7B00000000001140000001C0000001C0000000C
:10E7C0001F000000B400000002000000FFFFFFFF78
:10E7D00020000000E0F3FFFF980000007265647500
:10E7E00063655F696E697469616C2F426961734129
:10E7F00064643B626E5F696E697469616C2F62610B
:10E800007463686E6F726D2F6D756C5F313B626EF5
:10E810005F696E697469616C2F62617463686E6FA1
:10E82000726D2F6164645F313B726564756365313D
:10E830002F4D61744D756C3B726564756365312F46
:10E84000426961734164643B626E312F626174633B
:10E85000686E6F726D2F6D756C5F313B52656C75B4
:10E860003B626E312F62617463686E6F726D2F61EF
:10E8700064645F310000000002000000010000003D
:10E880002000000026F5FFFF00000001140000003A
:10E890001C0000001C0000001E000000CC00000056
:10E8A00002000000FFFFFFFF20000000B8F4FFFFA0
:10E8B000B10000007265647563655F696E697469B3
:10E8C000616C2F426961734164643B626E5F696E83
:10E8D000697469616C2F62617463686E6F726D2F09
:10E8E0006D756C5F313B626E5F696E697469616CF6
:10E8F0002F62617463686E6F726D2F6164645F3143
:10E900003B70726F6A656374696F6E312F4D61740D
:10E910004D756C3B70726F6A656374696F6E312FF1
:10E92000426961734164643B626E5F70726F6A65D5
:10E930006374696F6E312F62617463686E6F726D9C
:10E940002F6D756C5F313B626E5F70726F6A6563CD
:10E9500074696F6E312F62617463686E6F726D2FB0
:10E960006164645F310000000200000001000000EB
:10E970002000000016F6FFFF000000011400000058
:10E980001C0000001C0000001D0000003000000002
:10E9900002000000FFFFFFFF40000000A8F5FFFF9E
:10E9A000160000007265647563655F696E6974695D
:10E9B000616C2F4D61744D756C32000002000000D7
:10E9C00001000000400000006AF6FFFF00000001A7
:10E9D000140000001C0000001C0000001C000000CF
:10E9E0002800000002000000FFFFFFFF48000000B9
:10E9F000FCF5FFFF0F000000666C617474656E2FFC
:10EA0000526573686170650002000000010000003B
:10EA10004800000016F7FFFF000000011000000092
:10EA2000100000001B0000002400000038F6FFFF6B
:10EA3000140000006F75747075745F64656E7365A3
:10EA4000312F4D61744D756C000000000200000014
:10EA500010000000200000005AF7FFFF0000000136
:10EA600010000000100000001A000000200000004C
:10EA70007CF6FFFF12000000626F74746C656E65B7
:10EA8000636B322F4D61744D756C00000200000005
:10EA900010000000200000009AF7FFFF00000001B6
:10EAA000100000001000000019000000200000000D
:10EAB000BCF6FFFF12000000626F74746C656E6537
:10EAC000636B312F4D61744D756C000002000000C6
:10EAD0001000000020000000DAF7FFFF0000000136
:10EAE00010000000100000001800000024000000CA
:10EAF000FCF6FFFF160000007265647563655F69D0
:10EB00006E697469616C2F4D61744D756C310000D4
:10EB10000200000040000000480000000000160055
:10EB20001C001800170010000C0008000000000076
:10EB300000000700160000000000000114000000A3
:10EB40001400000017000000000000021C0000007C
:10EB50005CF7FFFF0D000000666C617474656E2F3A
:10EB6000436F6E737400000001000000020000009B
:10EB700072F8FFFF0000000110000000100000000C
:10EB8000160000003000000094F7FFFF2200000094
:10EB9000626F74746C656E65636B312F426961736B
:10EBA0004164642F526561645661726961626C658B
:10EBB0004F7000000100000010000000BEF8FFFFD1
:10EBC000000000011000000010000000150000000F
:10EBD00030000000E0F7FFFF22000000626F747455
:10EBE0006C656E65636B322F426961734164642F9B
:10EBF000526561645661726961626C654F700000B4
:10EC000001000000100000000AF9FFFF00000001F1
:10EC1000100000001000000014000000340000008C
:10EC20002CF8FFFF240000006F75747075745F642A
:10EC3000656E7365312F426961734164642F52655B
:10EC400061645661726961626C654F70000000001A
:10EC500001000000100000005AF9FFFF0000000151
:10EC60001000000010000000130000006C00000005
:10EC70007CF8FFFF5E000000626E5F6F7574707558
:10EC800074332F62617463686E6F726D2F6D756C73
:10EC90005F313B626E5F6F7574707574332F6261A4
:10ECA0007463686E6F726D2F6164645F313B6F7562
:10ECB000747075745F6C617965722F4D61744D75F8
:10ECC0006C3B6F75747075745F6C617965722F42FF
:10ECD00069617341646400000200000002000000EA
:10ECE00004000000E6F9FFFF000000011000000032
:10ECF00010000000120000003800000008F9FFFFBB
:10ED0000280000006F75747075745F6C61796572AE
:10ED10002F4D61744D756C3B6F75747075745F6CBD
:10ED2000617965722F42696173416464000000007B
:10ED300001000000020000003AFAFFFF000000019D
:10ED40001000000010000000110000008000000012
:10ED50005CF9FFFF73000000626E5F6F7574707581
:10ED600074322F62617463686E6F726D2F6D756C93
:10ED70005F313B626E5F6F7574707574322F6261C4
:10ED80007463686E6F726D2F6164645F313B6F7581
:10ED9000747075745F64656E7365332F4D61744D67
:10EDA000756C3B6F75747075745F64656E736533F5
:10EDB0002F52656C753B6F75747075745F64656E0A
:10EDC0007365332F4269617341646400020000007F
:10EDD0000400000008000000DAFAFFFF0000000154
:10EDE0001000000010000000100000004C000000A7
:10EDF000FCF9FFFF3D0000006F75747075745F646F
:10EE0000656E7365332F4D61744D756C3B6F757412
:10EE10007075745F64656E7365332F52656C753BF6
:10EE20006F75747075745F64656E7365332F4269B6
:10EE300061734164640000000100000004000000F0
:10EE400042FBFFFF00000001100000001000000066
:10EE50000F0000008000000064FAFFFF7300000054
:10EE6000626E5F6F7574707574312F626174636860
:10EE70006E6F726D2F6D756C5F313B626E5F6F757B
:10EE800074707574312F62617463686E6F726D2F68
:10EE90006164645F313B6F75747075745F64656E37
:10EEA0007365322F4D61744D756C3B6F7574707561
:10EEB000745F64656E7365322F52656C753B6F7558
:10EEC000747075745F64656E7365322F4269617327
:10EED000416464000200000008000000100000000F
:10EEE000E2FBFFFF00000001100000001000000026
:10EEF0000E0000004C00000004FBFFFF3D0000007E
:10EF00006F75747075745F64656E7365322F4D61D3
:10EF1000744D756C3B6F75747075745F64656E735A
:10EF200065322F52656C753B6F75747075745F64D4
:10EF3000656E7365322F426961734164640000003D
:10EF400001000000080000004AFCFFFF0000000173
:10EF500010000000100000000D000000280000005C
:10EF60006CFBFFFF1A000000626E5F657870616ED7
:10EF700064322F62617463686E6F726D2F6D756C91
:10EF80005F310000020000002000000010000000BF
:10EF900092FCFFFF000000011000000010000000C4
:10EFA0000C00000020000000B4FBFFFF1300000075
:10EFB000626E322F62617463686E6F726D2F6D7551
:10EFC0006C5F310002000000200000002000000003
:10EFD000D2FCFFFF00000001100000001000000044
:10EFE0000B0000002C000000F4FBFFFF1E000000DF
:10EFF000626E5F70726F6A656374696F6E322F62E2
:10F00000617463686E6F726D2F6D756C5F31000097
:10F010000200000020000000200000001EFDFFFF95
:10F020000000000110000000100000000A000000B5
:10F030002800000040FCFFFF1A000000626E5F65C0
:10F040007870616E64312F62617463686E6F726D87
:10F050002F6D756C5F310000020000002000000081
:10F060001000000066FDFFFF00000001100000001E
:10F0700010000000090000007800000088FCFFFF7D
:10F0800068000000626E5F696E697469616C2F626E
:10F09000617463686E6F726D2F6D756C5F313B626A
:10F0A0006E5F696E697469616C2F62617463686E0A
:10F0B0006F726D2F6164645F313B72656475636567
:10F0C000312F4D61744D756C3B72656475636531AC
:10F0D0002F426961734164643B626E312F626174D7
:10F0E00063686E6F726D2F6D756C5F31000000008C
:10F0F000020000002000000040000000FEFDFFFFB5
:10F1000000000001100000001000000008000000D6
:10F110008800000020FDFFFF7B000000626E5F6939
:10F120006E697469616C2F62617463686E6F726D71
:10F130002F6D756C5F313B626E5F696E69746961DA
:10F140006C2F62617463686E6F726D2F6164645FAF
:10F15000313B70726F6A656374696F6E312F4D61F8
:10F16000744D756C3B70726F6A656374696F6E3154
:10F170002F426961734164643B626E5F70726F6AB3
:10F18000656374696F6E312F62617463686E6F724C
:10F190006D2F6D756C5F31000200000020000000D3
:10F1A00040000000A6FEFFFF00000001100000006C
:10F1B000100000000700000028000000C8FDFFFF4D
:10F1C0001A000000626E5F657870616E64322F62B3
:10F1D000617463686E6F726D2F6164645F310000EB
:10F1E0000100000020000000EAFEFFFF0000000117
:10F1F00010000000100000000600000028000000C1
:10F200000CFEFFFF1A00000052656C755F333B6215
:10F210006E322F62617463686E6F726D2F61646409
:10F220005F31000001000000200000002EFFFFFF02
:10F2300000000001100000001000000005000000A8
:10F240002C00000050FEFFFF1E000000626E5F7089
:10F25000726F6A656374696F6E322F62617463687E
:10F260006E6F726D2F6164645F31000001000000F9
:10F270002000000076FFFFFF0000000110000000EA
:10F2800010000000040000002800000098FEFFFFAE
:10F290001A000000626E5F657870616E64312F62E3
:10F2A000617463686E6F726D2F6164645F3100001A
:10F2B0000100000020000000BAFFFFFF0000000175
:10F2C00010000000100000000300000028000000F3
:10F2D000DCFEFFFF1800000052656C753B626E316A
:10F2E0002F62617463686E6F726D2F6164645F3149
:10F2F00000000000010000002000000000001600D7
:10F3000018001400000010000C00080000000000AD
:10F3100000000700160000000000000110000000BF
:10F3200010000000020000002C00000038FFFFFF6A
:10F330001E000000626E5F70726F6A656374696FB1
:10F340006E312F62617463686E6F726D2F616464D9
:10F350005F310000010000002000000000001600E6
:10F360001C0018000000140010000C000000000039
:10F370000800070016000000000000011400000053
:10F380002000000020000000010000003800000004
:10F3900003000000FFFFFFFF09000000080000005D
:10F3A000ACFFFFFF1800000073657276696E675F3F
:10F3B00064656661756C745F617267735F303A3063
:10F3C0000000000003000000010000000900000030
:10F3D00008000000040000003C00000020000000C5
:10F3E0001800000004000000E0FFFFFF190000000B
:10F3F000000000190400040004000000F4FFFFFFF7
:10F4000009000000000000090C000C000B000000C7
:10F41000000004000C0000001600000000000016B0
:10F4200081B000F5E0700268914203D343681A444A
:10F43000914202D380680028F5D101B07047DFF80F
:10F440006817086890B94FF4805048604FF48032D4
:10F450004FF0FF308A60C86008610420DFF84C2755
:10F46000DFF84C374861C2F8BC010B6001207047DF
:10F4700001F1080313F0070F0EBF0023C3F10803C7
:10F4800003F007031944D21A8161C26042F00103FC
:10F490004B60091D28238B50DFF80C170A69C261E5
:10F4A00070472DE9FC4B074601F1080010F0070FEB
:10F4B0000FBF8946C0F1080000F0070001EB00090A
:10F4C00002F1080111F0070F06D002F10800C0F1A7
:10F4D000080000F0070002441546A5EB090009EBFF
:10F4E0000306A0EB030B43F00303C9F80430AE425C
:10F4F00028BF01F0FFF92879C10758BF01F0FAF9D8
:10F50000BBF1100F38BF01F0F5F9B869854207D19A
:10F51000F8685844F860BE6140F00100706050E146
:10F52000786985420AD1B8688344C7F808B07E611B
:10F530004BF00100706046F80BB042E1686800F0E3
:10F540000301012940F0AB80C008C0000190C00851
:10F550001F2839D8AC68D5F80C800090454508BF05
:10F5600001F0C8F9A54208BF01F0C4F96868009924
:10F57000C008C000B0EBC10F18BF01F0BBF9009983
:10F5800007F1280000EBC100844206D03A6994429A
:10F59000C0F08080E168A9427CD1A04506D10098E6
:10F5A0003968012282409143396075E0804506D078
:10F5B000386980456ED3D8F80800A8426AD1C4F8EB
:10F5C0000C80C8F8084067E0EC68D5F81880AC42B9
:10F5D0000CD0A8683969884222D3C168A94204BF07
:10F5E000A168A9421CD1C460A0601BE005F114020F
:10F5F000146834B905F1100214689CB101E01A4690
:10F60000146804F114031968002902BF04F11003FF
:10F6100018680028F3D139698A4228BF106001D2E6
:10F6200001F068F9B8F1000F36D0E96907F5987074
:10F6300000EB81000268954208D10460A4B9E86932
:10F640007968012282409143796025E038698045DC
:10F6500008D3D8F81000A84214BFC8F81440C8F85E
:10F66000104001E001F046F9B4B139698C4211D380
:10F67000C4F81880286928B1884226BF20618461B7
:10F6800001F038F9686938B13969884202D360619C
:10F69000846101E001F02EF901982D188344686817
:10F6A0004008400068604BF0010171604FEADB04E4
:10F6B00046F80BB01F2C23D807F1280000EBC40834
:10F6C0004546BBF1100F38BF01F014F9386820FA35
:10F6D00004F1C90705D4012101FA04F404433C6094
:10F6E00007E0D8F80800396988422CBF054601F0C8
:10F6F00001F9C8F80860EE60B560C6F80C8060E0FB
:10F700005FEA1B2008BF002123D0B0F5803F28BF4F
:10F710001F211ED2A0F58072120C02F00802904048
:10F72000A0F58051090C01F004018840A0F5804348
:10F730001B0CC2F10E0203F00203521AD21A9840B7
:10F7400002EBD032D01D2BFA00F101F0010101EBE8
:10F75000420107F5987202EB8100F16100227261AB
:10F7600032617A6822FA01F3DB0707D4012303FA36
:10F7700001F1114379600660B0611DE002681F2944
:10F780001DBF4908C1F119010BFA01F1594600E00A
:10F7900002465068C008C000584516D002F1100358
:10F7A000CC0F03EB8403490018680028F0D13869B6
:10F7B000834204D31E60B261F660B66001E001F0DE
:10F7C00099F809F10800BDE8F68B396990688A421A
:10F7D00028BF8842F3D3C6609660B060F260002014
:10F7E000B061EEE72DE9FE4F04468B46A5692E4633
:10F7F000904699463146FFF713FEA8F128020168AA
:10F80000406801EB000AAAF1270111F007000EBFC2
:10F810000021C1F1080101F007010AEB0100A0F18C
:10F820002F0706F11000874238BF374607F118004E
:10F8300001905946002000902046FFF719FE07F17D
:10F84000080010F0070F18BF01F054F81B20786073
:10F8500007F1080104F5E07090E80C5081E80C50C5
:10F86000C0F800B0C0F80480C0F80C908160019826
:10F87000009900E0001D07224260491C00F10802C7
:10F880005245F7D30129D8BF01F034F8B74200F050
:10F890009580BF1B301D311DC05940084000C85124
:10F8A00047F0010171604FEAD70BF751BBF11F0F11
:10F8B00021D804EBCB0000F12805A846102F38BF53
:10F8C00001F018F8206820FA0BF1C90705D40121CE
:10F8D00001FA0BF10843206006E0A868216988421C
:10F8E0002CBF804601F006F8AE60C8F80C60C6F880
:10F8F0000880F5606FE0380A08BF002123D0B0F51A
:10F90000803F28BF1F211ED2A0F58072120C02F08A
:10F9100008029040A0F58051090C01F004018840D4
:10F92000A0F580431B0CC2F10E0203F00203521A31
:10F93000D21A984002EBD032D01D27FA00F101F024
:10F94000010101EB420104EB8102002302F59870F2
:10F95000F16173613361626822FA01F3DB0707D456
:10F96000012303FA01F1114361600660B0611DE0FB
:10F9700002681F291DBF4908C1F1190107FA01F1E9
:10F98000394600E002465068C008C000B84216D0B0
:10F9900002F11003C80F03EB800349001868002828
:10F9A000F0D12069834204D31E60B261F660B56075
:10F9B00011E003B0BDE8F04F00F09CBF0BE02169FF
:10F9C00090688A4228BF8842F3D3C6609560B060D1
:10F9D000F2600020B06103B0BDE8F08F2DE9F04186
:10F9E000714F05463868884608B9FFF728FDB968A1
:10F9F00001EB08002F30491E20EA010188457DD225
:10FA000005F5D876B06828B1326889188A4275D26F
:10FA1000884273D300F08EFF01001CBF0C6811F107
:10FA2000010F6BD03068201805F5D872306053682C
:10FA3000984238BF18467060A86960BB286908B151
:10FA4000814200D22961316174610020F06105F1C9
:10FA50002802386868624FF0FF3028620020D260C8
:10FA6000926002F1080353611361801C1032202858
:10FA7000F5D34E48854208BFA4F1280228D055F896
:10FA8000040CC00805EBC002A2F108000A19121A02
:10FA9000283A01461CE005F5E070024600E0926855
:10FAA0007AB3136857683B449942F8D1137B1F0718
:10FAB00027D4AB691768BB4223D3D2F804C067448C
:10FAC000BB421ED2A444C2F804C0E868A969221847
:10FAD0002846FFF7CDFC1FE08068C0B10368934261
:10FAE000FAD1027B130712D4026801604368E4185C
:10FAF000446043462846BDE8F041D2E40020BDE81A
:10FB0000F0812A69914238BF29610A19E5E700238B
:10FB100022462846FFF766FEE8688045EED2A0EB55
:10FB20000800A969E86001EB0802AA6140F0010041
:10FB3000506048F00300486001F10800BDE8F08122
:10FB400038B4194B1A6882B94FF480525A604FF496
:10FB500080344FF0FF329C60DA601A610422134C4B
:10FB6000134D5A61C4F8BC211D6011F1400F17D22A
:10FB70008269AAB1C368283199420BD200F5E071BD
:10FB80000C68A24203D34D682C44A24202D3896878
:10FB90000029F5D1C16999423CBF4FF0FF31C161E5
:10FBA00032BC002070470000A42F002070260020E7
:10FBB0006859883C2DE9F84F00258946090AC9F1A2
:10FBC000000B08BF002323D0B1F5803F28BF1F23BF
:10FBD0001ED2A1F58072120C02F008029140A1F52C
:10FBE00080531B0C03F004039940A1F58044240CBE
:10FBF000C2F10E0204F00204D21A121BA14002EB61
:10FC0000D132D11D29FA01F303F0010303EB4203C2
:10FC1000074607F5987858F8230030B31F2B0FBF1D
:10FC20004C465C08C4F1190409FA04F4AC46594680
:10FC300000E064004268D208D200A2EB09028A42C6
:10FC400003D21100054600F06881426910304FEA86
:10FC5000D47B50F82B00002A1CBF82429446002817
:10FC6000E7D18B466046B0BBBDBB012000FA03F371
:10FC70005B00584203437868034000F04D815842CE
:10FC800003405B1E180B00F01000C340590901F03F
:10FC90000801CB409A0802F00402D3405C0804F04B
:10FCA00002040818E3401018C3F34006201830443B
:10FCB000F3401B1858F823000DE008464168C908B6
:10FCC000C900A1EB090159453CBF8B4605460169B6
:10FCD0000029F2D140690028F0D1002D00F01C81EC
:10FCE000B868A0EB0900834580F016813869854229
:10FCF000C0F010816868C008C00009EB0B018842A1
:10FD000018BF00F0F7FD05EB0906B54280F002814F
:10FD1000EC68D5F818A0AC420CD0A86839698842C4
:10FD200022D3C168A94204BFA168A9421CD1C46002
:10FD3000A0601BE005F11402146834B905F110024B
:10FD400014689CB101E01A46146804F114031968A0
:10FD5000002902BF04F1100318680028F3D13969A3
:10FD60008A4228BF106001D200F0C4FDBAF1000F32
:10FD700036D0E96908EB81000268954209D1046038
:10FD8000200014D1E86979680122824091437960AA
:10FD900026E03869824508D3DAF81000A84214BF7B
:10FDA000CAF81440CAF8104001E000F0A3FDBCB14D
:10FDB0003869844212D3C4F818A0286930B139696F
:10FDC000884226BF2061846100F094FD686938B1E3
:10FDD0003969884202D36061846101E000F08AFDE4
:10FDE000BBF1100F0CD2D94449F003006860291D03
:10FDF000281D50F8090040F0010041F8090088E092
:10FE000049F0030068604BF0010070604FEADB00CE
:10FE100046F80BB01F281DD807EBC00101F12804DC
:10FE2000396821FA00F2D207A34605D4012202FA6A
:10FE300000F00843386006E0A068396988422CBFAA
:10FE4000834600F057FDA660CBF80C60C6F808B0FA
:10FE5000F4605EE05FEA1B2008BF002123D0B0F50C
:10FE6000803F28BF1F211ED2A0F58072120C02F025
:10FE700008029040A0F58051090C01F0040188406F
:10FE8000A0F580431B0CC2F10E0203F00203521ACC
:10FE9000D21A984002EBD032D01D2BFA00F101F0BB
:10FEA000010101EB4201F16100227261326108EB54
:10FEB00081007A6822FA01F3DB0707D4012303FAF1
:10FEC00001F1114379600660B0611DE002681F29ED
:10FED0001DBF4908C1F119010BFA01F1594600E0B3
:10FEE00002465068C008C000584518D002F11003FF
:10FEF000CC0F03EB8403490018680028F0D138695F
:10FF0000834204D31E60B261F660B66001E000F087
:10FF1000F1FC13E100F0EEFC0DE18B46A3E639693C
:10FF200090688A4228BF8842F1D3C6609660B0606C
:10FF3000F2600020B061ECE72DE9F84F06468846F4
:10FF4000716848420140491E080B00F01000C14092
:10FF50004A0902F00802D1408B0803F00403D9409B
:10FF60004D0805F002051018E9401818C1F34004C7
:10FF7000281806F5987A2044E14009185AF821100B
:10FF80004868C008C0000D46A0EB080909E001461A
:10FF90004868C008C000A0EB080048453CBF814647
:10FFA0000D4608690028F2D149690029F0D130696D
:10FFB0008542C0F0BE806868C00808EB090BC0002D
:10FFC000584518BF00F096FC05EB080085420090EC
:10FFD00080F0AF80EF68AC69AF420CD0A86831699F
:10FFE000884222D3C168A94204BFB968A9421CD182
:10FFF000C760B8601BE005F11402176837B905F156
:020000040801F1
:10000000100217689FB101E01A46176807F1140340
:100010001968002902BF07F1100318680028F3D1FE
:1000200031698A4228BF106001D200F063FC002CC5
:1000300031D0E9690AEB81000268954208D1076076
:100040008FB9E8697168012282409143716022E0B2
:100050003069844205D32069A84214BF67612761D3
:1000600001E000F047FCB7B13069874211D3BC61B1
:10007000286930B13169884226BF3861876100F054
:1000800039FC686938B13169884202D37861876187
:1000900001E000F02FFCB9F1100F0BD24BF0030080
:1000A0006860291D281D50F80B0040F0010041F840
:1000B0000B003DE048F00301696049F00100291D93
:1000C00041F80800009840F80990D6F808804FEAF7
:1000D000D80BBBF1200F28BF00F00CFCB8F1000FCB
:1000E00022D006EBCB00776900F12804A246B8F1D4
:1000F000100F38BF00F0FEFB306820FA0BF1C90783
:1001000005D4012101FA0BF10843306006E0A06834
:10011000316988422CBF824600F0ECFBA760CAF828
:100120000C70C7F808A0FC60C6F8089000987061D1
:1001300004E000F0DFFB0020BDE8F28F05F10800CD
:10014000BDE8F28F2DE9FE4F0546AFF30080F52D97
:10015000DFF89C6780F004810B2D31BF10250B3533
:10016000ED08ED003068EC08E04010F0030F46D0D9
:10017000C04300F00100041906F1280000EBC40898
:10018000E700D8F808506868C008C000B84218BF37
:1001900000F0B0FBD5F80890454508BF00F0AAFB79
:1001A0004D4508BF00F0A6FB6868C008C000B84213
:1001B00018BF00F09FFBC84507D13168012000FA45
:1001C00004F421EA040434600DE03069814508D369
:1001D000D9F80C00A84204D1C8F80890C9F80C80DE
:1001E00001E000F087FB47F003006860291D281D2F
:1001F00005F10804C05940F00100C851F8E0B168A9
:10020000A94280F0BE80002800F0A1804FF00108D4
:1002100008FA04F1490000FA04F4484201430C4092
:1002200060420440641E200B00F01000C4406109CD
:1002300001F00801CC40A20802F00402D440630897
:1002400003F002030818DC401018C4F34007181824
:100250003818FC40241806F1280000EBC40AE70017
:10026000DAF80890D9F80400C008C000B84218BFF6
:1002700000F040FBD9F808B0D14508BF00F03AFBC8
:10028000D94508BF00F036FBD9F80400C008C0000B
:10029000B84218BF00F02EFBDA4506D1316808FAE3
:1002A00004F421EA040434600DE03069834508D386
:1002B000DBF80C00484504D1CAF808B0CBF80CA014
:1002C00001E000F017FB45F00300C9F804007F1BB4
:1002D00009F1040147F00100485109EB05000190C4
:1002E000C751B4684FEAD40ABAF1200F28BF00F012
:1002F00001FB34B3CDF800A006F12800756900EBCE
:10030000CA0AD346102C38BF00F0F4FA31680098BE
:1003100021FA00F2D30704D408FA00F00843306051
:1003200007E0DAF80800316988422CBF834600F004
:10033000E1FACAF80850CBF80C50C5F808B0C5F877
:100340000CA0B76009F108040198706150E0706872
:10035000C0B329463046FFF7EFFD040011D047E057
:1003600015F1400F28BF4FF0FF350AD20B35ED08CD
:100370007068ED0028B129463046FFF71BFC0400E9
:1003800036D1B068A8421DD3411B726910290AD327
:1003900050197061B16041F001034360415045F074
:1003A000030555600BE00021B1607161131D40F041
:1003B00003015160111D095841F00101195002F16A
:1003C000080415E0F06885420DD2401BB169F06069
:1003D0004A19B26140F00100506045F003054D60DC
:1003E00001F1080404E029463046FFF7F7FA044615
:1003F000AFF300802046FFF7EEBA002800D1704727
:100400002DE9FC47A0F10805AFF30080DFF8E064B8
:1004100032699542C0F05982686800F003010129F1
:1004200000F05382C1084FEAC109C10705EB090872
:1004300039D42C6810F0030F00F049826042054463
:100440009542A144C0F041827069854200F0C780A6
:10045000E408202C5ED2D5F80CA0AF68554508BF43
:1004600000F048FABD4208BF00F044FA6868C008CE
:10047000C000B0EBC40F18BF00F03CFA06F1280032
:1004800000EBC400874205D031698F423FD3F96841
:10049000A9423CD1BA452CD13068012101FA04F4BB
:1004A00020EA04043460454580F00F82D8F8044007
:1004B000E00740F10A82A00700F16881B069804539
:1004C00040F0A080F068B5618144C6F80C9049F016
:1004D000010068607069854202D100207061B060DF
:1004E000F069484580F0F38100213046FFF728FB92
:1004F000EDE1824506D03069824508D3DAF808007C
:10050000A84204D1C7F80CA0CAF80870CBE700F0E5
:10051000F1F9C8E7EC68AF69AC420BD0A86890422B
:1005200023D3C168A94204BFA168A9421DD1C460F8
:10053000A0601CE005F114031C6834B905F1100338
:100540001C68A4B101E063461C6804F1140CDCF8DB
:100550000010002902BF04F1100CDCF80000002894
:10056000F1D1934228BF196001D200F0C3F9002FE6
:1005700099D0E96906F5987000EB81000268954210
:1005800009D10460200011D1E8697168012282401C
:100590009143716087E73069874205D33869A84283
:1005A00014BF7C613C6101E000F0A4F9002C3FF431
:1005B0007AAF31698C42AAD3A761286928B18842F1
:1005C00026BF2061846100F095F9686900283FF436
:1005D0006AAF316988429AD36061846163E798F8B1
:1005E000040000F0030003287FF45DAFC6F8089014
:1005F00049F00101D8F8040040084000C8F80400A0
:1006000069600AE0706980450AD1B068756181440B
:10061000C6F8089049F00100686045F8099056E175
:10062000E408E400A144E408202C3AD2D8F80CA055
:10063000D8F80870D04508BF00F05CF9B84508BF8D
:1006400000F058F9D8F80400C008C000B0EBC40F9F
:1006500018BF00F04FF906F1280000EBC4008742F4
:1006600007D031698F42C0F08480F968414540F07D
:100670008080BA4507D13068012101FA04F420EAEC
:100680000404346077E0824506D031698A4570D32E
:10069000DAF8080040456CD1C7F80CA0CAF8087019
:1006A00069E0D8F80C40D8F8187044450DD0D8F857
:1006B00008003169884222D3C168414504BFA1685E
:1006C00041451CD1C460A0601BE008F1140214680D
:1006D00034B908F1100214689CB101E01A4614689C
:1006E00004F114031968002902BF04F1100318680B
:1006F0000028F3D131698A4228BF106001D200F08E
:10070000F9F8002F37D0D8F81C1006F5987000EBD8
:100710008100026890450AD10460200012D1D8F807
:100720001C007168012282409143716023E03069AE
:10073000874205D33869404514BF7C613C6101E0C4
:1007400000F0D8F8BCB131698C4212D3A761D8F857
:10075000100028B1884226BF2061846100F0CAF8E9
:10076000D8F8140038B13169884202D360618461DD
:1007700001E000F0BFF849F00100686045F8099019
:10078000706985420BD1C6F80890A0E06408640047
:10079000C8F8044049F00100686045F809904FEA44
:1007A000D907202F22D206F1280000EBC704A0466B
:1007B000B9F1100F38BF00F09DF8306820FA07F14A
:1007C000C90705D4012101FA07F70743376006E09E
:1007D000A068316988422CBF804600F08BF8A56084
:1007E000C8F80C50C5F80880EC6070E05FEA19208A
:1007F00008BF002123D0B0F5803F28BF1F211ED2A3
:10080000A0F58072120C02F008029040A0F5805111
:10081000090C01F004018840A0F580431B0CC2F1D3
:100820000E0203F00203521AD21A984002EBD032A1
:10083000D01D29FA00F101F0010101EB420106F59A
:10084000987202EB810000226A612A61E961726894
:1008500022FA01F3DB0707D4012303FA01F1114364
:1008600071600560A8611DE002681F291DBF49086D
:10087000C1F1190109FA01F1494600E00246506848
:10088000C008C000484526D002F11003CC0F03EB8E
:100890008403490018680028F0D13069834204D3EA
:1008A0001D60AA61ED60AD6001E000F023F8306AE0
:1008B000401E30620BD1D6F8C80100E080680028E5
:1008C000FCD14FF0FF30306201E000F013F8AFF3DD
:1008D0000080BDE8F387316990688A4228BF88426A
:1008E000E3D3C5609560A860EA600020A861DEE7F8
:1008F00070260020012000F033B80B78012B70B572
:1009000005460C460AD140684E6803687168DB688A
:100910009847686803683146DB6898470023686831
:100920006360C4E90433237003682146DB68BDE8D3
:10093000704018470749086808B10020704706480A
:10094000C008C00008600549C908C900091A01604B
:10095000704700BFD0300020FF650020F89A0020CB
:1009600080B500F007F8024A11001820ABBEFBE783
:100970002600020010B500F013F802000023DB434C
:1009800000241068984203D011000220ABBE14600E
:100990005068984203D0111D0220ABBE546010BDB8
:1009A0000148704700000000040100202E48006844
:1009B000704730B50D4683B0044641F6D83100F09B
:1009C0006BFF20462946462200F07CFF04F5267581
:1009D0004FF0FF3028614FF49670A8800020E88027
:1009E00004F1480000F0D4FF01F01EFA04F1880180
:1009F0001020642301F1800213800B8053804B8010
:100A000093808B80D380CB800831401EF2D1208828
:100A1000642110FB01F12980684601F043FA134874
:100A20001349019008680290694604F5916001F04D
:100A300040FA18B94FF0FF3003B030BD41F6F8105E
:100A4000204401F0E3FA41F68421601801F082FBB2
:100A500041F6B02004F525726421204401F0FEFB2C
:100A6000002003B030BD00002401002090010008E8
:100A70008C01000830B400F54773B3F9004094428C
:100A800011DA5B68D0F894525B1E03F01F0300EB91
:100A9000C30404F5497318682D1AA942A4BFB3F919
:100AA0000400904202DB30BC0120704730BC0020C3
:100AB000704778B400F54771B0F91840B1F90030CB
:100AC000A34200F5257217DB4C68166800EBC405DD
:100AD00005F54974761EA380266000F224404B6819
:100AE0005B1C03F01F034B60046813689C42BCBF8F
:100AF000002484801433036000200880B2F92000B1
:100B0000002802DD002111849181002072BC704711
:100B10002DE9F24F2DED108BA4B0B1F900108046F5
:100B200000EE901A9FEDE30AF8EEE00A349860EECA
:100B3000800ACDED080A08F58763B0F902103498F1
:100B400000EE901AF8EEE00A60EE800ACDED090A98
:100B500008F23442B0F90410349800EE901AF8EE1E
:100B6000E00A20EE800A8DED0A0ADFEDD30AB0F923
:100B70000610349800EE101AB8EEC00AC0EE200A33
:100B8000CDED0B0ADFEDCC0AB0F90810349800EE79
:100B9000101AB8EEC00AC0EE200ACDED0C0ADFED47
:100BA000C60AB0F90A1000EE101AB8EEC00AC0EE7C
:100BB000200ACDED0D0A08F5866108A801F052F96A
:100BC00008F2444308F5886208F23C4109A801F0A4
:100BD00049F908F58A6308F24C4208F589610AA8C8
:100BE00001F040F908F224449FEDB48A94ED030A21
:100BF00094ED061AD4ED090A20EE000A01EE010A6E
:100C000000EEA00A01F01AFC20EE08BABDEECB0AF5
:100C10008DED040A08F28A25049868809DED080A83
:100C2000DDED081A9DED091ADDED0A0A20EE210A14
:100C300001EE010A00EEA00A01F000FC60EE08BA25
:100C4000BDEEEB0A8DED010A08F25C4301982880A5
:100C500008F58B6208F254410BA801F003F918AEB5
:100C600008F58D6308F2644208F58C610CA801F068
:100C7000F9F808F2744308F58E6208F26C410DA889
:100C800001F0F0F894ED0C0A94ED0F1AD4ED120A6D
:100C900020EE000A01EE010A00EEA00A01F0CEFBF0
:100CA0009DED0C1ADDED0D0AB0EE40CA9DED0B0A6C
:100CB00020EE000A01EE010A00EEA00A01F0BEFBE0
:100CC000206BB0EE40DA01F0D1FBCDE91801FDEE6A
:100CD000CCCAE06B01F0CAFBC6E90201A06C01F0CE
:100CE000C5FBC6E90401E06801F0C0FBCDE91201D3
:100CF00012AEA06901F0BAFBC6E902019FED70AB2C
:100D0000606A01F0B3FBC6E9040100221EA80021BD
:100D100000230EC00EC01EA900919FED6B0B12ABFD
:100D200018AA08F1480102A800F0FCFE02A801F090
:100D3000C1FBD8F8480090ED008B806890ED00FB77
:100D400090ED02EB90ED049B53EC182B51EC1E0B35
:100D500001F0CAFB06460F4653EC1F2B51EC190B52
:100D600001F0C2FB02460B463046394601F094FCC6
:100D700053EC1A2B01F0B8FB01F006FD00EE100A4F
:100D800001F036FDF0EE40DA53EC182B51EC180B65
:100D900001F0AAFB06460F4653EC192B51EC190B38
:100DA00001F0A2FB32463B4601F050FD53EC1A2BFA
:100DB00001F09AFB0022DFF8C43A01F047FD01F090
:100DC000E3FC00EE900ACDED000A53EC1E2B51EC33
:100DD000190B01F089FB06460F4653EC182B51EC1A
:100DE0001F0B01F081FB32463B4601F02FFD53EC17
:100DF0001A2B01F079FB01F0C7FC00EE100ADDEDC3
:100E0000000A01F0DFFDB0EE409A1DEE900A01F0FD
:100E10002DFB9FEDBB8B53EC182B01F065FBDFF82E
:100E2000602ADFF8603A01F007FE01F02DFF064668
:100E300019EE100A01F01AFB53EC182B01F054FBC9
:100E4000DFF83C2ADFF83C3A01F0F6FD01F01CFF28
:100E50005A38029010F1B40FBCBF00F5B470029084
:100E6000AE8041F6D0110298E88008EB0107B8F98E
:100E700010004142B142BFBF86420298B8F9161035
:100E8000884225DA4F200790B8F80812491CA8F8C4
:100E90000812786A04281DD2B8F94200C642A1BFE0
:100EA000B042B8F944000299884213DB4FF0010ABE
:100EB00012E000BF000000396F1283420000C842F8
:100EC00000000000000000407B14AE47E17A943F30
:100ED000582007904FF0000A08F20A21B5F90800DF
:100EE000B8F8082221F8102041F69C2040440090D8
:100EF00008F5457901986428A4BF0499642972DA39
:100F0000386A401C012838620FD10020786241F60F
:100F1000F810404401F00AF908F5916001F06DF80D
:100F200041F68420404401F085F9796A042957D2BA
:100F30000B983860F0EE4D0A0D98786087ED02BA94
:100F400041F6F81087ED03CAB0EE6B0A404401F099
:100F50006BF841F6842087ED040A08A9404401F0AB
:100F600009F987ED050A9DED020AB8EEC00A87ED82
:100F7000060A009890ED000A3BEEC00A87ED070ACA
:100F80000098C0ED00BAB9F90800042821DDBAF1D3
:100F9000000F1ED00122394608F5916000F0BFFF16
:100FA00008F59061DFED580A4A6A116991ED010A6E
:100FB000786AB4EE600AF1EE10FA04DB401C0428F3
:100FC000786214D30CE090B1042810D2002078622B
:100FD0000DE00022394608F5916000F0A0FF06E020
:100FE0004FF0000A03E0386A08B10021396208F1C5
:100FF00088010498B5F9082021F81200B5F90820F5
:10100000019B08F5847008F5257620F8123008F564
:10101000C470B5F908301CEE902A20F813204FF068
:10102000000BB5F90820F388521F02F03F0230F898
:1010300012209A1AF2801CEE900A8218F28046F270
:10104000676012B212FB00F0401400EBD07000B2E7
:101050000590B5F90830B8F90000B2881B1A03F002
:101060003F0331F81310511AB18004984118B18030
:1010700009B2B8F9000091FBF0F008EE100A3498BC
:10108000616DB0F90600002902DD002809D501E0F4
:10109000002806DDA165C4F854B008F590623168F7
:1010A0005160616D4018606508F59060019AB0F973
:1010B0000010462A2ADB491C0180B9F90820002AC1
:1010C00028DDBAF1000F25D0B8F93E20B6F9083076
:1010D0009A4211DBB8F93C300AB29A420CDA09B2F2
:1010E000022917DD31684068091A042912DAA16D56
:1010F000DFF8940781420DDB4046FFF7DAFC09E098
:1011000000000000008066409A99593F0029C8BF3E
:10111000A0F800B0B5F90810C91E08F5847201F0F6
:101120003F01308932F81120821A328101988218E9
:10113000328108F5C472708932F81110411A718138
:101140001CEE900A411871810199B6F9200082299C
:101150001CDB316818B9716289F804000AE0B06AD2
:10116000081A062806DD716289F804B0A6F820B0D6
:10117000A6F80CB03068318CB062019AA2F164001C
:101180004118B08D3184401CB08538E0002836DD30
:10119000049A642A33DA60282FDB3368716A5B1A99
:1011A000022B2ADD46F2610210FB02F2901500EBE1
:1011B000D07000B20A28B6F90C10A8BF09208142ED
:1011C00002DAB0813068306141F27B41B6F920002B
:1011D00010FB01F1C81400EBD07000B2B8F91A107E
:1011E00008308142B8BF08463168401808F52571BB
:1011F000CA699042B8BF1046F061A6F820B0D9F88D
:101200000000B6F92C2008EB4001B1F9C202131A14
:101210000393A1F8C222D9F80000401CC9F80000CD
:101220002828A8BFC9F800B099F8040001280AD1FD
:1012300003990A29A4BF09200390B6F90C00039969
:101240008142B8BF0390B8F9040001998842BEBF3B
:101250000846B8F90610884242DAB6F918108842F2
:101260003EDB052205214046FFF704FC002837D16C
:101270000198316830837161019A019B643AAF2B08
:1012800008DA0D204243DFF8040682FB00EC4FEA47
:101290006C101CE0C82B12DAA3F1AF00C0EBC00049
:1012A000DFF8E83580FB03C3DB1003EBD3730D33AA
:1012B0005A43DFF8D80582FB00E0401107E002EB5B
:1012C00082008000DFF8C42580FB02325011B8F99B
:1012D0001A2000EBD0708242B8BF10464018F0616F
:1012E0003068F169884208BFA6F818B0306828282D
:1012F000C0F2B282B8F90210049AB9F9080091421A
:10130000C0F20D81401CA9F8080000B205280DD1DB
:10131000009A3068136900F164018342116105DAB3
:1013200041F6B02108EB010000F0A4FF99F8040099
:1013300038B93168B06A091A1929BCBF012189F886
:101340000410B8F9380050B10298B8F91610884264
:1013500005DA01984F28C8BFCDF810B002DCB9F902
:101360000800049008F20A22B5F90800014632F894
:1013700011301093A1F1110C0CF03F0C32F81C202D
:101380009A1A0A2A08DD4FEA620C6FF0050302EB95
:101390009C72A3EBA20205E0C2F11102531002EB12
:1013A00093729210B8F92E30ADF81A30BDF91AC008
:1013B000B9F90830ACEB020C634545DBD6F800E028
:1013C000AEEB03035B1C0F93D9F80C305B1E03F0EC
:1013D0001F0C08EBCC0303F5497ECDF838E0DEF8AE
:1013E0000030DDF83CC0B8F932E0ACEB030CACF1F6
:1013F000010CF445A4BFB8F934E0E64524DBDDF880
:1014000038C0BCF904E0B8F92CC0ACEB0202964538
:10141000A2BF5A1CD6F81CC06245A2BFB4F9042072
:10142000B8F936C062450FDBA2689342BCBF0F9B80
:101430009A4209DA401C00F03F0028813068401CC5
:10144000306024B0072011E208F54573B3F9082095
:10145000042A5ADD33689B1A5B1C0F93D9F80C30B1
:101460005B1E03F01F0308EBC30C0CF549730E93CE
:10147000DDF83CC01B68B8F932E0ACEB030CACF112
:10148000010CF445A4BFB8F934E0E6453DDBDDF8D6
:1014900038C0BCF904E0ADF818E0F446B8F92CE027
:1014A000F445A2BFB9F90890BDF91AC0E145A1BF42
:1014B000BDF918909144B8F930C0E14525DB08F238
:1014C0000A2E891A01F03F01DDF840C03EF81110E4
:1014D000ACEB010102EBD279B1EB690F15DAB4F98B
:1014E0000410B8F9369049450FDBA1688B42BCBFA8
:1014F0000F9B994209DA401C00F03F0028813068B8
:10150000401C306024B00820B0E1042A0EDB3068B3
:1015100000990F3048600099A1F80AB006E0002851
:10152000C4BF4046FFF7C5FACDF810B03168226855
:101530009142BEBFB4F904000199884202DAA18049
:101540003068A0603068F1698842BEBF0298B8F97F
:1015500016108842C0F2EC80DDF81090B9F1000F4F
:1015600040F3E680039800286FDD07994F290AD1E0
:10157000BAF1000F83461CD0B8F9400000EBD070E0
:101580000BEB600B15E0B8F916000299884210DBEE
:10159000786A70B99DED030AB8EEC00A10EE100A21
:1015A00000F064FFBA4ABB4B00F09EFF01F06CFBF9
:1015B0008346B8F908000599814210DAB8F90000AD
:1015C00058448145C0F2A3802889401C00F03F00A8
:1015D00028813068401C306024B0032046E1B8F90F
:1015E00000105944894557DA059AB8F90A309A42E9
:1015F00080F28D80101A00EE900AF8EEE00A9FED5E
:101600009D1A60EE810ADFED9C1AB8EEC80AC0EEA2
:10161000A11AF0EE400A40EE610ABDEEE00AB8F908
:101620000C2010EE100A904271DA01EBD171B9EB87
:10163000610F6CDB2889401C00F03F002881306876
:10164000401C306024B0042010E107984F2807D1D7
:10165000BAF1000F18BFB8F940B003D1786A08B1E9
:10166000B8F93AB0B8F90800059981420FDAB8F92B
:101670000000584481454ADB2889401C00F03F00A7
:1016800028813068401C306024B00120EEE0B8F9B9
:101690000010594489450ADB2889401C00F03F00AE
:1016A00028813068401C306024B00C20DEE0059AB0
:1016B000B8F90A309A422ADA101A00EE900AF8EEC7
:1016C000E00A9FED6C1A60EE810ADFED6B1AB8EE4E
:1016D000C80AC0EEA11AF0EE400A40EE610ABDEE63
:1016E000E00AB8F90C2010EE100A90420FDA01EB74
:1016F000D171B9EB610F0ADB2889401C00F03F0073
:1017000028813068401C306024B00220AEE0B8F977
:1017100000100498123188420ADB2889401C00F02E
:101720003F0028813068401C306024B009209DE0D3
:10173000B6F90800B8F922108842A2BF0298B8F999
:1017400016108842A2BF606D42F21171884213DB0D
:10175000B8F92620B8F924104046FFF78BF9012884
:101760000AD12889401C00F03F0028813068401CC5
:10177000306024B0102079E000983168026991420D
:1017800025DA41F6B02108EB0104349A019920468C
:1017900000F0ACFD01281AD1204600F0FFFD002822
:1017A0000ADD2889401C00F03F0028813068401C79
:1017B000306024B00A2059E00098316842689142B4
:1017C00005DA418B418100983168491EC16000985B
:1017D0003168426891423FDA3498B0F9081001F557
:1017E0001C51103144F62160814203D300980189D5
:1017F000491C06E00099B1F90800002802DD0098B4
:10180000002101810099B1F90800042824DBB5F911
:10181000081008F20A22084632F810300F3800F09B
:101820003F0032F810001B1A0C2B15DC009AB2F99D
:101830000A00C82810DB009B3268D868121A921F71
:10184000092A09D2491C01F03F0129813068401C56
:10185000306024B0052009E02889401C00F03F00DA
:1018600028813068401C306024B00020BDEC108B13
:10187000BDE8F28FCDCC4C3E000048430000F0BFE5
:10188000182D4454FB210940A18601001F85EB510E
:101890009A9999999999E93F002201F013BA202960
:1018A00002460DD00023101D01E05B1C1C30D2F855
:1018B00074C0634504D2D0F814C08C45F5D170478C
:1018C0000020704762B38B0708D0521E11F8013B0D
:1018D00000F8013B00F024808B07F6D1830740F02D
:1018E000208000BF103A07D330B4B1E83810103A66
:1018F000A0E83810F9D230BC530724BFB1E8081073
:10190000A0E8081044BF51F8043B40F8043BD2075C
:1019100024BF31F8022B20F8022B44BF0B78037050
:101920007047121F17D35B0009D151F8043B20F810
:10193000023B1B0C121F20F8023BF6D20BE051F8C1
:10194000043B00F8013B1B0A20F8023B1B0C121F52
:1019500000F8013BF3D238BF121D521E24BF11F80C
:10196000013B00F8013BF8D8704700F5805210B5F4
:101970005368B3F5806F09DA946800EB8300214463
:101980000133446091605360002010BD0120FCE7EA
:1019900010B50446102001F0AFF908B101F0BEF90E
:1019A00020600022DFF84C34C0E9002381689FEDFD
:1019B0000C0B81ED000B816881ED020B806880EDDE
:1019C000040B84ED020B84ED040B84ED060B84ED17
:1019D000080B84ED0A0B84ED0C0BA26310BD000014
:1019E00000000000000000002DE9F0412DED108BFB
:1019F0000D46174682B00646984695ED009B97ED3A
:101A000000ABB0EE408AF0EE608A51EC1A0B53EC5A
:101A1000192B00F041FECDE9000195ED02BBD7E99D
:101A2000020153EC1B2B00F037FE41EC1D0BD7E9F4
:101A3000040195ED04CB53EC1C2B00F02DFEB46B90
:101A400041EC1E0B6CB3DDE9002351EC180B81F067
:101A5000004101F027FD41EC1F0B5AD2DDE90001E6
:101A600053EC182B01F01EFD53D251EC1F0B53EC1D
:101A70001D2B01F017FD4CD251EC1D0B53EC182B14
:101A800001F010FD45D251EC1F0B53EC1E2B01F061
:101A900009FD3ED251EC1E0B53EC182B01F002FD58
:101AA00037D2601C01F016FD41EC180B204601F006
:101AB00011FD53EC192B00F017FD53EC1A2B00F01D
:101AC000C5FE53EC182B00F0B7FFC5E90001204616
:101AD00001F000FD53EC1B2B00F006FDD7E90223BB
:101AE00000F0B4FE53EC182B00F0A6FFC5E902018C
:101AF000204601F0EFFC53EC1C2B00F0F5FCD7E97D
:101B0000042300F0A3FE53EC182B00F095FFC5E969
:101B100004014445BCBF641CB46302B0BDEC108B2F
:101B2000BDE8F0812DE9FC412DED088B04460D4602
:101B30009846B0EE40AAF0EE60AA9AB016469FED25
:101B4000AE0B42F2107305F108012846FFF74CFF77
:101B5000D6E90401D5E9062300F09EFD9FEDA8BB60
:101B600053EC1B2B00F0C0FC53EC1A2B00F0BCFC18
:101B7000D5E9042341EC120BD6E90201B0EE428A0A
:101B8000F0EE628A00F088FD53EC1B2B00F0ACFCF9
:101B900053EC1A2B00F0A8FCD5E9022341EC110B01
:101BA000D6E90001B0EE482AF0EE682AB0EE418A8C
:101BB000F0EE618AB0EE429AF0EE629A00F06CFDAF
:101BC00053EC1B2B00F090FC53EC1A2B00F08CFC18
:101BD00041EC100BB0EE492AF0EE692AB0EE481A3B
:101BE000F0EE681A0EA801F039F902462968684635
:101BF00001F0ECF92868694601F07DFC012102A89A
